:020000040800F2
:1000000000A00020852F010859DD0008B91F010854
:1000100057DD000855DD000853DD00080000000032
:1000200000000000000000000000000051DD00089A
:100030004FDD0008000000004DDD0008476A0008A1
:10004000ED2F0108ED2F0108ED2F0108ED2F01081C
:10005000ED2F0108ED2F0108ED2F0108ED2F01080C
:10006000ED2F0108ED2F0108ED2F0108ED2F0108FC
:10007000ED2F0108B14800087BD80008ED2F0108DA
:10008000ED2F0108ED2F0108ED2F0108ED2F0108DC
:10009000B9DD0008ED2F0108ED2F0108ED2F010853
:1000A000E9F8000815F90008ED2F010825F9000806
:1000B00009F90008F9F80008ED2F0108ED2F0108F3
:1000C000ED2F0108ED2F0108ED2F0108ED2F01089C
:1000D000ED2F0108D5FA0008C9FA0008BDFA00089A
:1000E000556A0008ED2F01083DDD0008ED2F0108DD
:1000F000ED2F0108ED2F0108ED2F0108ED2F01086C
:10010000000000000000000000000000ED2F0108CA
:10011000ED2F0108ED2F0108ED2F0108ED2F01084B
:10012000ED2F0108ED2F0108ED2F0108ED2F01083B
:10013000ED2F0108ED2F0108000000000000000075
:10014000ED2F0108ED2F0108ED2F01080000000040
:10015000000000000000000000000000000000009F
:100160000000000000000000ED2F0108ED2F010845
:10017000ED2F01080000000000000000000000005A
:0801800000000000ED2F010852
:100188002DE9F04F2DED028B6B4F6C4B3B60AFB000
:1001980000237B6010F0AAF818B910F0C9F80AF02B
:1001A800E5F80AF09DF9664B664C1A7842F00102B0
:1001B8001A70654A4FF47001C2F88810002209923B
:1001C8000A92226842F4803222600493236803F47E
:1001D80000330A93099B013309930A9B1BB9099BB6
:1001E800B3F5A04FF2D1236813F4003318BF0123ED
:1001F8000A930A9B012B76D0534E544BF360636AE3
:10020800BB60636ADFF874B1DFF87491DFF874815A
:1002180043F080736362636943F4FC032EAD63614A
:1002280003238DF86A3041F6FF7325F8503D4FF0EF
:100238009040294604F02EFC4FF6FF734448ADF871
:100248006830294604F026FC5846294604F022FC6A
:100258004048294604F01EFC3F48294604F01AFC91
:1002680029463E4804F016FC28460BF08FFD1A9BE1
:100278003B4AB3FBF2F33B4A13603B4B3B4A4FF01C
:10028800000AC3F800A03A4B5A60F02286F82320EF
:100298000722C3F808A0374E1A60D9F80830C8F802
:1002A80000300FCEAE46AEE80F00636996E8030053
:1002B80043F400238EE803006361636943F4002379
:1002C8006361636943F4002363614FF40043CBF82F
:1002D80018304FF48043CBF818304FF40053CBF864
:1002E8001830103E50E0244B12221A606368636095
:1002F80063686360636843F480636360636823F4DE
:100308007C136360636843F4E8136360236843F015
:100318008073236022680B4B9201FBD55A6822F048
:1003280003025A605A6842F002025A60636803F096
:100338000C03082BFAD15FE7880100201B9C0008FA
:10034800282F00200010024000ED00E00005FA050B
:1003580000040048000C0048001000480014004841
:1003680040420F00381300203C1300203F190100C1
:1003780010E000E0B07301080020024000080048C7
:1003880094240020342400200AF1040155F80A00BE
:1003980029440AF1080A04F07DFBBAF1180FF3D1D9
:1003A800642006F042FBA022B648002114F037FE74
:1003B800E369B54A43F00303E361A36943F4843373
:1003C800A361636943F42023636102F1B00C937B5A
:1003D800506892F80FE003F00701DB0800EB830395
:1003E8008900186A4FF00F0A0EFA01FE0AFA01F1A5
:1003F80020EA01011962196A10324EEA01016245C8
:100408001962E4D10023DFF8B4A20AF10C0200213A
:10041800995401330B2BF6D1FF239C4A8AF81730E5
:100428008AF818308AF819308AF81A30984BDFF8A9
:1004380090B21360974A03930420107058463022F4
:1004480014F0EDFD142202218BF800208BF8241003
:1004580001229149039B8BF8182099F805B081F87F
:1004680000B0A3F5EE71CAF81C108C49D8F80080CA
:10047800A3F58E730B608A4B03EBCB0318F0200FA8
:100488005B78CAF8203018BFCAF820200023854AB4
:1004980040F2DC5122F813100133082BF7D113A8CE
:1004A80000211C2214F0BBFDBBF10E0F03D00BF092
:1004B800EF03082B02D101238DF85C30022007F0EE
:1004C8009DFD18B14088003018BF0120C8F34003D3
:1004D8008DF85230C8F380138DF85430C8F3403388
:1004E8008DF84C30C8F3C03300F001008DF84F3060
:1004F80018F400638DF8510007D099F8863103F19C
:10050800FF3EDEF1000343EB0E038DF85030C8F3D5
:1005180000438DF855303B6AB9F84801ADF86000E2
:10052800003318BF01238DF85630C8F300538DF8F7
:100538005730B9F84A31ADF85A3018F4805FB9F835
:10054800563118BF5848ADF85830C8F380438DF875
:100558005330B9F854311CBFB0F85001ADF8600001
:10056800B3F5FA7FADF85E3084BF0023ADF8603094
:100578004E4899F8D63187F82430002387F825307B
:1005880043709DF85C3008F00101002BC8F3C002ED
:100598008DF84D108DF84E200CBF0023022301B9B1
:1005A80002B1013306EB83064FF0000AB3699A1EC5
:1005B800143303920593039A32F8023F03924FF6DD
:1005C800FF72934200F094819DF851004FEA132C7A
:1005D800DAB25FFA8CF378B12B4E354806EB021687
:1005E8007168814208D13089B0F5806F00F07B8155
:1005F800B0F5006F00F077819DF8550090B11001BB
:10060800DFF884E00EEB00065EF800E02948864536
:1006180000F069817068B0F1904F03D1B07B062873
:1006280000F061819DF8520050B1174E224806EB48
:1006380002167168814203D13089012800F0538184
:100648009DF84F0050B1104E1B4806EB021671681A
:10065800814203D13089042800F045819DF850007B
:1006680050B1094E144806EB02167168814203D155
:100678003089022800F03781BCF1020F22D19DF8A1
:100688004C1024E08413002090930108A422002039
:10069800842600201112002084090020A0140020C4
:1006A800C89801088011002094240020AD01002082
:1006B8000004004800440140000800488801002068
:1006C800A8220020BCF1010F04D19DF84D1000298B
:1006D80000F009819DF85610BB4E4FEA021859B137
:1006E8009DF85C1041B9511F032905D856F8081028
:1006F800B1F1804F08BF04239DF85710464431B12B
:100708009DF85C1019B9043A032A40F2D380012BF2
:100718004AD1AD4ADFF8BC92079202EB0801FF23E9
:1007280091F80DE089F86C3089F86D304868C9F89F
:100738007C6001F108030989ADF868104FF0000BDF
:1007480002218DF86B1089F870B01AA98DF86AE04B
:10075800069389F828B0C9F82CB0C9F830B0C9F8A0
:1007680034B0C9F868B089F86EB089F86FB004F091
:1007780091F9069B079A997852F808005A4603F0AF
:10078800DDFF304610F0A0F9904BC9F88030904B4F
:10079800C9F88430C9F888B0304609F1800109F1F8
:1007A80084020FF02DF99EE0022B49D15FFA8AF2FC
:1007B8001C2101FB02FC874ACDF81CC002EB0C0986
:1007C800814A89F871A0012189F8701002EB0801AB
:1007D8004FF0000B91F80DE0486889F872B001F10C
:1007E80008020989ADF8681089F87AB01AA9C9F819
:1007F8007C608DF86AE006928DF86B3004F04AF957
:10080800714B069A53F8080091785A4603F096FF00
:10081800304610F059F96F4BDDF81CC06E4AC9F824
:10082800802003EB0C016D4AC9F884208031C9F897
:1008380088B030460A1D0FF0E3F80AF1010A52E0C9
:10084800032B35D19DF85330DFF88881DFF8C0914C
:100858003BB198F826B0304608214FF6FF720023C6
:100868001AE0BDF85E2098F826B0BDF86030B2F501
:10087800FA7F0BD95A49B1FBF2F23046082192B2FD
:1008880004F031F9574B49F82B000AE05649B1FBFF
:10089800F2F23046012192B204F025F9534B49F89F
:1008A8002B00C36098F82630013388F826301AE008
:1008B800042B18D1DFF81C81BDF8582098F8259032
:1008C800494B93FBF2F23046BDF85A30012192B2FF
:1008D80004F009F998F8253008EB89090133C9F8BB
:1008E800500188F82530039B059A93427FF463AE44
:1008F80097F8252087F870213D4A3E4B92F800E092
:10090800AEF117020026022A1E709C461AD8FB690F
:100918003344D3ED007AF5EE407AF1EE10FA02D1C5
:100928003B6A63BB26E0344A06EB02080FCB88E833
:100938000F009CF8003010360133C02E8CF80030C0
:10094800E5D1EDE72D4B13F83E908CF8009003EBC2
:10095800CE03D3F804A0BAF1000FE1D04E45DFDA98
:10096800254A330103EB020853440FCB013688E8CC
:100978000F00F3E7224E3368D8044DD41DE0214B15
:10098800214A13F83E00107003EBCE035E68002E78
:10099800F0D000238342EDDAC3EBC3017218DFF80D
:1009A8007480D2F8009041F8089001EB080791880C
:1009B800B9809279BA710133ECE70EF0EF03082B96
:1009C800124B49D14BE000BF90930108D94400086D
:1009D800B94500088801002041480008B1440008D2
:1009E80000127A00D945000840420F00C9450008A6
:1009F8008409002080130020C0080020C89801083E
:100A080034240020C88001082C140020541200202F
:100A1800501300202D1400209CF80020012ACCD966
:100A2800174B03EB0212103210339342C5D053ED2B
:100A3800047AB6EE007A67EE877A43ED047A53EDCE
:100A4800057A67EE877A43ED057A53ED037A67EE08
:100A5800877A43ED037AE7E7BEF10E0F09D11A78DA
:100A680042F010021A70BEF1180F0BD106F02EFAE0
:100A780008E01A7822F010021A70BEF1190FF4E794
:100A8800C808002006F006FA3368BC4E59035EBF5A
:100A9800BB4B01221A70049B049A1B7843F0040391
:100AA800137062694FF400534FF002094FF0010BC5
:100AB80042F48022ADF86830304629468DF86AB095
:100AC8008DF86B90626103F0E5FFAE4AAE491160A4
:100AD800002005F0C3FFA26942F48052A261E268D7
:100AE80042F48052E260626942F480226261326AB2
:100AF80022F470423262326A42F4A0423262326AAE
:100B080022F470223262326A42F4A0223262326ADD
:100B180022F470023262326A42F4A0020027326282
:100B28004FF0030A3822304629461A928DF86C9005
:100B38008DF86DA08DF86E708DF86F700BF094FACB
:100B4800E268924E42F48052E260E26822F48052F7
:100B5800E2608F4A918821F480510904090C918040
:100B6800918889B241F480519180118801F44151F2
:100B780041F4457141EA0A011180918821F47061BC
:100B88000904090C41F4E0619180918B21F4006122
:100B980009040723090C91831382118889B241F053
:100BA800400111807B4A1660626942F4003262613A
:100BB800E26942F48002E261226B22F020022263A1
:100BC800226B42F080524FF0904842F0200222639C
:100BD800D8F8242022F0F002C8F82420D8F82420DD
:100BE80042F04002C8F82420D8F8242022F4706289
:100BF800C8F82420D8F8242042F48062C8F82420B9
:100C080040464FF4007229461A928DF86E708DF89E
:100C18006F708DF86C908DF86DA00BF025FA4FF47D
:100C28008062404629461A920BF01EFA3268DFF8B5
:100C3800848122F0010232603168574A0A403260EA
:100C4800564A3261326842EA0B023260B760F76096
:100C5800B760B26842F40042B260326832607268CB
:100C680022F0784222F400427260326842EA0B02B3
:100C78003260D8F800504A4E05F4004303933046DA
:100C880005F4006339461022049314F0C8F915EAF4
:100C980009058DF83D908DF83E708DF83F708DF800
:100CA8003CA00DD03F48CDF838B00EA90BF0DCF9C8
:100CB8000622072332707770F37086F802B05D461B
:100CC800039B73B1042337480E930EA90BF0CCF99C
:100CD800082333710723F371012375711D44B37120
:100CE800EDB2049B6BB102232E480E930EA90BF0B4
:100CF800BBF907233373F373012375731D44B3736F
:100D0800EDB20EA9082327480E930BF0ADF909237D
:100D1800337207237572F3720123B3721D44E36AB9
:100D2800214823F4F873E362E36A43F4D873E36277
:100D3800636943F0805343F0010363610AF05BFF8A
:100D48001AA80AF02DFF194B1A93EDB2184B1B93F2
:100D5800012D4FF000030CBF1A4680221F924FF45A
:100D68008072114C20924FF48062219220222046FA
:100D780022921AA94FF400521EE000BF0004004856
:100D8800F00D0020382F002015680008005800409A
:100D9800003001404C110020FFE0CF007A25E00030
:100DA80004190020000800480800024040000050D4
:100DB80014190020342400201C931E93239224939A
:100DC800ADF874500AF0F9FE236843F0010323607C
:100DD8004FF0A0440A20A36823F04053A360A368FF
:100DE80043F08053A36005F020FEA36823F08043FE
:100DF800A360A368A360A36843F00043A3604FF017
:100E0800A0418B68002BFADB8B688F4A23F0405394
:100E18008B608B6843F000538B6090688B4B03406A
:100E280043F468339360CA68894B134043F4005312
:100E3800CB600A6B013D22F00F0215430D630024BD
:100E480001233219917800296CD05D1C042B375D81
:100E5800D078EDB24FF0A04E0ED803EB43035A0002
:100E6800DEF830101F23934021EA030107FA02F34A
:100E78000B43CEF8303031E0092B0ED8053B062263
:100E88005A43DEF834101F23934021EA030107FA7E
:100E980002F30B43CEF8343020E00E2B4FF006015E
:100EA8000ED8A3F10A024A43DEF838C01F23934044
:100EB8002CEA030107FA02F30B43CEF838300DE0B1
:100EC8000F3B01FB03F2DEF83CC01F2393402CEAE2
:100ED800030107FA02F30B43CEF83C30092F4FF019
:100EE800A0420FD99369A7F10A0303EB430397695B
:100EF8000721994027EA01019161916998400843C7
:100F080090610EE053697B1E03EB43035769382158
:100F1800994027EA01015161516903339840084318
:100F280050612B460434102C8BD14FF0A0429368AB
:100F380043F0010393604FF0A0431A68D207FAD533
:100F4800DA68444C22F00202DA60DA6842F00202FF
:100F5800DA60DA6842F00102DA609A6842F0040264
:100F68009A60B4F85C31002B40F0D086B4F95E2169
:100F7800002A40F0CB86B4F96021002A40F0C686EA
:100F8800354A94F86B3112680493B2F85630B4F8C5
:100F9800646194F8635194F86CB10593B4F80CA0AB
:100FA800E37B2E4C2E48039300210C2214F037F8D3
:100FB80000211422204614F032F82A4A0021117028
:100FC8000EF049FC074650B3274A2260274A626060
:100FD800274AE260BB2E274A2261274A01D901210C
:100FE8000EE0612E01D902210AE0292E01D9032140
:100FF80006E0132E01D9042102E0092E0DD905219E
:101008001170184A042111701C4A072111701C49DB
:101018000A6842F001020A600EE00621F0E70320A8
:1010280005F070FD9AE10122AA4040F20221114028
:1010380051B3012D41D90025DFF848900022092D30
:1010480089F80020F7D8EEE700030050E010FCFF15
:1010580007C0FFFD9424002090110020A414002054
:1010680000240020B81400208FF70008FDF60008BF
:10107800D9F6000890C1793D000000201001002039
:1010880050120020572F002040F2FD111140002976
:10109800CFD00EF0E0FB0028CBD0874A87491160FB
:1010A80087495160042289F80020864A0821517036
:1010B80085490A6842F002020A60BBF1040F73D83E
:1010C800012505FA0BF212F0160975D112F0090F75
:1010D80067D00A2005F0A9FC7720A0212A460EAB8C
:1010E80003F0EEFD002867D077201E212A4603F082
:1010F80063FE4FF42F6005F08DFCA9F16001002517
:10110800C9B202221AAB77208DF868508DF8695061
:1011180003F0D6FD9DF869309DF8682043EA022265
:101128006A4B03F5B97129F8012009F10209B9F1EF
:10113800100FE2D1B3F8802102F00F0E02F47F42C3
:10114800A3F8802101202B462946DFF880C121F031
:1011580001056544B5F87251002D18BF002011F043
:10116800010F03D0EDB26B40082502E083EA152396
:10117800FAE713F4004F18BF83F4C053013D4FEA58
:101188004303F6D101311029DFD1504942EA0E025A
:10119800A1F8802180B9C3F303339E4500F09685FA
:1011A8000AE0BBF1010F07D05B46464A9370464AF6
:1011B800136843F004031360434D2B689A0702D564
:1011C8003D4B1B689847039BDFF8009140492BB3C0
:1011D80016F0FF0F0AD12B6813F0020F4FF07D02B3
:1011E80040F2712308BF4FF4FA7302E04FF47A73A8
:1011F8001A469A4505DBBAF57A6FA8BF4FF47A6AA2
:1012080000E09A46531E5344B3FBF2F3013BDBB2B2
:1012180003FB022289F882310A6005E09DF80C3050
:1012280089F88231C1F800A02A4B1B689847DDF87D
:1012380010A0294E0023BAF1020F337006D0BAF17C
:10124800030F1AD0BAF1000F40F055852EAB0022DB
:1012580003F8502DC9F884211E200A21012203F029
:101268002FFD50B19DF86830482B06D11B4B1C4A06
:101278001A601C4A5A60002F3AD12EAB4FF0000B6F
:1012880003F850BD0C205946012203F019FD00282F
:1012980000F064859DF86830482B0AD10F4B124A3C
:1012A8001A60124A5A603846002F00F05785032307
:1012B8001FE0584600F052BD00240020F1F5000858
:1012C80039F7000810010020501200208801002082
:1012D800742C0020A4140020542F00209C06002009
:1012E80071900008E18E000801900008758F0008D1
:1012F8000223BB4AD3702B6843F008032B60B94B19
:1013080093F858210AB1B8490A7093F859210AB1DB
:10131800B6490A7093F85A3103B133702B68B4494F
:1013280013F0080F00F0EE84BDF91400DFEDB16A88
:10133800642290FBF2F302FB130212B207EE902A2A
:10134800B8EEE77A07EE903AF8EEE77AE7EE267A13
:10135800B2EE047A67EE877AC1ED007AA64F3B7841
:1013680043F002033B70A54B4FF480421A854FF4BB
:1013780000429A610A25A14EB38A9BB283F4804346
:10138800B382B38A9BB283F40043B382192005F079
:101398004CFB012005F062FB192005F046FB013DDE
:1013A800002005F05BFB15F0FF05E4D14FF4004386
:1013B8004FF48049924DB361C6F818902B681B070B
:1013C80009D5904BA6F828901B6898478E4BC6F80D
:1013D800189001221A708D4B9FED8D8A1B688D4ED7
:1013E8001B7B00EE103AB8EEC00A20EE080A08F09F
:1013F800C7FE338807EE903AF8EEE77A27EE800AC0
:1014080014F01CF8844B9FED857A1880338807EE1A
:10141800903AF8EEE77A824BC7EE277AFF211A2234
:101428009FED807AC7EE877A9FED7F7AC3ED007AC9
:10143800D4ED047A7D4C7E4B67EE887A204667EEC1
:10144800877AC3ED007A13F0EAFD002323702B6836
:10145800784A012113F0020F18BF617011701FBF85
:10146800032111700221A1705D0748BF1178204641
:1014780041BF4C1C14700324445413F00A0F0CD0C1
:1014880013780421C154591CC9B205244454D91CE9
:101498000233DBB211700621C154D8F800108C0653
:1014A80041BF13785C1C1470072448BFC4540B0652
:1014B80008D513780924C4549C1C0133DBB214707A
:1014C8000A24C454474E7479082C01D00E2C04D138
:1014D80013785D1C15700B25C554137811F4803FE3
:1014E8004FF00C0E00F803E003F101051CBFDFF814
:1014F80044E10233EDB215701FBF8EF800304B4B3C
:101508004FF00E0E03F805E04B0741BF13785D1C42
:101518001570102548BFC55413785D1CEDB24FF007
:10152800120E11F4806F157000F803E00ED096F8D3
:1015380014E2BEF1000F09D0DFF8F8E002338EF8AC
:1015480000303A4B4FF0130E03F805E0137811F40E
:10155800007F4FF0140E00F803E003F101051CBFF3
:10156800DFF8D0E00233EDB215701FBF8EF80030FF
:101578002E4B4FF0150E03F805E0182C0DD11378FB
:101588001625C5545D1CEDB24FF0170E00F805E0A6
:10159800DD1C0233DBB21570C4540C0341BF137851
:1015A800591C1170192248BFC254002198222248A0
:1015B80013F035FD0DF0F1FD204B214A21491A6049
:1015C80000234B800B7120490A60B6F8982190B22D
:1015D8001E4921F813000133122BF9D138E000BF5E
:1015E8001001002094240020B8140020572F002058
:1015F800241300208988883C282F002000080048F0
:10160800501200209C060020B40600204C15002033
:1016180035FA8E3C04000020681500200AE81C41B9
:10162800D407002000401C46BD37863559110020DC
:101638004815002058110020002200202C0F0020FF
:101648001E2600207C0E00201C2F00207024002065
:10165800D8F80030D8045CBFB6F89E0108801B0794
:1016680040F1C88096F89231062B00F2BD80DFE881
:1016780003F004070E3D5878780045F2F05201E077
:1016880042F6F822854B1A800DF035FEABE007EEE6
:10169800902ADFED836A814BB8EEE77ADFED817A35
:1016A800E7EE267A42F6F82119800023FCEEE77A65
:1016B8007D4A17EE901A42F823100133122BF7D106
:1016C8007A4A7B4911607B4A4020137006F072FD0C
:1016D800002800F0898001234FF0070890F90000E6
:1016E800754A8DE808014021744B77E06B4B42F650
:1016F800F8221A806D4B724A1A606E4B10224020F5
:101708001A7006F057FD00286ED001234FF0000C28
:1017180090F900006B4A8DE8081040214FF4E1333E
:101728005CE05E4B42F6F8221A80604B664A1A600B
:10173800604B082240201A7006F03CFD002853D068
:1017480001234FF0000E90F90000604A8DE8084030
:1017580040214FF4E13306F017FB5D4BC3F88801D5
:101768003EE04E4ADFF8A081DFF8A0C1DFF8A0E133
:10177800584D594C594842F6F82111804D490C22D0
:10178800062B0A700ED0002388F800308CF8003041
:101798008EF800301B232B700523227003704FF442
:1017A800E1340BE0002188F800108CF800108EF866
:1017B8000010227021214A4C297003703B4B494A82
:1017C8001A60402006F0F6FC70B101230025464A55
:1017D80090F9000040218DE82800234606F0D4FA4D
:1017E800003018BF012028B9082008F08DFD2F4BC4
:1017F8003E4A1A603E4A1368904613F4804F2D4AB9
:101808001FBF3C4808211170284918BF086042F2E0
:101818000101194003F0010003F4005479B11F4994
:1018280044F620650D8024B1082111701F49324CFF
:101838000C6020B10C2111701C49304808601178E7
:1018480004395170190640F19F802148DFF8C4908F
:101858002B4DC0F88C5100242146152200F5C87084
:10186800DFF8B4A089F80140C9F80440C9F8084075
:10187800053D13F0D4FB2046CAF8005007F0BEFF20
:10188800204B02201B68C9F80C3006F093FC002896
:1018980044D1802008F038FD6EE000BF2C080020FD
:1018A800CDCCCC3F0000B0C46C2E0020000100203D
:1018B800A11D01089C220020AD1E0108A086010080
:1018C800D9B70008051E0108C1B700080DB90008FE
:1018D800880100209A1800201B1800209B1800205F
:1018E80090D00300DDB60008EDB70008011E01081E
:1018F80034240020D51D0108F11D0108E11D01084F
:1019080084260020582400201C1800209918002044
:1019180098180020E807002008080020447999F862
:101928000130C8490C2202FB03125278A24204D0AB
:101938000133DBB2042BF4D9002389F80130DAF83B
:10194800003099F801201B7890F90000002B4FF027
:101958000C0303FB021314BF0324012400225B7849
:1019680000940192022106F00FFAB74B1860002884
:101978008FD0012007F042FFB44B1868B44B00F534
:10198800C5721A6007F0E8FFB24AB34B1360B34A56
:10199800B34D80331360D8F800300024DA032C707C
:1019A80040F1AD800CF00CFEDFF818C3DFF818A387
:1019B800CDF810C040F22A3B4FF00109604621469D
:1019C8005A4685F8009013F02AFBDAF81430A54D32
:1019D8004FF0904043F40033CAF81430036A23F000
:1019E80070630362036A43F0807303624023022238
:1019F8000C930CA903238DF8342003928DF835300D
:101A08008DF836408DF837900AF02EFBDAF818304A
:101A1800039A43F40033CAF818302B8823F4407330
:101A28001B041B0C2B801D23EB620EA92A85602347
:101A38002C862846C5F814900E93ADF83E401094B5
:101A4800ADF84440ADF84640ADF84840ADF84A40DE
:101A5800ADF83C900AF05CF9AB6943F00803AB6160
:101A68006B6C43F400436B64DAF8143043EA0903FF
:101A7800CAF81430AAF57D6A50460AF0BCF81AA8CC
:101A88000AF08EF8784B1A9310231C9380231F9327
:101A98004FF48073DDF810C020931AA94FF4005357
:101AA8005046CDF86CC02393ADF874B01E942194C1
:101AB800229424940AF081F8EB6843F40073EB60F5
:101AC800DAF8003043F00203CAF800300BA80D23FF
:101AD8008DF82C308DF82D908DF82E408DF82F90A4
:101AE8000EF0D4FF2146614B1A68614B43F8212060
:101AF80001312029F7D102F0EFFE02F0EDFED8F80F
:101B080000305B0556D55B4D5B4BD5F8D094C3F8D8
:101B18000090042006F04EFB0421C5F8D40406F01A
:101B280023FB564B85F8D8040820C3F8009006F02C
:101B380041FB534B534C1860082106F015FB00215C
:101B480085F8D9042C22204613F069FA8E23637095
:101B58004FF07C0BE0234FF07D0AE37084F800B06F
:101B680084F82BA0484C2C220021204613F057FA69
:101B78008A2363701020A023E37084F800B084F8EF
:101B88002BA0C5F8DC9406F015FB1021C5F8E0047D
:101B980006F0EAFA85F8E4042020C5F8E89406F08F
:101BA80009FB2021C5F8EC0406F0DEFA85F8F004FC
:101BB8000FF0F2FFD8F80030344A13F4002318BFAE
:101BC8000123137004F00AFF314B18607379052B59
:101BD80002BF304B4FF4C8721A802F4B4FF47A7201
:101BE8001A802E4BC8221A802D4A137843F0080316
:101BF80013702C4A137823F002031370D8F80020CE
:101C080040F6020313406BB1274B284A1A60284B51
:101C180003221A70274B01221A70274A00231380C7
:101C2800264A1380B368C8F80030254B01221A7081
:101C38003B7863F07F033B702FB0BDEC028BBDE8AF
:101C4800F08F00BF107401089C170020901100202D
:101C5800800F0020D8170020B8260020D4170020B5
:101C6800F10D00200044014034440140D8730108BC
:101C7800F20D002088010020441200209C12002050
:101C8800E81200206C120020A1120020702C002005
:101C9800740E0020141500204E2F00204C2F002019
:101CA80054120020562F00203C120020102600203D
:101CB800A01200200801002020100020221000207F
:101CC800F00D00202D03002000100240284B42F2A6
:101CD80010721A805A80274A5A60274A9A60274AFF
:101CE800DA60274A1A61274A5A61002F3FF464AA2A
:101CF8000323FFF75ABABAF1010F7FF600AB9A46F1
:101D0800FFF797BA00230B60FFF728BB1BB207EE5B
:101D1800903ADFED1D6AB4F95E311C4AF8EEE77AB5
:101D280007EE103A67EEA67AB4F96031CDED1A7A6B
:101D380007EE903AB8EEC77AF8EEE77A002127EE78
:101D4800267A67EEA67A11701AA811498DED1B7ACA
:101D5800CDED1C7A08F01CFAFFF712B9BAF1010FA1
:101D68007FF6CDAA4FF0000A3070FFF76FBA00BFB8
:101D7800C00600200BF600084DF6000801F6000822
:101D88003DF6000831F4000835FA8E3C7400002056
:101D9800E0180020864A2DE9F04F1368854C03F5BA
:101DA8009C4320332DED028B2360A3880133A3804D
:101DB800814B196889B011F4804F0592019305D1C0
:101DC80010F0C2F810B9237B0133237300277B4B33
:101DD800DFF800821E78FDB2AE4230D9D8F8003064
:101DE8007648072D98BF595D754B88BF29461B68F3
:101DF8009847032D1ED8D8F8002005F10E0302EBF2
:101E080083039988DA88A8B14FF47A73401A584343
:101E1800531A90FBF3F040F6C90300F57A70984224
:101E280005DC40F2EE239842B8BF184601E040F6C0
:101E3800CA0080B204EB45050137E881C7E70F23E4
:101E4800277B84F83230032594F83330B7FBF5F557
:101E580005EB45057D1B029394F834300393D8F8BD
:101E680000A0DFF878B1EBB204930025B54255DA4B
:101E78005449029B31F815904FEA450853B910F0C0
:101E880063F828B1039B002B08BF4FF0000901E05D
:101E9800DDF80890BAF81400484503D8BAF81600D7
:101EA80048450ED2E8B210F025F8032D8146DFBF71
:101EB80094F832E00120A8402EEA0000D8BF84F848
:101EC800320010F041F818B13F4828F8009021E09E
:101ED800049B94F87E002BF8139028B9022F15D98B
:101EE8003449012081F87E00BBF80210BBF80000DD
:101EF8000844BBF804100844344980B228F80100AB
:101F080000B2032190FBF1F080B200E048462E4970
:101F180028F8010001350BF1060BA7E794F83250B9
:101F2800244BA5F10F077D427D4184F898503DB1BF
:101F38009A8811B21429CCBF143A00229A800BE077
:101F480083F83350B54207DAE8B20FF0D3FF1E4BDF
:101F580023F815000135F5E7019B1B68D80405D562
:101F68001B4B1B68D90701D40FF0AAF9059B196808
:101F7800184B1868837A9BB3013B134D027B35F8E5
:101F880013301AB1C3F53B6308339BB21BB2A3F5F8
:101F98007A73B3F57A7FA8BF4FF47A7323EAE373B1
:101FA80007EE903A9FED0C7AF8EEE77A51E000BF21
:101FB800302F0020780E0020342400209C2200209E
:101FC80000010020860E002070240020F80E00205A
:101FD800541100201C2F002000007A44AE0E00206F
:101FE800019A1268120440D5D4F89C20AD4E8A1A82
:101FF800002A3ADB01F59C422032C6F89C20AA4A06
:10200800C07A5579A94A32F8152096F8A0500135BA
:1020180092B292FBF0F205F00F0086F8A00030446F
:1020280080F8A1201A46A248185C01330244102BFC
:1020380092B2F8D112B292FBF3F31BB2642BA8BF91
:10204800642323EAE37307EE903A9FED9A7AF8EE59
:10205800E77AC7EE877A984A9FED987A67EE877A8B
:10206800FCEEE77A17EE903A1380019B944D1B68BB
:10207800DFF8708213F4807F7AD0924B994204D9AA
:10208800237A13B9874B01221A72B4F904E098F83D
:102098000060844BBEF1140FCCBF4FF0000E4FF020
:1020A800010EC6F38006BEF1000F03D000279F7211
:1020B8005F7200E00327A07AD4F8B4B0D4F8B8C0AF
:1020C800B4F90490617AE3882A88032848D8DFE8BD
:1020D80000F0020E1B35BEF1000F02D02A8000224C
:1020E8002AE0002E40F05D862A80A6723AE09CF82D
:1020F800000000EB8000814502DC2A8001221BE001
:1021080001206EB300F0CCBE3EB1BBF80E206A8051
:10211800AA80BCF80200E88002279CF800A09CF87E
:102128000100504400EB8000814500F33D86002EFD
:1021380000F03A862A800222A27213E02A80032243
:10214800A2726172E3807EB198F8003043F0020316
:1021580088F80030534B00225A720FF0B1F803E0B0
:102168002A80A0726172E38017B1384604F090FCAF
:10217800554EB6F852010EF0FDFE834668B90FF0D1
:102188007FFC524BC3F800B0C3F804B0C3F808B0E2
:102198004F4B00221A605A609A6098F800305F0727
:1021A80036D5019B1B68D80632D54A4B1B78D90611
:1021B8002ED4494B1B7893B196F8DE31BBF1000F52
:1021C80015D17BB1454B1A68D4F8BC309B1A002B4B
:1021D80008DA0FF075F8334B83F8C0B018E0BBF19C
:1021E800000F0DD1102004F053FC01230EE03BB189
:1021F8003A4A12684FF47A7101FB0323C4F8BC30E1
:1022080094F8C03023B104F02FFC002384F8C030C8
:10221800002396F8DCA196F8DD11B6F89A71B6F8A5
:102228009CE1184635F913208008BA42C4BF60F013
:102238007F00C0B201337245B8BF40F04000042BA4
:10224800F0D194F8C130174A834205D192F8C230D0
:10225800F92B04D8013300E0002382F8C2301E4A6B
:1022680084F8C10010780F4B1D4F914600283ED1CD
:102278003A68D20709D5BBF1000F38D198F8003079
:10228800DB0734D50EF090FE31E098F800205007B7
:102298002DD593F8332052B35B7A43BB21B30FF0AB
:1022A8000FF824E0780E00200419002014190020EB
:1022B800190F00200000C842B011002000C07F4460
:1022C80070240020404B4C0094240020C8190020A2
:1022D800841A0020541200200300002058240020F3
:1022E80054110020562F0020BBF1000FD7D094F8CE
:1022F800C2307C4ADFF81CB2142B40F0928099F867
:1023080000301AF1000A18BF4FF0010A7BB392F8A7
:10231800C1305F2B12D198F8003003F0040303F0AA
:10232800FF0113B10EF0CCFF08E00B2003910292DD
:1023380004F0AEFB029A039982F8C210BAF1000FBA
:1023480015D094F8C1307D2B11D198F8003003F0E6
:10235800040303F0FF0213B10EF0B2FF07E00B20F5
:10236800029204F095FB5F4B029A83F8C22098F81A
:10237800003003F0040303F0FF01002B51D194F85F
:10238800C130584A572B16D1574B4FF47A721A80DE
:10239800019B1B68190601D507F040FB534B1B68CE
:1023A8005A0742BF524A0A21118013F0080338D154
:1023B800504A138035E001980068400716D55A2B1B
:1023C80014D14D4B187820B119704C4B01221A705A
:1023D80027E092F8C33083F0010382F8C3300BB1D1
:1023E8000C2000E00D2004F053FB1AE05D2B00F0F8
:1023F800DE845B2B00F0FC845E2B02D1032000F00E
:10240800F8BC562B01D108F007FA99F80030002BD8
:1024180000F0048594F8C1306F2B40F0F9840EF079
:10242800C3FD019B1B68580733D594F8C330A3B18B
:1024380098F80030590710D5B5F90620B6F89A3142
:102448009A420ADD3B6813F0010301BF2C4A32218E
:102458001180244A08BF82F8C3303B68DA030AD5E2
:10246800284B1A782AB9244A127812B9244A3221F8
:10247800118001220CE0204A137853B198F80030FB
:1024880003F0040303F0FF011BB91C4B1170012278
:102498001A70DBF8009000233B6009F17B0609F114
:1024A800CB0A3278737816F8010C9A420BD231466F
:1024B80004F034FA38B116F8022C012303FA02F2B8
:1024C8003B6813433B6004365645EAD10E4B1B78F4
:1024D80013B30E4D054F2B680D4E13F0020F40F04D
:1024E80042833AE3780E00204E2F0020501200203D
:1024F8004C2F00202C1200204115002042150020EE
:102508002815002040150020582F002054110020C5
:10251800181300209011002009F1CA0609F58977DF
:102528003278737816F8010C9A4225D2314604F0B5
:10253800F5F908B3B37896F804E0C04A96F8039022
:10254800BF480C21013B01FB0E4103EB430313443D
:10255800D1F8C8209A420FD0C1F8C830002390F8AB
:10256800F420C1F8CC30012303FA0EF322EA030366
:1025780081F8C49080F8F4300636BE42D0D1B14B11
:10258800DFF8CCB21E68B04B1B68039394F8333065
:10259800049300230293DBF80030002B00F0D48270
:1025A80093F80090B9F1000F00F0CE82DBF8042018
:1025B80003998A1A002A0CDB01F5FA720299CBF802
:1025C800042001228A4094F8F41021EA020284F8D7
:1025D800F420049A002A00F0B7821BF8042C5978DA
:1025E8000432D2B2002940F0718235F91210974AAC
:1025F800934FB2F8982102F1C800814202DD93F8A6
:1026080002A015E0C83A914203DA9978C1F1000AAC
:102618000EE0029A0123934097F8F42022EA03037C
:1026280087F8F430039B03F5FA73CBF804308BE298
:1026380097F8F430029A1341DB0700F18582BAF16A
:10264800000FCCBF0220012004F044FA09F1FF3347
:10265800132B00F27082DFE813F0140021002F0022
:1026680043005C006300CA004001A701D7010702CC
:102678006E02430052006300CA0040019A00120132
:10268800770137785744FA2FA8BFFA2727EAE77760
:102698003046377004F028F901200BE0777857446A
:1026A800642FA8BF642727EAE7773046777004F0DD
:1026B8001BF902203946D4E196F80390D144B9F1C8
:1026C800640FA8BF4FF0640929EAE97986F80390F6
:1026D8003046D7F8F81005F075FD03204946C0E1EB
:1026E800717951446429A8BF642121EAE1717171AB
:1026F8000D2004F05FF9B9F10D0F00F01C8231795B
:1027080051446429A8BF642121EAE17131710E2086
:10271800A7E1B179514481F30801B1710520A0E125
:10272800D7F8FC301A78022A22D107EE90AAF8EEE0
:10273800E77AB2EE040A87EE800AD3ED097A30EE22
:10274800270AB5EEC00AF1EE10FA09D4DFED427A95
:10275800B4EE670AF1EE10FAC8BFB0EE670A01E0FE
:102768009FED3E0A83ED090A0F2004F00EF90AE0F6
:1027780099785144C829A8BFC82121EAE171997004
:102788000F2004F017F9B9F10F0F00F0D481D7F832
:10279800FC301A78022A20D107EE90AAB8EEE78A10
:1027A800B2EE040A88EE008A93ED080A38EE000AB1
:1027B800B5EEC00AF1EE10FA09D4DFED277AB4EECF
:1027C800670AF1EE10FAC8BFB0EE670A01E09FEDA4
:1027D800230A83ED080A12206BE159785144C8296D
:1027E800A8BFC82121EAE1715970122039E1D7F850
:1027F800FC301A78022A33D107EE90AAB8EEE70A1D
:10280800DFED157A93ED0C7A80EE270A30EE070A91
:10281800B5EEC00AF1EE10FA07D4B4EE670AF1EE8D
:1028280010FAC8BFB0EE670A01E09FED0C0A83ED0D
:102838000C0A102004F0A9F81DE000BFFC7701087D
:10284800780E0020B4110020582400209424002081
:10285800400F002000007A440000C8420000000039
:10286800197B5144C829A8BFC82121EAE17119730D
:10287800102004F09FF8B9F1100F00F05C81D7F830
:10288800FC301A78022A1ED107EE90AAB8EEE78A21
:102898005FED0F7A93ED0B0A88EE278A38EE000A6F
:1028A800B5EEC00AF1EE10FA07D4B4EE670AF1EEFD
:1028B80010FAC8BFB0EE670A01E01FED180A83EDF1
:1028C8000B0A1320F5E0D97A5144C829A8BFC821BA
:1028D80021EAE171D9721320C3E0D7F8FC301A78E5
:1028E800022A22D107EE90AA1FED260AF8EEE77A0F
:1028F80087EE800AD3ED0F7A30EE270AB5EEC00ACC
:10290800F1EE10FA09D45FED2C7AB4EE670AF1EE15
:1029180010FAC8BFB0EE670A01E01FED300A83ED78
:102928000F0A112004F031F80AE0997D5144C829B2
:10293800A8BFC82121EAE1719975112004F03AF87D
:10294800B9F1110F00F0F780D7F8FC301A78022A95
:1029580020D107EE90AA1FED410AB8EEE78A88EE6B
:10296800008A93ED0E0A38EE000AB5EEC00AF1EEC1
:1029780010FA09D45FED487AB4EE670AF1EE10FA5E
:10298800C8BFB0EE670A01E01FED4C0A83ED0E0ADE
:1029980014208EE0597D5144C829A8BFC82121EAD6
:1029A800E171597514205CE0D7F8FC301A78022AD6
:1029B80020D107EE90AAB8EEE78AB2EE040A88EEB4
:1029C800008A93ED0A0A38EE000AB5EEC00AF1EE65
:1029D80010FA09D45FED607AB4EE670AF1EE10FAE6
:1029E800C8BFB0EE670A01E01FED640A83ED0A0A6A
:1029F80009205EE0D9785144C829A8BFC82121EA36
:102A0800E171D97009202CE0D7F8FC301A78022A35
:102A18001ED107EE90AAB8EEE78A5FED717A93EDC2
:102A28000D0A88EE278A38EE000AB5EEC00AF1EEE4
:102A380010FA07D4B4EE670AF1EE10FAC8BFB0EE88
:102A4800670A01E01FED7B0A83ED0D0A0A2030E0DA
:102A5800597B5144C829A8BFC82121EAE17159739B
:102A68000A2003F0A7FF66E0D7F8FC301A78022A9C
:102A780022D107EE90AA1FED890AB8EEE78A88EE00
:102A8800008A93ED100A38EE000AB5EEC00AF1EE9E
:102A980010FA09D45FED907AB4EE670AF1EE10FAF5
:102AA800C8BFB0EE670A01E01FED940A83ED100A73
:102AB8000B2003F06AFF3EE0D97D5144C829A8BF26
:102AC800C82121EAE171D9750B20CAE7012932D161
:102AD800987835F91230B3F5617F05DB40F633029B
:102AE8009342A8BF134601E04FF46173B9F10C0F8C
:102AF80021D14FF4966292FBF0F0AE4AA3F56173D0
:102B080093FBF0F3DFB21378BB4214D0042F34BF29
:102B18003B4602231370A84A09FB0323A74A06333E
:102B2800136007F0B9FC4846394603F043FF781CA8
:102B3800C0B203F0CFFFA249029A0123934091F853
:102B4800F420134381F8F430029B0133042B0293E1
:102B58000BF10C0B7FF41FADBBE4019B1B68D80580
:102B68000ED5637A63B13B68990709D5338813F0AA
:102B780001090AD10EF084FF012007F0B5FB04E03B
:102B8800012007F0A0FB012300E000232A68520778
:102B98000CD55BB1012007F096FB3388980708D461
:102BA8000EF06EFF022007F09FFB02E0022007F004
:102BB8008AFB3388834A13F0030F4FF480410CBF1C
:102BC800916111853A6812F00A0F23D02A68D1065C
:102BD80009D55A070AD4042007F086FB7A4B1B88CC
:102BE800A4F8003102E0042007F06DFB2B689B0677
:102BF80006D53388580606D4402007F075FB02E056
:102C0800402007F060FB2B68590642BF6E4B1B88BB
:102C1800A4F802313B689A0608D42B681B0540F1DA
:102C28008C804FF4807007F05FFB8AE0674B1B785D
:102C38009F074FD5664B1B78042B4BD92B68604FE9
:102C480013F400790ED03388DC0637D4102007F04F
:102C58004BFB202007F037FB5E48011D06F032FED3
:102C6800022327E0348804F01004A4B22CB1102009
:102C780007F029FB012487F804912B68580512D521
:102C8800D7F8083154495A89B1F90030002BB8BF38
:102C98005B42934207DAB1F90230002BB8BF5B42BE
:102CA8009342C0F203813388990608D5202007F0A3
:102CB8000AFB002387F80431012400E0002497F878
:102CC8000C31B3B90E2003F0E3FE3D4B012283F82B
:102CD8000C210EE0338803F03003002B9DD0102028
:102CE80007F0F1FA202007F0EEFA002384F8043107
:102CF80001E0002C91D0394B002003F1280603F1A4
:102D08005004374A002122F81010364A596022F838
:102D180010100432716022F8101000221A609A60B4
:102D28003260B26022606160A260143314361434D9
:102D380000287FF472AF0120E3E74FF4807007F0BA
:102D4800C2FA294B5A79082A1C4601D00E2A02D108
:102D5800402007F0B8FA019B1B685A0540F1BB8078
:102D680094F8143223B998F8003013F0040F02E0F5
:102D78002B6813F4002F0BD01C4B00221A703C2038
:102D88000CF002FB002800F0A6800CF0A5FFF6E787
:102D98000EF002FF09B0BDEC028BBDE8F04F0CF05D
:102DA800FCB90120FFF791B90320FFF78EB9012084
:102DB8001FE000BFE02300203C2C0020B4110020BD
:102DC800780E0020000800482C1200205412002021
:102DD8005A120020BC11002034120020880F002055
:102DE800502F00200010002094240020A122002051
:102DF80002205FFA80F909F1FF3386F8AC3707F053
:102E0800B5FA07F06DFB484603F064FEFFF709BB0F
:102E1800BAF1000F02D07E2B3FF401AB94F8C13019
:102E2800972B05D12E4B4FF4C8721A80FFF7F9BAC9
:102E3800A72B06D12B4A137843F004031370FFF72E
:102E4800F0BA0022BB2B079201D1022303E0B72B73
:102E580004D14FF6FE73ADF81E300AE0BE2B01D147
:102E6800022304E0BD2B7FF4DCAA4FF6FE73ADF815
:102E78001C30DBF80030BDF81C10B3F858200A44A9
:102E8800A3F85820BDF81E10B3F85A200A44A3F836
:102E98005A2007F0C1FC002384F8C230FFF7C1BAFA
:102EA800013301469BB20220FFF70FB933889B0616
:102EB8003FF505AF202007F017FA0B480B4B011D13
:102EC8001A685B684360026006F0FCFC084B01244A
:102ED80083F80441F3E609B0BDEC028BBDE8F08F3E
:102EE8001415002054120020C41100205C12002088
:102EF800780E00202DE9F04FC14BB3F90610C14BF5
:102F08002DED028B1F687A8985B0914201930EDB03
:102F1800B1F5FA6FFC79BDBF8B1A6343A2F5FA6469
:102F2800C4F16404BCBF93FBF4F4643400E064248B
:102F3800B54BB64AB3F898B193F962311268029268
:102F48009BB2154603930022AD4B33F912E0CBEB4D
:102F58000E0303F2F31640F2E63086424FEA420CC3
:102F680003D8002BB8BF5B4201E04FF4FA73022A82
:102F78002ED0029E96F811611EB1B342CCBF9B1BA6
:102F88000023A34E6FF0630A642093FBF0F836F831
:102F980018900AFB083A08F1010836F918600FFA88
:102FA80089F8C8EB060606FB0AF696FBF0F6994880
:102FB8004E4420F80C60BE18642036797343964E50
:102FC80093FBF6F364339BB2634393FBF0F02DE07D
:102FD800029890F812611EB1B342CCBF9B1B00232C
:102FE800DFF860926FF06308642093FBF0F008FB51
:102FF800003A39F910600130002B39F91000A0EBC4
:10300800060000FB0AFABDF80C009AFBF8FAC6EBBA
:103018000A0A1AFB00FA7F48A0F804A0B879B8BFDA
:103028005B4243437C4893FBF0F064306B787B4E03
:103038004FF06408434393FBF8F3B354784EEB7AAC
:10304800434393FBF8F3B3546B7D724E5843754B6F
:1030580090FBF8F0022A9854734B0ED1DE4583F8A2
:1030680002800DDB684CB4F89A21914214DBB1F56B
:10307800FA6FA8BF4FF4FA610FE0DE459C5404DAFA
:1030880036F80C305B4226F80C300132032A05F181
:1030980001057FF459AFE5E71146DFF8BCE15D4D66
:1030A800891A4FF47A736FF063075943C2F5FA62CD
:1030B8006423B1FBF2F191FBF3F23EF8120007FB37
:1030C8000211013207B23EF91220D21B514391FB83
:1030D800F3F30344F380554B1B885F0635D5544BF7
:1030E800544A1B881288DFED547A9B1A1BB208EEEB
:1030F800103AB8EEC88A28EE278AB0EE480A07F0D8
:103108003FF8F0EE408AB0EE480A06F0D6FFB5F96F
:10311800023006EE903AB5F90030F8EEE66A07EEAE
:10312800903A20EE667AF8EEE77AA7EEA87A67EE8C
:10313800807ABDEEC77AE6EEA87A17EE103AFDEE71
:10314800E77A2B8017EE903A6B803C4D2B689807F6
:1031580040F1A1803A4B3B4F1A687B6945F2072141
:10316800D31A8B4240F397807A6109F06BF8364B9B
:10317800DFF8E8901A78032A9846B9F8003022D187
:103188000A2B2AD90023282088F8003003F04DFCA8
:1031980009F058F82D4B188809F03EF82C4B1A689E
:1031A800D37890FBF3F0013008282A4BA8BF0820F9
:1031B8001870537980B213FB00F33B83137913FB28
:1031C80000F0788309E00A2B07D80323214A88F8FE
:1031D8000030002313703B837B8398F800301A4A31
:1031E800012B3DD002D3022B4CD054E03A8BB9F8D6
:1031F80000309A424FDD012388F8003040E000BFDC
:1032080070240020B4110020942400209011002084
:1032180028130020341200200CFEFFFF441A00205F
:10322800161000205C1A0020A8190020181300208E
:103238002C1200207A0F002035FA8E3C342400200E
:10324800302F002008100020A01200201C19002098
:103258003C12002008010020D21500204012002056
:10326800B9F800107B8B8B4202DD022313700FE04C
:10327800A24B1B8B0133994202DD002313700AE035
:10328800082006E07B8BB9F8002001339A42B2DCB3
:10329800072003F0FDFB2D68290575D5984B974F3E
:1032A8001A68FB69C3EB020845F2072398456BDDF2
:1032B800B6F90630FA61A3F57A7B924BB4F852015D
:1032C800D3F80090904E99F80A30012B4FF47A7198
:1032D80098FBF1F803D040D3022B1FD03FE08B4B73
:1032E800386A5A7B8A4B33F812204FF0080E92B294
:1032F80090FBFEF3C01A8318BA843B6240F6E4429E
:1033080093FBFEF39BB25343B9F80820C2EB133387
:103318004B43B9F9062093FBF2F31FE07D4BB9F854
:1033280008A01B78C6F800A05A0718D50DF022FE91
:1033380020B915F0100F18BF4FF0000BB9F906208F
:103348000BFB0BF1322391FBF3F35B445A434FF42D
:103358007A7392FBF3F3534400E000233360D7E918
:103368000A0133686C4A03FB08F84FF47A7398FB38
:10337800F3F810EB080041EBE8710023C7E90A01F4
:103388000EF030FE654B1860654E3368DB0427D5B8
:103398002F0622D5634B1B789D071ED5624B1878E4
:1033A80004281AD90022614BD7180521951C4FF023
:1033B8000A0E122AD154E9B287F801E004D0B0EB22
:1033C800510F2A46EFD800E014215A18322002F88B
:1033D800010CFF225A540F2000E00A2003F058FB8A
:1033E800534D2A68002A50D0524B534F18683968F9
:1033F8008142984649D8514BDFF84C911978526868
:10340800E1B94FF0010A83F800A0B9F80030D35CA5
:1034180023B3504603F022FB494B83F800A00EF07B
:103428009FFDB9F80030CBB92B681B78053B534595
:1034380014D803F0D3FA434B18600FE04FF0000A9A
:1034480083F800A0B9F80030D35C3BB1504603F0D4
:1034580005FB3B4B83F800A00EF082FD2A68B9F803
:10346800003052683848D25CFE2A01D100230BE0B4
:10347800FF2A02D103F0F8FA07E0D8F800500A2131
:1034880011FB02523A6001330380224D2B78580712
:1034980004D52E4B4FF400421A856FE03268D107ED
:1034A8005CBF43F001032B701E4B1B781F075EBFE8
:1034B8002B7823F001032B70D60248BF2B78204AC3
:1034C80044BF23F001032B70214B1B6813F0040F3A
:1034D80002D02049098851B91F49098809B19807BC
:1034E80005D41E4B1B88003318BF0123C3B3022326
:1034F80013702B7823F001032B7036E0081000209E
:10350800302F00203C12002048120020041900200F
:1035180014190020562F0020407E05004C12002070
:1035280054110020541200205A1200200C240020AC
:103538004C1300205824002044130020401300207E
:10354800202F0020142E00204813002000080048D7
:10355800501200204C2F0020141500204E2F002060
:103568002978C90758BF0223137003F037FAAF4B05
:103578001B68C01A002801DB0EF0F2FC0EF00CFBF1
:10358800AB4B1E789846002E00F0A980A94E3368F0
:10359800002B00F0D286306803F0F7FA002800F01C
:1035A800CC86A44BA44C186803F0ECFA092801D087
:1035B8003F2850D14FF0000AD4F800909F4D57464D
:1035C800B9F1000F05D09E4829684A4611F074FDEC
:1035D80010B9AA4607B92F469A4B10359D42EFD32A
:1035E800C7B1D7F800E0DAF800C023681EF8035026
:1035F8001CF80300A8420DD15A1C914938B92D2B4B
:1036080005D88D4D2A602025CD54885402E0CD542C
:103618002260EAE723680BB1574511D08A480CF0BD
:103628004FFC574507D857F8100B0CF049FC0920F8
:103638000CF03EFCF5E785480CF042FC4FF0000921
:1036480023689945A7D27E4B13F809000CF030FC8B
:1036580009F10109F4E72368002B40F05286042899
:1036680040F09486764807F025FA00F066BED9F84F
:103678000000DFF8E8A103F088FA30B3DAF80000B8
:1036880003F080FADBF8003093F84810024600296E
:1036980033D124286AD1012283F84820DBF800308E
:1036A800DFF8B4A193F84820062AE0D193F849003E
:1036B80001F0F0FB834600287BD03B6898790CF03A
:1036C80048FB3B68002283F84820614B93F835306B
:1036D800002B40F004864C36982E00F02E865D4B69
:1036E800F21892F84A100129F5D15B4FF3583A6065
:1036F8005A4ABB4613609146B9E7012904D14D28BF
:1037080014BF00220222C7E7022904D13C2814BFB3
:1037180000220322C0E703290CD140284FF0000102
:1037280002D983F84810B9E758711971D97198719D
:103738000422B1E7042906D1997983F849004A405F
:103748009A710522A8E70529A8D1587919798842DC
:10375800987906D950409871481C18710B441A7210
:103768009CE790420CBF0622002295E72B78580769
:1037780094D4232ADAF800300ED1012188F80010F9
:103788002C4937480B60324902920B630CF098FBC6
:103798002E480CF095FB029A324B1B681B7893421B
:1037A80001BF314B314A1A60314B04BF314ADA60EC
:1037B80074E7DAF8002092F849304C2B00F0968430
:1037C80000F28580332B00F0CC8421D8292B00F01F
:1037D800598409D8252B00F01384272B00F017846F
:1037E800232B40F0CF8539E22D2B00F05C8407D8DD
:1037F8002B2B40F0C7850CF08FFA607100F06ABD82
:103808002F2B00F01A85312B00F02C8500F0BABD63
:103818003E2B00F0198144D8372B00F0D6842BD8E2
:10382800352B00F06F8200F0ADBD00BF242F0020C3
:10383800582F0020FC230020D0170020C07E01084C
:10384800A0170020708001085E970108639701089F
:103858000810002000220020F8120020FC1200208E
:1038680093970108A4220020FC9F0020EFBEADDE44
:1038780000ED00E00400FA05392B00F0D5833C2B5D
:1038880040F08085DFF84C94D9F800A00CF044FA99
:103898008AF80000D9F80030187809F071FC00F0B7
:1038A80019BD432B00F06E8406D8412B40F06A8581
:1038B8004FF0000900F05ABC442B00F007854A2B52
:1038C80040F060850CF032FAA08100F003BDD02BE7
:1038D80000F00F8355D8CA2B00F0C08009D8C82B38
:1038E80000F0858000F226834E2B00F00C8400F057
:1038F80049BDCD2B00F0088304D8CC2B00F02A82D8
:1039080000F040BDCE2B00F00883CF2B40F03A8565
:103918000CF00CFA6FF4AF6283189BB2C62B98BFF9
:10392800A4F898010CF002FAA4F844010CF0FEF98E
:10393800A4F846010CF0FAF9A4F848010CF0F6F9DD
:10394800A4F8DA010CF0E8F984F8EB010CF0E4F9DA
:103958000CF0E2F984F8EC010CF0DEF984F8870148
:103968000CF0DAF984F894010CF0D6F9D94BD3F8B5
:1039780000900CF0DBF900EB80004000A9F856003D
:1039880052E3D62B00F039820AD8D22B19D0C0F0D6
:10399800F882D32B25D0D42B00F03B8200F0F2BC68
:1039A800EF2B41D005D8D82B40F0EC844FF0000A1B
:1039B800E6E0F22B00F07582FA2B00F0B78200F0F7
:1039C800E1BC2B78590700F185840CF0A5F9022891
:1039D80084F8AC0740F29382BF4B002283F8AC27EF
:1039E8008DE20CF0A3F9BD4B188000F073BC92F87F
:1039F80005904FEA5909B9F1120F03D90BF0C0FC31
:103A080000F068BC4FF0000ACA4507D20CF08EF9E6
:103A1800B34B23F81A000AF1010AF5E7B14B01226A
:103A280083F8342000F056BCDFF8A892D9F800A03B
:103A38000CF07CF9AAF85A00D9F800900CF076F945
:103A4800A9F8580000F046BC0CF066F984F8DE01CD
:103A58000CF062F984F8DD0100F03CBC9D4B1A685B
:103A68001278022A824699466FD1D9F800B00CF034
:103A780053F907EE900AF8EE677AB2EE048AC7EEB9
:103A8800887A0BEB8A0BCBED087AD9F800B00CF0EA
:103A980043F907EE900A9FED947AF8EE677A0BEBFC
:103AA8008A0BC7EE877ACBED0B7AD9F800B00CF009
:103AB80033F907EE900A9FED8D7AF8EE677A0BEBF3
:103AC8008A0BC7EE877A0AF1010ABAF1030FCBED28
:103AD8000E7ACAD1BAF1070FD9F800B01CD10CF090
:103AE8001BF907EE900AF8EE677AC7EE887ACBEDF5
:103AF800117AD9F800B00CF00FF907EE900AF8EE39
:103B0800677AC7EE887ACBED127AD9F800B00CF054
:103B180003F98BF84C0012E00CF0FEF8D3448BF854
:103B28000100D9F800B00CF0F7F8D3448BF80B007B
:103B3800D9F800B00CF0F0F8D3448BF815000AF16E
:103B4800010ABAF10A0FC5D1C4E3D9F800B00CF0E4
:103B5800E3F8D3448BF80100D9F800B00CF0DCF896
:103B6800D3448BF80B00D9F800B00CF0D5F8D34447
:103B78000AF1010ABAF10A0F8BF81500E5D1A9E399
:103B8800DFF850919FED598AD9F800B00CF0CEF8C3
:103B980007EE900AF8EE677A0BEB8A0BC7EE887A85
:103BA800CBED087AD9F800B00CF0C0F807EE900A0F
:103BB800F8EE677A0BEB8A0BC7EE887ACBED0B7AB7
:103BC800D9F800B00CF0B2F807EE900AF8EE677A70
:103BD8000BEB8A0BC7EE887A0AF1010ABAF1030FD8
:103BE800CBED0E7ACCD1BAF1070FD9F800B01CD1C1
:103BF8000CF09CF807EE900AF8EE677AC7EE887A20
:103C0800CBED117AD9F800B00CF090F807EE900AD5
:103C1800F8EE677AC7EE887ACBED127AD9F800B059
:103C28000CF084F88BF84C0012E00CF07FF8D344C9
:103C38008BF80100D9F800B00CF078F8D3448BF871
:103C48000B00D9F800B00CF071F8D3448BF81500CC
:103C58000AF1010ABAF10A0FC5D13BE30CF05CF88E
:103C6800132883463FF6CAAEDFF868A0DAF800905A
:103C78000CF052F800231E4A0C2101FB0322117A92
:103C8800814222D10FFA8BFB09EB8B09137889F853
:103C980079300CF041F889F87A000CF03DF889F891
:103CA8007B000CF039F8134B134A1A6089F87C0032
:103CB800124BDAF8000018600021793002F054FE47
:103CC8000F4B80F00100187004E301331B2BD2D195
:103CD80094E600BF9011002094240020780F002063
:103CE80070240020081000200000C84200007A4418
:103CF80068780108700F0020D8250020740F002074
:103D0800030000200CF008F80B2882463FF676AE38
:103D1800CE4BD3F800900BF0FFFF03283FF66EAEB2
:103D2800062303FB0A9989F8CE000BF0F5FF89F802
:103D3800C9000BF0F1FF89F8CA000BF0EDFF89F814
:103D4800CB000BF0E9FF89F8CC000BF0E5FF89F810
:103D5800CD00BFE25379092B7FF650AE019BD3F813
:103D680000900BF0D9FF019B89F80000D3F8009070
:103D78000BF0D2FF89F801000BF0CEFF019B6428FD
:103D88001B68A8BF642018710BF0C6FF019B64284C
:103D98001B68A8BF642058710BF0BEFF019BFF2869
:103DA8001B68A8BFFF2098710BF0B6FF019B642821
:103DB800D3F8009028BF642089F807000BF0ACFF07
:103DC800019B89F80200D3F800900BF0A5FF019B36
:103DD80089F80300D3F800900BF0A8FF3B68A9F816
:103DE8000A005B790A2B40F27582994BD3F8009050
:103DF8000BF092FF89F808006CE282460BF096FF00
:103E0800944B23F81A000AF1010ABAF1080FF5D108
:103E180060E253790F2B7FF4F1AD0BF07DFF07289B
:103E280081463FF6EBADDFF824A2DAF800B00BF0DC
:103E38007DFF0E2303FB09F9CB44ABF81901DAF82F
:103E480000B00BF073FFCB44ABF81B01DAF800B0FD
:103E58000BF06CFFCB44ABF81D01DAF800B00BF0A7
:103E68005BFFCB448BF81F01DAF800B00BF054FF6E
:103E7800CB448BF82001DAF800B00BF04DFFCB44AF
:103E88008BF82101DAF800B00BF046FFCB44DAF8E2
:103E980000A08BF822010BF053FFD144C9F823018D
:103EA80018E20BF039FF0F2881463FF6A7AD0BF05B
:103EB80033FFC9EBC909A14489F8D4000BF02CFFE2
:103EC80089F8D5000BF028FF89F8D6000BF024FFFD
:103ED80089F8D7000BF020FF89F8D8000BF01CFFF9
:103EE80089F8D9000BF018FF89F8DA0002F0EEFF24
:103EF800F0E12B785B0700F1ED810CF019FA06F080
:103F080035FA06F0EDFAE5E12B78580700F1E28181
:103F1800514B4FF4C8721A80DCE12B78590700F135
:103F2800D9814E4A137843F0040328E02B785A07C6
:103F3800E5D527E20BF0F0FE484B1A7810B142F0B5
:103F4800020201E022F002021A700BF0E5FE444B77
:103F5800DFF82C9118700BF0F3FEC9F800000BF095
:103F6800EFFEC9F804000BF0E1FE3E4B18800BF0A1
:103F7800DDFE3D4B3D4A1880137843F00203137071
:103F8800A8E10BF0C9FE02900BF0DAFE83460BF0B5
:103F9800D7FE82460BF0D4FE81460BF0C7FE0BF02D
:103FA800C5FE0BF0B9FE029BA3B9314B1020C3F834
:103FB80000B0C3F804A006F086F9284A137843F045
:103FC80001031370B9F1000F00F08481294BC3F885
:103FD80000907FE1102B40F07D81274BC3F800B0A3
:103FE800C3F804A0B9F1000F02D0224BC3F8009027
:103FF8002148224B0222011D1A7005F063FC69E179
:10400800A0600BF09DFEA3681843A06062E10BF06E
:104018008DFEA4F85C010BF089FEA4F85E010BF09C
:1040280085FEA4F8600155E10BF076FE84F87C016A
:104038000BF072FE84F880010BF06EFE84F87F01AD
:104048000BF06AFE84F8810144E100BF9011002062
:10405800B4110020E223002014150020541200207F
:104068005A1200205812002056120020BA110020BF
:10407800BC110020CC110020C41100207C0F0020AE
:104088005C1200200BF052FEA4F882010BF04EFEE9
:10409800A4F884010BF040FE84F886010BF046FE7C
:1040A800A4F8880116E10BF037FE84F892010BF0B2
:1040B8003DFEA4F89C010BF039FEA4F898010BF022
:1040C80035FEA4F89A010BF027FEDAF8003084F8E0
:1040D80093015B79082B40F2FD800BF027FEA4F8D2
:1040E8009E010BF023FEA4F8A001F3E00BF014FEF0
:1040F80084F8D8010BF010FE84F8D9010BF016FEF5
:10410800A4F8DA01E6E092F805900323B9FBF3F985
:10411800B9F1120F3FF672ACDFF888A34FF0000B2D
:10412800CB4580F0D7800BF0F7FD8AF8A2010BF0A1
:10413800FDFD40F2ED23984205DD40F6CA039842A2
:10414800A8BF184601E040F2EE20A0F2EE201923A5
:104158000BF1010B90FBF3F00AF1020A8AF8A101B6
:10416800DEE70BF0D9FD84F89401B3E00BF0D4FD41
:1041780004EB090309F10109B9F1080F83F88A0171
:10418800F4D1A7E00BF0C8FDC4F808B060710BF0DB
:10419800D7FDA3681843A0600BF0BEFD84F8920118
:1041A8000BF0C4FDA4F85C010BF0C0FDA4F85E019F
:1041B8000BF0BCFDA4F860010BF0B8FDA4F8820177
:1041C8000BF0B4FDA4F8840184E053794FF0070A9A
:1041D800B3FBFAF2C2EBC2029A1A12F0FF0F7FF495
:1041E8000DACB3FBFAFA0AF1FF3A5FFA8AFABAF1B0
:1041F800FF0F6FD00BF090FD5FFA80FB4FFA8BF04A
:1042080003F0FCFE814600283FF4F8AB80F800B0CC
:104218000BF08CFDA9F802000BF07EFD89F8040074
:104228000BF07AFD89F805000BF076FD89F8070098
:104238000BF072FD89F80600D5E7DFF8689209F1FE
:10424800400A0BF073FDA9F8A4020BF065FD89F88C
:10425800A6020BF061FD09F1040989F8A302D14512
:10426800EFD137E00BF058FD1F2881463FF6C6AB6B
:104278003B685B79082B7FF4C1AB0BF057FD09F164
:10428800880904EB890900F03F00A9F806000BF043
:104298004DFDB9F80630800100F4FE501843A9F826
:1042A80006000BF039FD000189F804000BF034FD1D
:1042B80099F8043000F00F00184389F804000BF057
:1042C8002BFD89F805000AF07BF903E0624B012217
:1042D80083F8352000200BF06BFDFFF7EEB95F4B3C
:1042E800985902F049FC18B9322002F09EFBF6E713
:1042F80002F0ACFD06F010F8594B5A4ADA60FFF7A5
:10430800EAB90C2844D00A284BD1574D57480BF02E
:10431800D7FD2846232110F0B8FE08B1401B2060C5
:104328002368002B60D1504823600021302210F010
:1043380076FE98F80030002B2DD14D4B1B689B065C
:1043480015D54C4B44491B688A6B9A1A002A0EDB18
:10435800494A1278042A0AD9484A03F5123303F560
:10436800F8738B63938A9BB283F480439382444BA4
:104378009B68002B6BD0434805B0BDEC028BBDE8B1
:10438800F04F18470AF0FCFFFFF797B90C2804D143
:104398003D480BF095FD3D480DE07F2812D1FFF711
:1043A800FAB80D28B1D07F2809D1013B2E4A3848E8
:1043B80023600021D1540BF083FDFFF7ECB82F2BBD
:1043C8003FF6E9A8A0F12002D2B25E2A3FF6E3A8A0
:1043D80013B920283FF4DFA85A1C2260224AD0547F
:1043E8000BF066FDFFF7D7B85A1EA95C202901D14A
:1043F800134696E71C4A23600021D154254B264DCD
:10440800D3F800A0D5F800B0DFF85C90584610F05B
:104418004AFE07463A464846594610F04DFE1F4A9E
:1044280028B919F8073053445B785B0703D0103577
:104438009542E7D306E0954204D2781CEB684844DD
:10444800984702E016480BF03BFD00236BE705B0E8
:10445800BDEC028BBDE8F08F081000200022002080
:1044680000ED00E00400FA05A017002021A30108D0
:1044780050120020302F00205A1200200008004857
:10448800A4140020441000206897010863970108CD
:104498008F97010818010020C07E0108708001086C
:1044A800739701089424002010F80A3C0133DBB20A
:1044B8000A2B84BF10F8131C044A00F80A3C82BF78
:1044C800002322F8113000F80A3C7047B42E00206F
:1044D800334A136C90681944081A40F68C239842A2
:1044E80070B513469160D06051603BD9127893F94A
:1044F80045108A4210460BD1111F082908D893F895
:104508004610182901D8013103E083F8442002E05D
:10451800002183F8461093F944402149A24219D159
:1045280091F84740B4B10C310024944206DA1D4D8D
:1045380051F8046F25F814600134F6E70C2805D00B
:104548001849002421F810400130F7E7164801788F
:104558000131017083F84520002201211A7083F887
:10456800471070BD92F84710C9B1A0F2EF2440F28D
:10457800DA518C4208D811780B2905D80B1D013166
:10458800117042F8230070BD002283F84720074BC2
:1045980003F13002002143F8041F9342FAD170BDA1
:1045A800B0010020B42E002084060020BC010020A9
:1045B800024A136C0133194411647047B00100209A
:1045C800024B53F820301B681960704750130020C5
:1045D800064B53F820301A681B89A1F57A715943A4
:1045E8004FF47A7391FBF3F1116070475013002078
:1045F800054B98420CBF054A054A138801339BB204
:1046080013800020704700BF005400405011002064
:1046180052110020F0B5046D8668236823F0010369
:1046280023608379054613F0020F40790CBF4FF0E1
:10463800000E4FF4005E13F0040F14BF4FF48067B0
:10464800002710F0010F14BF042100218307206800
:1046580020F001002060626822F440524EEA020213
:104668006260226822F4B05323F00C0348BF41F083
:1046780008013B430B432360A36895B023F44073C0
:10468800A360684607F082FB284B9C4201D10C9B33
:104698000EE0274B9C4201D10D9B09E0254B9C4223
:1046A80001D10E9B04E0244B9C420CBF0F9B109B36
:1046B8002268A879170448BF5B00B3FBF6F206FB33
:1046C8001233B3EB560F236828BF01321E0441BFD3
:1046D8004FF6F073C2F34201134041EA03026B79CB
:1046E80092B213F0020FA28100F0010114BF4FF43F
:1046F80000320022DC0748BF42F480322B6D11B132
:1047080059680A4302E0596821EA02025A609A6825
:1047180001074CBF42F0080222F008029A601A68AA
:1047280042F001021A6015B0F0BD00BF0038014028
:104738000044004000480040004C00403D4B1B78BE
:10474800012B30B514BF00240324B1B9036A23F048
:10475800010303628169036A21F0F30123F00A036C
:1047680041F0010142F001021A4341EA041181615A
:104778000262836923F00C031BE004291DD1016A3E
:104788004FF6EF730B4003628169056A120121F449
:1047980073414FF65F7342F0100241F480712B4071
:1047A80092B2134341EA043181610362836923F4BD
:1047B800406383618369836130BD0829016A1AD126
:1047C8004FF6FF630B400362C169036A9BB289B26B
:1047D80023F4206343F4807321F0F30143EA0222B7
:1047E80041F0010192B241EA0411C1610262C26959
:1047F8004FF6F37319E04EF6FF730B400362C3697B
:10480800056A40F6FF41194045F6FF732B4043F413
:10481800805343EA023241F4807192B241EA043192
:10482800C1610262C2694FF2FF331340C361C369B9
:10483800C36130BDAC01002038B510F80E2C50F81B
:10484800043C044652B9012200F80E2C20F80C1C36
:10485800997A18680222BDE838406FE730F80C2CC6
:1048680020F80A1C891A89B220F8081C074A10F88F
:104878000F0C002522F8101004F80E5C1868997ABD
:104888002A46FFF75BFF04F8065C38BDB42E00200B
:10489800044B53F820301BB107289CBF1B681960D4
:1048A800704700BFD8020020084A13689B050BD543
:1048B800074B00211970074908684FF6FE7303403B
:1048C8000B604FF400735360704700BF0000024054
:1048D800552F0020300002402DE9F047664D2B6827
:1048E80066490A78581C02F0FF068E460AB103464C
:1048F800F6E72B60687BAB6895F80C80AA7B374697
:1049080039B2202900F09B80DFF880C10CEB8103CD
:104918003CF82110DC789B78C3F1FF039BB2002B95
:1049280065D0C3F1FF0363434FF03C0C1B12B1FB8E
:10493800FCF9B9F1050F5DD8DFE809F0030B1A2976
:104948003A4AE01ADAB24143B1FBFCF01044C0B273
:1049580051E0B1FBFCF00CFB101189B2DAB2C1F1E5
:104968003C01E31A4B432046B3FBFCFC94442CE087
:10497800B1FBFCF00CFB10115FFA83F8E21A89B264
:104988004A43B2FBFCF24244D2B2204632E0B1FBC9
:10499800FCF90CFB191189B25FFA83F8E01AC1F12E
:1049A8003C014843B0FBFCF04044C0B2224621E041
:1049B800B1FBFCF80CFB1811D8B289B2E31A01FB61
:1049C80003F2B2FBFCFC224684445FFA8CF412E04A
:1049D800B1FBFCF80CFB181189B2D8B2C1F13C014B
:1049E800E31A4B43B3FBFCF20244D2B203E0224683
:1049F800204600E044464FEA042C4CEA004C4CEABE
:104A0800020C172306F117014FF0010808FA03F802
:104A1800C91A18EA0C0F89B2DFF8748014BF4FF076
:104A280011094FF0090913F1FF3308F80190E9D291
:104A380018360137B6B2BFB2114BA04660E7AA7369
:104A4800AB60104AE98001238EF800300E4985F8E2
:104A58000C8040F22A336873AE80536000234B62A7
:104A68000B889BB243F001030B80136843F00103EA
:104A78001360BDE8F08700BF48100020552F0020C4
:104A8800541000203000024000440140F20D002084
:104A98002D03002073B506460D46002401232A88FD
:104AA800A34013421AD0AA78009302F003038DF8AA
:104AB8000430EB78022B03D0032B0CBF0323012314
:104AC8008DF805303046C2F301136946C2F38102FE
:104AD8008DF806308DF8072007F0C6FA0134102C3F
:104AE800DCD102B070BD2DE9F04F734EF57B07465F
:104AF8000C4687B011469A4600686B1C91462246C0
:104B08004FF0020BF3730AF011FF3B897868ADF898
:104B1800043001A98DF806B08DF807B0FFF7BAFF89
:104B28000023ADF80A30ADF81230ADF81630702316
:104B38000193BA7A3C68CDF80CA0012306F110085D
:104B48002D01ADF808304FF48073A844ADF810B0CB
:104B5800ADF814300C2A7ED8DFE802F0077D7D7DA1
:104B68000F7D7D7D387D7D7D5E00204601A907F0A3
:104B7800CFF8A36943F0080326E0236A4F4823F0DF
:104B880010032362236A6168A26922F0807222F40A
:104B9800E642844242F4E04206D000F500608442D6
:104BA80002D043F0300307E023F0E00321F4406132
:104BB80043F0300341F480616160A261C4F838A019
:104BC8002362A36943F40063A36144E0236A3B487A
:104BD80023F480732362226A6168E369844223F0C4
:104BE800730343F0700306D000F50060844202D0DE
:104BF80042F4407207E022F4606221F4405142F42A
:104C0800407241F480516160E361C4F83CA02262C3
:104C1800E36943F008031DE0236A284823F480531E
:104C28002362226A6168E369844223F4E64343F419
:104C3800E04342F4405203D000F50060844201D1C1
:104C480041F480416160E361C4F840A02262E369F5
:104C580043F40063E3613A7B3B681AB15A6C42F44F
:104C680000425A641A8892B242F001021A80BA7A53
:104C78000C2A18D8DFE802F0071717170B171717B1
:104C88000F1717171300721903F134010AE072198C
:104C980003F1380106E0721903F13C0102E07219D0
:104CA80003F14001116135444046A5F818906B6145
:104CB80007B0BDE8F08F00BF48100020002C01406D
:104CC800F8B53A4E3A4C4000C7B24FF42045306828
:104CD800C4F8D050D0F818E01EF4004F05D0AE4606
:104CE800013DBEF1000FF5D116E0D0F804E0314DDA
:104CF8000EEA050545F490353D4345604FF42045DF
:104D0800C4F8D050D0F818E01EF0020F2DD1AE46EE
:104D1800013DBEF1000FF5D1C4F8D0501FE029467F
:104D2800013D0029F8D081694906F8D5C4F8D0506A
:104D380020494568294041F0007141F4105141EA89
:104D48000241394341604FF42041A2B1306885697E
:104D58006D071ED411F1FF31F9D2C4F8D010FFF756
:104D680047FC003018BF0120F8BD4FF42045816290
:104D7800C4F8D050D7E73068C4F8D0100B46826921
:104D880092060CD41A46013B002AF8D1C4F8D03058
:104D9800E5E7416A03F8011B013AD2B2D3E7C4F848
:104DA800D0302023C3610120F8BD00BF4C11002082
:104DB80048100020009800FC400070B5C5B2324889
:104DC800324B00684FF42044C3F8D040866936045B
:104DD80004D52646013C002EF8D113E046682C4C39
:104DE800344044F0807444F490342C4344604FF4CD
:104DF8002044C3F8D0408669B60729D42646013C2A
:104E0800002EF8D1C3F8D0401CE02146013C00290F
:104E1800F8D081690E06F8D544681D49214041F053
:104E2800007141F48031294341604FF42041C3F8B7
:104E3800D0108469A40711D40C460139002CF8D18C
:104E4800C3F8D010FFF7D4FB003018BF012070BDA5
:104E58004FF420448162C3F8D040DAE782624FF40D
:104E68002042C3F8D0208169890606D41146013A48
:104E78000029F8D1C3F8D020E4E7C3F8D0202023D4
:104E8800C361012070BD00BF4C11002048100020F4
:104E9800009800FC2DE9F0474D282DED028B0446C3
:104EA80000F05A8600F2B980302800F0BB8651D84D
:104EB800222800F0978423D8032800F0058214D80C
:104EC800012800F0F581022840F0FB8604200AF052
:104ED8006FFF43200AF03DFF4C200AF03AFF4620BE
:104EE8000AF037FF4C2000F05DBE042800F0F58181
:104EF800052840F0E6861A200AF05AFF0024FCE153
:104F0800282800F0E88515D8242800F0CF85262821
:104F180040F0D786D94C06200AF04AFFB4F85C0165
:104F28000AF049FFB4F85E010AF045FFB4F86001E1
:104F380000F0B9BD2C2800F0E1852E2800F05C8631
:104F48002A2840F0BE8601200AF032FFCB4B587960
:104F580000F028BE3D2800F0F8821ED8362800F060
:104F680032860BD8322800F01786342840F0A986FC
:104F780048200AF01DFF002500F056BC3A2800F032
:104F8800BB823B2800F02784382840F09A8604200A
:104F98000AF00EFFB94C00F08FBD452800F07E8660
:104FA80027D8402800F00186422840F08A86B34C72
:104FB80010200AF0FDFE60790AF0CBFEA0680AF026
:104FC80003FF94F892010AF0C4FEB4F85C010AF0F9
:104FD800F2FEB4F85E010AF0EEFEB4F860010AF0E1
:104FE800EAFEB4F882010AF0E6FEB4F8840100F0A3
:104FF8005ABD492800F0B4824B2800F09E85462807
:1050080040F05F860D200AF0D3FE00200AF0A1FED2
:1050180000200AF0D9FE00F04CBE702800F0F082A3
:1050280000F2DE80692800F0478200F2AF8066282F
:1050380000F0A18100F29F80642800F07781652844
:1050480040F03F868E4C0B200AF0B2FE20880AF012
:10505800B2FE62688B4B9A420CBF2089608980B28D
:105068000AF0A9FE884B1B68C3F3C000C3F3800293
:10507800800040EA4200C3F340021043C3F34012E9
:1050880040EAC20003F0100318430AF094FE7F4B75
:105098001A88E36812F0010F14BF4FF0020C4FF0AA
:1050A800000C12F0020F02F0080814BF4FF0040EB3
:1050B8004FF0000E03F4475912F0040F14BF1027E5
:1050C800002749EA080912F0400F03F4804814BF8A
:1050D8002026002649EA080912F0100F03F40048B8
:1050E80014BF4FF40075002549EA080912F0200F93
:1050F80003F4803814BF4FF48060002049EA08099F
:1051080012F4807F03F4003814BF4FF400610021CB
:1051180049EA080912F4007F03F480285C4A49EA46
:10512800080903F4002849EA0809127803F48018EA
:1051380049EA080903F0007349EA0303C2F380024D
:1051480043EA020343EA0C0343EA0E0E4EEA07075A
:1051580046EA070645EA060540EA050041EA000175
:1051680014BF4FF400184FF00008002041EA080867
:105178000346217CEAE0672800F02581682840F092
:10518800A08510200AF014FE00248CE16C2800F0A1
:10519800A68117D86A2800F00B846B2840F0918507
:1051A80005200AF005FE3B4B18880AF004FE3A4B2E
:1051B80018880AF000FE324B93F8720000F00100E4
:1051C80000F0F0BC6E282E4D00F09A8100F2CE81DE
:1051D80006200AF0EDFD686E0AF0F6FD2F4B89E116
:1051E800782800F0FD8018D8742800F03E830AD88B
:1051F800722800F09D83732840F0638508200AF028
:10520800D7FD0124CDE3762800F0F28300F266830F
:105218002F200AF0CDFD224CD5E2A42800F00F84FF
:1052280014D87B2800F07582A02840F04A850C200D
:105238000AF0BEFD1B4B18680AF0C6FD1A4B186829
:105248000AF0C2FD194B186800F037BDF12800F0CC
:105258000381FE2800F01A84F02840F03285084CBB
:1052680004200AF0A5FDA36CB3F85A000AF0A3FDC8
:10527800A36CB3F8580000F016BC00BF94240020BB
:10528800481100200054004050120020181300203C
:10529800562F0020CE120020D01200202412002009
:1052A80037780108ACF7FF1FB0F7FF1FB4F7FF1FEF
:1052B80003200AF07DFD00200AF04BFD20460AF08D
:1052C80048FD0C2000F06EBC0AF072FD01200AF0C7
:1052D80040FD0A200AF03DFDAFE306200AF068FD14
:1052E80043200AF036FD4C200AF033FD42200AF034
:1052F80030FD52200AF02DFDD4E3B04B185D013487
:105308000AF027FD0B2CF8D10024AD4B185D0134B1
:105318000AF01FFD082CF8D10024AA4B185D0134AF
:105328000AF017FD072CF8D100F0C9BC07200AF0D5
:105338003FFDE7200AF00DFDA34B58790AF009FD5F
:1053480000200AF006FD042000F0B7BC8B420BD207
:105358009E4A9C5C012202FA04F414EA080F1CBF5E
:105368009A4010430133F1E70AF02EFD964B93F86B
:10537800AC0700F017BC12200AF01AFD944B1B88EA
:10538800B3F5806F8CBF082501250024914B33F9B4
:10539800140090FBF5F0013480B20AF00CFD032CE8
:1053A800F4D18D4CA08D0AF006FDE08D0AF003FDC6
:1053B800208E0AF000FD608E0AF0FDFCA08E0AF037
:1053C800FAFCE08E6FE310200AF0F2FC0024834B15
:1053D800185D01340AF0BDFC102CF8D100F06FBC48
:1053E80070200AF0E5FC00267B4D0E24AB6C74435C
:1053F80023440136B3F819010AF0DDFCAB6C2344F1
:10540800B3F81B010AF0D7FCAB6C2344B3F81D01B9
:105418000AF0D1FCAB6C234493F81F010AF099FC05
:10542800AB6C234493F820010AF093FCAB6C234443
:1054380093F821010AF08DFCAB6C234493F8220108
:105448000AF087FCAB6C1C44D4F823010AF0BCFCBE
:10545800082EC9D100F033BC70205B4C0AF0A8FCC0
:1054680004F1700594F8D4000AF073FC94F8D500A0
:105478000AF06FFC94F8D6000AF06BFC94F8D70099
:105488000AF067FC94F8D8000AF063FC94F8D90095
:105498000AF05FFC073494F8D3000AF05AFCAC42D7
:1054A800E0D100F00CBC4E4B185D01340AF051FC01
:1054B800102CF8D100F003BC4A4D2878400000F0C9
:1054C800FE000AF075FC00242B789C4280F0F783DC
:1054D800454B33F814000AF06EFC0134F4E7434CF2
:1054E80006200AF065FC20880AF065FC60880AF04E
:1054F80062FC3F4B1888D6E204200AF059FCDBE333
:1055080007200AF055FC3B4B1888FF28A8BFFF204E
:10551800C0B20AF01EFC384B186880F3100080B245
:105528000AF049FCB5F868000AF045FC264B93F8E8
:105538008721324B186822B10A23584380F31000A0
:1055480001E000F30F0080B2ADE21F4C02200AF028
:105558002FFC94F8DE010AF0FCFB94F8DD0121E34E
:1055680002200AF025FC184B98899CE20B200AF0CF
:105578001FFCEB6E18780AF0ECFBEB6E58780AF01B
:10558800E8FB0026EB6E144C3344013618790AF018
:10559800E0FB032EF6D1E36ED8790AF0DAFBE36E6E
:1055A80098780AF0D6FBE36ED8780AF0D2FBE36E5F
:1055B80058890AF000FCE36E187AF3E2989401081F
:1055C800A49401087994010894240020591100201A
:1055D800040000201E120020481100208011002025
:1055E800941100209C220020702400202C240020EC
:1055F8002C120020401200204C12002048120020DB
:10560800C64C1E200AF0D4FBA36C1B78022B4FF06B
:1056180000056BD1A36C03EB850393ED080AB2EE8A
:10562800048A20EE080A0FF009FF80F30800C0B2D0
:105638000AF08FFBA36CDFEDBA7A03EB850393EDD9
:105648000B0A20EE270A0FF0F9FE80F30800C0B21B
:105658000AF07FFBA36CDFEDB37A03EB850393EDD0
:105668000E0A20EE270A0FF0E9FE80F30800C0B208
:1056780001350AF06EFB032DCCD1072DA36C23D185
:1056880093ED110A20EE080A0FF0D8FE80F3080007
:10569800C0B20AF05EFBA36C93ED120A20EE080A72
:1056A8000FF0CCFE80F30800C0B20AF052FBA36CE6
:1056B80093F84C3000EE103AB8EE400A0FF0BEFEF8
:1056C80080F30800C0B20BE02B4458780AF041FB85
:1056D800A36C2B44D87A0AF03CFBA36C2B44587D6E
:1056E80001350AF036FB0A2DC7D1E8E2A36C2B443A
:1056F80058780AF02EFBA36C2B44D87A0AF029FBC1
:10570800A36C2B440135587D0AF023FB0A2DEDD1FB
:10571800D5E23C200AF04CFB0024804D9FED818AA5
:10572800AB6C03EB840393ED080A20EE080A0FF034
:1057380085FE80B20AF03FFBAB6C03EB840393ED6C
:105748000B0A20EE080A0FF079FE80B20AF033FB4C
:10575800AB6C03EB840393ED0E0A20EE080A0FF0FE
:105768006DFE013480B20AF026FB032CD5D1072C3C
:10577800AB6C16D193ED110A20EE080A0FF05EFE0D
:1057880080B20AF018FBAB6C93ED120A20EE080AFF
:105798000FF054FE80B20AF00EFBAB6C93F84C008D
:1057A8000BE0234458780AF006FBAB6C2344D87A04
:1057B8000AF001FBAB6C2344587D01340AF0FBFA74
:1057C8000A2CD4D17BE214F8010F002800F077826C
:1057D8000AF0BFFAF7E701200AF0EAFA4F4B9B6C90
:1057E8001878DFE150200AF0E3FA00254B4B9C6C57
:1057F8004D4B04EB85040C2194F8792001FB02330E
:10580800013593F838000AF0A4FA94F87A000AF0FF
:10581800A0FA94F87B000AF09CFA94F87C000AF04D
:1058280098FA142DE2D14AE23C4B9C6C062303FB08
:105838000544013594F8CE000AF08BFA94F8C900B3
:105848000AF087FA94F8CA000AF083FA94F8CB00B1
:105858000AF07FFA94F8CC000AF07BFA94F8CD00AD
:105868000AF077FA0C2DDFD129E24FF00008012663
:1058780000272A4B1A7C974227DA11330024FA5C56
:10588800294D0C2305F130016343595C914207D13E
:105898002B44586B0FF007FC82462EB9B14605E041
:1058A80001341B2CECD10EE080440CE0D1450ADA1F
:1058B8000C2303FB04535B6B13F809000AF049FA45
:1058C80009F10109F2E70137D3E7002E00F0F7816B
:1058D8005FFA88F00AF06CFA0026C9E70F4D287CB9
:1058E8000AF066FA00242B7C9C4280F0E8810F4B7A
:1058F800E65C00210C480C2200F1300702FB01F3A2
:10590800DA5DB24205D1034493F838000AF021FA6F
:1059180002E001311B29EDD10134E4E748110020F0
:105928000000C84200007A44387801085911002064
:10593800CF4C16200AF03CFAB4F898010AF03BFA6A
:10594800B4F844010AF037FAB4F846010AF033FA19
:10595800B4F848010AF02FFAB4F8DA010AF02BFA81
:1059680094F8EB010AF0F5F900200AF0F2F994F83E
:10597800EC010AF0EEF994F887010AF0EAF994F8D4
:1059880094010AF0E6F900200AF0E3F9B94B9B6CA0
:105998000A20B3F9563093FBF0F080B20AF00BFA04
:1059A8008AE0E0B201340AF0D4F9092CF9D186E191
:1059B80010200AF0FDF9B04BB04C187800F0020046
:1059C8000AF0C7F9AE4B18780AF0C3F920680AF054
:1059D800FBF960680AF0F8F9AA4B18880AF0EBF9A5
:1059E800A94B18880AF0E7F9A24BB3F870005AE0FF
:1059F8000AF092F9074612200AF0DAF99D4C17B915
:105A0800666FA56F06E0102F13BF0025E66FD4F868
:105A180080502E4638460AF09CF930460AF0D4F9F0
:105A280028460AF0D1F9D4F884000AF0CDF900200C
:105A38000AF0C1F900200AF0BEF90020B2E08D4D4D
:105A480095F8880080000130C0B20AF0B1F995F8E5
:105A580088000AF07EF900242E4696F888309C4289
:105A680080F02D81894D285D0AF073F905F1100346
:105A7800185D0AF06EF905F120033035185D0AF05B
:105A880068F9285D0AF065F90134E6E708200AF0AC
:105A98008FF900200AF08FF900200AF08CF9002015
:105AA8000AF089F900200AF086F908E104200AF0D2
:105AB8007FF96F4B986800E194F87C010AF049F986
:105AC80094F880010AF045F994F87F010AF041F949
:105AD80094F8810166E0664C07200AF069F9B4F889
:105AE80082010AF068F9B4F884010AF064F994F8BC
:105AF80086010AF02EF9B4F88801D4E75C4C0C2032
:105B08000AF056F994F892010AF023F9B4F89C01C6
:105B18000AF051F9B4F898010AF04DF9B4F89A016D
:105B28000AF049F994F893010AF013F9B4F89E01C0
:105B38000AF041F9B4F8A001B5E74D4C04200AF089
:105B480037F994F8D8010AF004F994F8D9010AF061
:105B580000F9B4F8DA01A6E74D4C4E4D207800EB79
:105B68004000C0B20AF024F9002623789E4205F1CD
:105B7800020580F0A48015F8020C0AF0EAF815F87E
:105B8800010C00EB800000EB800000F2EE2080B2F8
:105B98000AF011F90136E8E701200AF009F9344B57
:105BA80093F894010AF0D5F889E008200AF000F982
:105BB80000242F4B2344013493F88A010AF0C9F8D2
:105BC800082CF6D17BE02B4B294C93F8C900C0EB8D
:105BD800C000C0B20AF0ECF804F1200594F8F20114
:105BE80000232D4AD25C90426DD00C33302BF8D173
:105BF8000834AC42F2D162E040201D4C0AF0D8F8DB
:105C080004F14005B4F8A4020AF0D5F894F8A60205
:105C18000AF09FF8043494F8A3020AF09AF8AC4208
:105C2800F0D14CE0E020124C0AF0C2F804F18005F3
:105C3800B4F8260200F03F000AF0BDF8B4F82602D6
:105C4800C0F386100AF0B7F894F8240200090AF0A5
:105C580080F894F8240200F00F000AF07AF804346F
:105C680094F821020AF075F8AC42E1D127E000BFB0
:105C78009424002048110020541200205C120020B7
:105C88005A1200205812002056120020D11100206C
:105C98009C22002036260020A822002013200AF08B
:105CA80087F80024154B185D01340AF052F80B2CC4
:105CB800F8D100200AF088F800200AF085F80120C1
:105CC80018E0002016E00AF044F8B4F8F4010AF0ED
:105CD80072F894F8F6010AF03CF894F8F7010AF023
:105CE80038F894F8F9010AF034F894F8F8010AF051
:105CF80030F87DE7BDEC028BBDE8F0879894010889
:105D08002DE9F047C24CC34E237886B00746002BD6
:105D180000F0048232686368D31A7C2B40F2FE815B
:105D2800237A6260013323724FF0000808F12400DF
:105D3800B74DC0B20BF020FF05F10A0333F9183054
:105D480007EE903AB44B1B88B8EEE77A07EE903A24
:105D5800F8EEE77A08F10108C7EE277A9FEDAF7AE7
:105D680067EE877AFDEEE77ACDED037ABDF90C0090
:105D78000BF0F0FEB8F1030FD8D130200BF0FCFE89
:105D8800B5F910000BF0E6FE0BF0EEFE2B7A9A0741
:105D98002CD16A6841F288339A4218D910200BF046
:105DA800EBFE4FF06408686990FBF8F000B20BF066
:105DB800D1FE21200BF0E0FE686990FBF8F308FBA8
:105DC80013000028B8BF404200B20BF0C3FE1420F5
:105DD8000BF0D2FEB4F918000BF0BCFE1C200BF03F
:105DE800CBFE00200BF0B6FE0BF0BEFE237ADFF8E8
:105DF80020825B0740F06F8102200BF0BDFED8F8CF
:105E08001C00DFF82C926423323090FBF3F000B2D0
:105E18000BF0A0FE0320B8F926500BF0ADFE804B26
:105E28001B7813F0040F4FF0050A95FBFAF5ADB295
:105E38000BD038460BF09EF828B9D9F8003013F08B
:105E4800100F18BF002528B205E0D8F82830988927
:105E5800B0FBFAF000B20BF07DFED9F800309F07D6
:105E680040F18180DFF8CC91E78D99F80030A28D60
:105E7800674D3F014FF06408BFB208FB02325B0078
:105E8800B2FBF3F347EA0327BFB2C3F303231F436D
:105E980006200BF071FE38B20BF05CFEE38D99F82A
:105EA800001001339BB293FBF1F201FB1233E3853F
:105EB800236B9B7B012B05D139200BF05DFEB5F9D7
:105EC8002C0019E0AD8D6E233A205D4315270BF0A9
:105ED80053FE95FBF7F5AFB2B7FBF8F528B20BF018
:105EE80039FE08FB15753B200BF046FEA8B2451D90
:105EF8000A2095FBF0F000B20BF02CFE28200BF0E6
:105F08003BFE636B424D0A2093FBF0F000B20BF0AE
:105F180021FE04200BF030FEA36AA86B9A894FF685
:105F2800FF739842A8BF1846C2B10028ACBF131A25
:105F3800134607EE903A9FED3B7AF8EEE77A67EE64
:105F4800877A07EE102AB8EEC77AC7EE877AFDEE91
:105F5800E77A17EE900A6428A8BF642020EAE07068
:105F680000B20BF0F7FDE36B294F9D0640F1A880C6
:105F780097F8403098071DD511200BF0FDFDB7F8B4
:105F88004200294B4FF4F365684390FBF3F000B2ED
:105F98000BF0E0FD19200BF0EFFDB7F84200454388
:105FA800642095FBF0F595FBF0F300FB135000B26D
:105FB8000BF0D0FD94F84030B4F8445013F0020FC1
:105FC80008BF002501200BF0D7FD28B20BF0C2FD59
:105FD80009200BF0D1FD00200BF0BCFD134B94F809
:105FE80046501A88B2F5967F0AD9094B1B7A03F0F6
:105FF8000F03072B04D842F20F75954228BF1546A8
:1060080005200BF0B9FD236B5B7BBBB928B232E0EE
:1060180014120020582400200400002000007A44B4
:10602800562F00200000C842A08601000A01002067
:1060380034240020080100206666E63FA5F120030D
:1060480007EE903A1FED047AF8EEE77AF6EE006A6A
:10605800C7EE877ABEEE007AF5EEC07AF1EE10FA56
:1060680058BFB0EE667A77EE877AFDEEE77ACDED27
:10607800037ABDF90C000BF06DFD94F84020C54B78
:10608800910703D493F84720012A04D1012384F807
:106098004730C1481BE01B6BDFEDC06A93ED017A06
:1060A800D3ED027A27EE267A67EEA67ABDEEC77A96
:1060B800FDEEE77A8DED047ACDED057A04A806E0C9
:1060C800B74A92E8030004AB83E80300184602F0DD
:1060D80011FE0BF049FD237A282B1FD1AD4B00226E
:1060E8001A723C2733684FF47A70B3FBF0F8172024
:1060F8000BF042FDB8FBF7F5B5FBF7F007FB1050C6
:10610800000200B20BF026FD18200BF035FD07FB4E
:10611800158000B20BF01EFD0BF026FD94F85030F0
:106128009C4D002B00F05B8100F058FC6B6D9D4A84
:10613800C31A9342074640F2C180002385F85A30BB
:1061480085F85C30AB8DDAB21B0A85F8762085F8C5
:10615800773085F86C2085F86D30D5F88420336861
:106168009A1AD5F88830D97B4FF47A734B439A4200
:106178000ED38D4B1B68C5F8843095F88C30013BE5
:10618800012B9FBF102385F85A30022385F85C3015
:106198000A20626B92FBF0F284F87420121284F8E1
:1061A800752094F84020A36B93FBF0F384F87830C3
:1061B8001B1284F87930920794F84630754984F8B0
:1061C800A73003D42D2381F8A83076E0042BD4F827
:1061D8004890E66CDFF8E081744A8CBF33233223A1
:1061E80081F8A8304FF0060C714B99FBF3F096FB41
:1061F800F3F308FB009108FB036803EB83030CFB34
:1062080001F103EB830391FBF2FE642502FB1E11EF
:106218009B0091FBF5F184F8991009120CFB08FC1E
:1062280084F89A109CFBF2F143FA81F39BB202FBCB
:1062380011C292FBF5F284F89E20121284F89C3069
:1062480084F89F201B0AB4F8422084F89D30242348
:10625800534393FBF5F5B4F8BA3084F8A03000EB5B
:1062680080001B0A00EB8000800084F8A1300A221D
:10627800B4F84430B3FBF2F303F5FA739BB240FA77
:106288008EF080B284F8A2301B0A4FEAD97984F8DC
:106298009700F60F000A84F8945084F8A330C5F3E9
:1062A8000725B4F8BC3084F8969084F8980084F8F0
:1062B8009B6084F8955084F8A930676594F8BE808F
:1062C800344DB8F1000F0DD1D5F8C40000F05DFCD5
:1062D800012807D90228374E00F0558202F0FCFC4D
:1062E8000123B370D4F8C8202A4D002A77D095F836
:1062F800BE603EB1D5F8D03040F6B731FB1A8B42BC
:1063080019D86CE00123D5F8C40085F8BE3001F037
:1063180028FDD5F8D43093F9000002238DE8480011
:10632800082132464FF4964301F02EFD85F8D860D7
:10633800C5F8C40051E095F8CC60CEB9D5F8C400D2
:10634800C5F8C86085F8BE6001F00BFDD5F8D430FB
:1063580093F9000001238DE84800082132464FF4E4
:10636800964301F011FDC5F8C40002F0B5FC34E015
:10637800013EF6B285F8CC6095F8D81095F8D9307A
:10638800E6B94A1C013385F8D82085F8D930D5F804
:10639800C40020E0141200205C1200208096184BE4
:1063A800B87901083F0D03005824002040420F002F
:1063B8008096980004000020806967FF12F8016B3E
:1063C800C5F8C820701885F8D8000133D5F8C4007E
:1063D80085F8D930314600F0DBFBC4F8D07094F86A
:1063E800DA309D4DF3B1D5F8DC30DBB1D5F8E030CB
:1063F800C3B1C5F8E4301B68984AC5F8E830D5F849
:10640800EC301344187AFEF745FDD5F8E430987956
:1064180009F09FFCD5F8EC300133092B88BF002325
:10642800C5F8EC308E4D94F8F0202E688A4B002A7F
:1064380000F0E381D3F8F420002A00F0DE8193F81D
:10644800F830013B012B00F2D881D4F8F400824FD8
:1064580000F09BFBE0B1D7F8F40000F093FB97F84D
:10646800F930D5F800907E2B80460ED102231B28E8
:1064780087F8F83009D1D7F8F40000F086FB20B986
:106488000123C7F8FC9087F8003184F8F980DCE72D
:10649800D7F8FC202B689B1A41F6583293421DD935
:1064A800032387F8F830A8E16E4A32F8130010B9D0
:1064B80003464FF403600133B0F5C06FDBB275D00B
:1064C8001DD9B0F5006F7AD031D9B0F5036F3ED140
:1064D80084F80131E36B604F99063FD494F80011BA
:1064E80094F80131002900F04B812A68921B012A97
:1064F800DAD984F80131002384F800317DE1B0F560
:10650800007F42D007D8B0F5807F47D0B0F5887FAC
:1065180000F08580E6E7B0F5806F00F0A780B0F561
:10652800826F00F0EC80B0F5047FDBD123E0B0F59A
:10653800E26F00F08480B0F5E46F00F08580B0F57C
:10654800E06FCFD184F80131B4F90A1080E0B0F5DA
:10655800046F6DD0B0F5026FC4D1FBE097F84030FE
:106568009A07BBD5B7F8421024234B431233642152
:1065780093FBF1F1FEE084F801313B4B364F1B6889
:106588009B07ABD5BB8D0A21F3E084F80131364B6C
:10659800314F1B681905A1D5796BEBE084F80131FF
:1065A800E36B2D4F5A0799D57969E3E084F80131F7
:1065B8002D4B294F1B681B0590D5B96BDAE0E16BB1
:1065C800254A84F801318F0688D592F8401088074B
:1065D80084D5D90711D5D36C83EAE371002BA1EBDD
:1065E800E37101EB51014FF01902B1FBF2F1ACBFBD
:1065F80041F0004141F040410EE0936C83EAE371C1
:10660800A1EBE371002B01EB51014FF01902B1FB33
:10661800F2F1B8BF41F080414FF4006089E084F89E
:106628000131E36B0C4F5B077FF558AF3969A1E087
:10663800B4F9181084F801316423594379E084F8D7
:106648000131B4F90C1003E0B4F90E1084F80131EB
:106658002C2391FBF3F16CE014120020B8790108A7
:1066680058240020A69801083424002084F8013119
:1066780094F80231624A0133DBB2032B88BF01234D
:1066880082F8023194F8021142F2107359435D4BBB
:106698001B78D80748BF01319A0748BF02315F0706
:1066A800B4F8043148BF0431D80748BF0A319A0703
:1066B80048BF14311F0648BF2831D80548BF2831C4
:1066C8005A0748BF64311F0748BFC831980548BFFB
:1066D80001F5C8719A0648BF01F57A71DF0648BF0F
:1066E80001F5FA61580648BF01F57A614FF48060F8
:1066F80002F0BEFA424B002283F80021EEE6E16B7D
:10670800DFF8FC8084F8013111F0200717D098F8E1
:10671800402012F0020F14BF4FF47A71002112F0DA
:10672800010F14BF4FF4FA6300230B4494F846108A
:10673800194402F09DFA002384F80031CEE6324B6A
:106748001B6819067FF5CAAE394602F091FA88F837
:106758000071C3E684F80131E36B294F9A067FF58F
:10676800BDAE97F840309B077FF5B8AEB7F8443018
:106778006421594302F07CFA002387F80031ADE622
:1067880084F8013139E0B37823B1C5F8C07086F8D0
:106798000280A7E5D5F8C030FB1AB3F57A6FFFF48D
:1067A800A1AD0123D5F8C400B37000F0EBF906469B
:1067B800D5F8C40000F0E6F976067FF493AD8A2890
:1067C80002D08E280CD08DE5EB6B98067FF58AAD4C
:1067D80095F8BE30002B7FF485AD05F18D0306E0FA
:1067E80095F8BE30002B7FF47DAD05F15803C5F850
:1067F800C8302D2385F8CC3074E506B0BDE8F087A5
:1068080014120020562F002034240020034B4FF48C
:10681800005208B19A6170471A8570470004004811
:10682800034B4FF4005208B11A8570479A617047BC
:106838000004004838B5294C2DED048B94ED008AEE
:10684800B0EE480A054603F09BFCF0EE408AB0EE35
:10685800480A03F032FC94ED019AB0EE408AB0EE9B
:10686800490A03F08DFCF0EE409AB0EE490A03F0B5
:1068780024FC95ED017AD5ED027A95ED006A68EE73
:10688800676A27EE088AE7EE286A68EE000A67EE6C
:10689800807AE6EE290AB0EE660AE7EEA80A0EF05C
:1068A800CFFEDFED0F7A20EE270ADFED0E7A80EEBD
:1068B800270AD4ED027A30EE270AF2EE047A80EE47
:1068C800270A0EF0BBFDBDEC048B83B21A0444BF4B
:1068D80000F5B47083B218B238BD00BF1C13002095
:1068E8000000E144DB0F494010B5447800780022ED
:1068F80002FB02F3193B634303F6C413534340F608
:10690800C411434393FBF1F3034921F812300132D8
:10691800072AEDD110BD00BF281300200430114B09
:1069280033F91000B0F5617F10B506DB40F633038C
:1069380098420246A8BF1A4601E04FF461720C78EB
:10694800192340F2833013FB0404944207DA497890
:1069580013FB01039342B4BF0020012010BD0020A7
:1069680010BD00BF7024002010B500F1500302785C
:106978008A4203D18478C278944204D3043098427E
:10698800F5D1002010BD012010BD1FB5084B1B68B4
:106998001B030AD58DF8040001230D2001A98DEDF4
:1069A800030A8DF8053001F0D3FD05B05DF804FB4E
:1069B800342400201FB5084B1B681B0309D58DF82C
:1069C8000400029100230D2001A98DF8053001F083
:1069D800BFFD05B05DF804FB3424002010B50A4A59
:1069E8000A4B11689B6800BF12689142F7D1084AA8
:1069F800D4694FF47A7000FB04F2D31AB3FBF4F3B2
:106A080000FB013010BD00BF5824002010E000E05A
:106A18001C13002038B50446FFF7E0FF0546FFF7D2
:106A2800DDFF401BA042FAD338BD10B504462CB197
:106A38004FF47A70FFF7EEFF013CF8E710BD024A09
:106A4800136801331360704758240020024B1B6AF7
:106A580003B11847704700BF1C130020014B1B6887
:106A6800184700BF382F002010B50020FFF7F6FFA9
:106A7800054B00241C700BF073FA044B83F8244078
:106A88009C629C851C6310BD202F00201C130020D5
:106A980010B510B9BDE81040E6E700230C225A43B0
:106AA8000A4C1119125D824203D00133102BF5D123
:106AB80010BD074B186B18B14A784078824203D250
:106AC800002219639A859A6210BD00BFB883010835
:106AD8001C13002010B540001428A8BF1420002360
:106AE800074A022199540B4499181424834201F847
:106AF800014CF5DBFF21D1540F20BDE81040C7E75A
:106B08000C24002038B5174B4FF4804240F2DB15B7
:106B18001A8568434FF400429A61851E0B24013C94
:106B280014F0FF0417D00F4A938A9BB283F4804372
:106B38009382938A9BB283F4004393822846FFF79B
:106B480074FF0120FFF78AFF1920FFF76EFF00206E
:106B5800FFF784FFE3E7044B044A1A60044B054A35
:106B6800DA6038BD00080048FC9F0020EFBEADDEAB
:106B780000ED00E00400FA0503681B691847036884
:106B8800DB68184703689B68184703685B68184701
:106B980003681B6818472DE9F84FB0F90230934293
:106BA80018BF00232DED028B18BF0370057804462B
:106BB8000E469146002D40F08B8007EE902A9FEDFF
:106BC800770AF8EEE77AB6EE008A27EE800ADFED5C
:106BD800747A20EE270AA04620EE080A0EF0A4FCDC
:106BE800DFED706A60EE266AB7EE006AB0EE667A8C
:106BF800A0EE007A40F2DC536365D0EE006A102301
:106C0800A4F8523037EE067A76EE866AC6EE077A30
:106C18001823A4F85030274684ED046A27EE807ABA
:106C280027EE007A77EE075A84ED017AC4ED025A0E
:106C380070EE005A84ED037AB8EE007AA5EE807AF9
:106C480027EE877A67EEA67A84ED057AC4ED067A90
:106C5800DFED557A98ED047A27EE277AF0EE678A09
:106C6800B5EEC07AF1EE10FA4CBF77EE487A77EEBF
:106C7800087A013517EE900A0BF0D0F9D8ED017AB1
:106C880067EEA87AC7E90E01F5EEC07AF1EE10FAC0
:106C98004CBF77EEC87A77EE887A08F1040817EEC9
:106CA800900A0BF0BBF9032DC7E9080107F10807A3
:106CB800CED1A6F2DC531B042367E3676367C4F8ED
:106CC8008030A367C4F884300123A4F802902370AD
:106CD800D4F85490B4F95280636A276A206FE26F3F
:106CE800D4F840C0D4F88010C4F88020C9EB060658
:106CF80006FA08F64FEAE67B734307FB0B33266771
:106D0800A7FB06671F44636C656F60674FEAE27B09
:106D180053430CFB0B3EACFB02237344B61A67EBE0
:106D28000307E36AA26AC4F884104FEAE07B43438E
:106D380002FB0B3EA2FB00237344B6185F41E36CD1
:106D4800A06CB4F95020A5674FEAE17B4B4300FBE8
:106D58000B33A0FB01011944636B361A206B4FEA11
:106D6800E57B05FB03F300FB0B3367EB0107A0FB97
:106D780005011944801979410BF026F908F1FF3211
:106D880001239340E067C01841EBE37142460BF0E2
:106D98001BF9BDEC028B4844BDE8F88F6F12833AAB
:106DA800DB0F4940F404B53F0000804B2DE9F84360
:106DB8000024234B93F86460E0B2B0420CD203EB9A
:106DC8008003204A5B6B32F810101BB10B2801D8E6
:106DD800DB6898470134ECE71B4B1B685B032DD538
:106DE80000242346E2B2B24228D2DFF8549009F1D7
:106DF80034074FEA840857F8242055689D4215D077
:106E0800284608F0E1FDEFF31283502282F312883E
:106E180028216A6A01FB00900132C0F88C206A6957
:106E280042F001026A61DBB283F3118857F8083037
:106E38001B6800221A6001342B46D3E7BDE8F883AB
:106E48001C130020941100203424002008B50E4B98
:106E58001B6813F4805F0D4B14BFD3F80821D3F8D7
:106E68000C2193F8641092880023D8B2884204D287
:106E7800074820F813200133F7E7FFF797FF322080
:106E8800BDE80840D1E500BF342400201C130020D1
:106E9800941100200A4B1A680A4B30B502F480524C
:106EA800D3F80841D3F80C5100230AB1A18800E0B7
:106EB800A988054820F8131001330C2BF5D130BDF3
:106EC800342400201C130020E223002070B5124D4A
:106ED8000024214605F21110702285F810410EF0A9
:106EE8009EF82146D5F884310B4A0B4493F90200E9
:106EF80080B102F211141E680E5108199C88848012
:106F08009B79837192F8103107310133702982F827
:106F18001031E7D170BD00BF1C130020094B1A685F
:106F28000E2303FB0020437AFF2B07D0064A127872
:106F38009A4203D9054A32F8130000E0808800B26B
:106F4800704700BFDC1700209C220020702400201E
:106F58002DE9F04F2DED048B944C954FD4F88C31DE
:106F6800DFF850828DB0064692489847914894F8C9
:106F78009C21014605F0B4F83B8804F5F672002B15
:106F880073D0D4F8A0311B7808EE103A04F5D27902
:106F980004F5D8754FF0000AB7F800B038F91A00B0
:106FA800BBF57A7F02BF0023C9F800302B61D9F8FE
:106FB80000300344C9F800302B6907EE900A01330A
:106FC800012B4FEA4A01F8EEE77A2B6106D100233C
:106FD800C5ED017AC5ED007AAB601BE0D5ED006A1E
:106FE80007EE103A37EEE66AB8EEC77A86EE077A09
:106FF80036EE877AD5ED026A85ED017A77EEC77AA3
:1070080085ED007AE6EE276AF0EE667AC5ED036A4A
:10701800C5ED026A0023BBF1010F28F80130535275
:107028002ED12B69012BC3BF03F1FF3300EE103AB9
:10703800D5ED037A9FED600AC8BFB8EEC00A8DE8A7
:107048000600C8BF87EE800A0EF09EFC9DE8060089
:1070580018EE103A5BB1F8EEC87AB4EEE70AF1EE32
:1070680010FA04DD4FF47A733B8000231CE0D9F852
:1070780000304FF47A7003F5FA7393FBF0F3535230
:107088000AF1010ABAF1030F09F1040905F114051F
:1070980082D1BBF1010F04D158460092FFF7F8FCEA
:1070A800009A3B88013BDFE738F8131032F81300E9
:1070B8003E4D091A28F813100133032BF4D13F4F22
:1070C8003B6813F0020300F0C9823D4B05F5F970E7
:1070D8005B6898473B4B05F5F9701A78014604F050
:1070E800FFFFB5F8F83105F5F979002B41D0D5F84F
:1070F800FC010023B4F8F821334939F913E02B4D8A
:10710800B2F5C87F04BF002241F823204FEA830C60
:1071180051F80C20724441F80C20002129F8131072
:1071280020F813100133032BE4D1B5F8F831012B03
:107138001AD1D5F800324FF4C87EC83393FBFEF35A
:107148000380D5F80422C83292FBFEF242801F4A1F
:10715800D5F808321288C83393FBFEF39B1A838054
:107168003180718003F058FBB4F8F831013BA4F882
:10717800F831174B1B68590740F18D80B4F80C2281
:107188000A4B322A26D1D3F8FC211188A3F80E1213
:1071980051889288A3F812223288A3F814227288A0
:1071A800A3F81012A3F8162216E000BF1C13002043
:1071B8004E2F002074110020000000005012002003
:1071C80000240020572F00201C1500200400002058
:1071D80034240020002A3DD0D4F8FCC10023B4F8A0
:1071E8000C22AA4939F91300A94D322A04BF0022FA
:1071F80041F823204FEA830E51F80E20024441F84B
:107208000E20002229F813202CF813200133032B19
:10721800E5D1B5F80C32012B17D10C2085F82422C2
:1072280085F82532FFF734FCD5F8FC31B5F80E2285
:107238001A80B5F810225A80B5F812229A80B5F84B
:1072480014323380B5F816327380B4F80C32013B2F
:10725800A4F80C3294F826328D4AE3B1D2F8FC51E6
:10726800D2F81802002182F826124FF0320E90FB55
:10727800FEF02880D2F81C0290FBFEF06880D2F85D
:107288002032844A93FBFEF312889B1AAB8031802C
:10729800718003F0C1FAD4F8FC21B4F8F2311188F6
:1072A8005B1AA4F8F2315188B4F8F4315B1AA4F8E7
:1072B800F4319288B4F8F6319B1AA4F8F631FFF746
:1072C8008DFBD4F8283294ED8B6AD4F83062C4F878
:1072D8002802C3EB000A07EE90AAB8EE678A0025D9
:1072E80028EE066A96F800C06B486C490DF10C0E42
:1072F8002A4638F9123007EE903AF8EEE77A67EE48
:10730800867AEEEC017ABCF1000F1CD007EE90CA29
:10731800F8EEE76AB7EE007AC7EE266A39F9123056
:1073280007EE903AF8EEE77A37EE667A67EEA67AD5
:10733800D1ED006AE6EE877AC1ED007AFDEEE77AD4
:1073480017EE903A01E039F81230438030F8023FE6
:107358000132032A13FB035501F10401C9D1DFF8F7
:1073680034814F4864236B43B8F800506D4393FB56
:10737800F5F5493D03A9ADB202F068FF3B2DD6ED06
:10738800016A11D9B4F94C32D4ED920A07EE903A59
:10739800F8EEE77A434BF4EEE70AF1EE10FA1EDD59
:1073A8001A7842F008021DE0F7EE007A36EEA77A66
:1073B8003B4A87EE877A00233B4931F913100133A2
:1073C800032B07EE901A92ED006AF8EEE77AE6EEE4
:1073D800267A67EE877AE2EC017AEDD1D2E71A785D
:1073E80022F0080294ED910A1A700EF029F9B0EE15
:1073F800409A84ED000A94ED920AD4ED917AD4ED86
:10740800908ADFED2A9A2A4D20EE000AF1EE688A6A
:10741800A7EEA70A0EF0B8FAF0EE400AB0EE680A36
:107428000EF00EF9F0EE408A84ED010A29EE290AE1
:107438000EF004F828EEA90A28800DF0FFFF3B683B
:1074480068801A073AD51B4803A902F0FFFED6ED5B
:10745800026A184AF7EE007A36EEA77A002387EE1A
:10746800877A154931F913100133032B07EE901A67
:1074780092ED006AF8EEE77AE6EE267A67EE877A0A
:10748800E2EC017AEDD10B4843E000BF341500204F
:107498001C130020040000201C120020501500209E
:1074A8005C150020541200201E1200204C3D0F4491
:1074B8002C2400206C1500207A1100206D4D03A9A2
:1074C800284602F0C3FE95ED010A95ED007AD5ED48
:1074D800027A20EE000AA7EE070AA7EEA70A0EF026
:1074E80053FAB5EE400AF1EE10FA11D0D5ED007A54
:1074F800C7EE807AC5ED007AD5ED017AC7EE807ABD
:10750800C5ED017AD5ED027A87EE800A85ED020A8B
:107518005848FFF78FF9584BDFED587A1880564BCB
:107528009FED577AB3F9003028EE278A07EE903A94
:10753800544BF8EEE77AB3F9002067EEC77AB1EE5C
:10754800499ACDED087A07EE902AB3F90220B3F9EB
:1075580004308DED069AF8EEE77AF1EE688ACDED03
:10756800097A07EE902AF8EEE77A09A8CDED0A7AAB
:1075780007EE903AF8EEE77A06A9CDED078ACDED49
:107588000B7A02F063FE73789DED0B7A012B19D10B
:107598003D4B1B785B070FD4D4F85C32402293FB39
:1075A800F2F29B1A07EE903AF8EEE77A77EE877ACE
:1075B800FDEEE77AC4ED977AD4F85C32402293FB6B
:1075C800F2F301E0B8F800309DED090A07EE903AB1
:1075D800F8EEE77A37EE677AD4ED987A8DED0B7A84
:1075E80094ED997A38EE077A88EE078A9DED0B7A42
:1075F80037EE677AE8EE077AB0EE678AC4ED987AD4
:107608000DF01CFFD4F86852297802F047FDD4F831
:107618006C329DED0A0A1844C4F86C020DF00EFF96
:10762800297802F03BFDD4F87032B0EE480A1844CD
:10763800C4F870020DF002FF697802F02FFDD4F84B
:107648007432124A18441368C4F87402534413601D
:10765800D4F878320133C4F8783205E0A5F8F2316D
:10766800A5F8F431A5F8F6310DB0BDEC048BBDE8F2
:10767800F08F00BF080000202C120020BD3786358F
:1076880035FA8E3C1E120020562F0020342F002081
:10769800F8B504460E4617460025204620210DF071
:1076A800F4FC0446D0B1013420460DF053FDB0F58A
:1076B800617F05DB40F634039842A8BF184601E015
:1076C8004FF46170A0F56170192390FBF3F00DB9C8
:1076D800307000E070703B7801333B700DB90125C4
:1076E800DBE72046F8BD30B505460C46134629466B
:1076F80022460248BDE8304002F0B1BC9899010822
:107708007FB504780646E4B9354B1B6803EB840360
:10771800192193F87B0093F87C6093F8792093F80B
:107728007A304FF4617511FB005011FB065100903F
:1077380001912C482146013402F091FC142CE3D12C
:107748004BE00DF007FD1328054641DC244B701C67
:107758001C68202100238DF80F300DF096FC1E3593
:10776800064670B1013630460DF0F4FC19289FBF6B
:1077780004EB850358709DF80F30013398BF8DF8DE
:107788000F30304620210DF080FC064670B10136DE
:1077980030460DF0DFFC0D289FBF04EB8503987081
:1077A8009DF80F30013398BF8DF80F3004EB850436
:1077B8003046E11C0DF10F02FFF76AFF9DF80F300C
:1077C800042B0AD0601C002104220DF028FC04E0E0
:1077D800054800211322FFF786FF04B070BD00BFE3
:1077E80090110020B7990108CC990108014808F0C8
:1077F80067BB00BFD2990108F8B50478064674B98A
:10780800304DB5F8C621B5F8C8312F4821460134A6
:1078180002F025FC042C05F10405F2D1F8BD2B4932
:107828000DF006FCA8B9274B4FF47A714FF4FA62B1
:10783800A3F8C611A3F8C821A3F8CA11A3F8CC214C
:10784800A3F8CE11A3F8D021A3F8D211A3F8D4211C
:10785800F8BD30460DF07EFC032805462BD830468F
:1078680020210DF012FC044630B1013420460DF001
:1078780071FC0126074600E00646204620210DF04F
:1078880004FC10B9BDE8F840B0E701300DF062FC27
:10789800012EF7D1A7F2EE2240F2DC539A42F1D83A
:1078A800A0F2EE229A42EDD8064B703503EB850321
:1078B800DF801881F8BD064800210322BDE8F840A2
:1078C80011E700BF94240020E0990108F39901080A
:1078D8004FA501082DE9FF4104780546002C39D150
:1078E8007348744D08F0ECFAD5ED057AF5EE407A58
:1078F800F1EE10FA00F0D88021466F4802F0AFFB95
:1079080095ED050A684602F03FFA01466B4802F019
:10791800A6FB95ED060A684602F036FA0146674866
:1079280002F09DFB95ED070A684602F02DFA014624
:10793800624802F094FB95ED080A684602F024FAC2
:10794800013401465E4802F08AFB0C2C05F1100553
:10795800CAD1A9E05B4905220DF0AEFB40B9554BF1
:1079680003F1C0020021596110339342FAD19BE020
:107978002846554904220DF09FFB04462846002C52
:1079880040D120210DF081FB002800F08D80451C9E
:1079980028460DF088FB07464C4B53F824601EB967
:1079A8004B4808F08DFA7FE028463146FAB20DF0D0
:1079B80083FB01340028EFD13E4B03F1C0029E4601
:1079C8000021596110339342FAD1424B03EBC402B0
:1079D8009846D2F804C0BCF1000F04D131463E48A5
:1079E80002F03DFB57E0002718F834309F42F5DAE3
:1079F8003B010EEB030563440FCB143585E80F00FC
:107A08000137F1E70DF0A6FB0B28064647DC2846B0
:107A180020210DF03AFB054650B10135284602F009
:107A280029F9244B03EB061383ED050A012400E032
:107A38000446284620210DF028FB054648B10135AB
:107A4800284602F017F91B4B03EB061383ED060AD1
:107A58000134284620210DF018FB054648B10135B0
:107A6800284602F007F9134B03EB061383ED070AC8
:107A78000134284620210DF008FB10B9FFF7B6FEA7
:107A880012E0013002F0F6F80A4B032C03EB06165D
:107A980086ED080AF2D11148FFF71CFF04E01048F0
:107AA80001210C22FFF71FFE04B0BDE8F08100BFE2
:107AB800F999010894240020149A01081A9A0108D7
:107AC80063A20108F39901081E9A0108EC910108C4
:107AD800239A0108C8980108329A01089297010868
:107AE800CC990108F0B5047887B006461CBB514B09
:107AF8001968062303FB0411192091F8CA5091F85C
:107B0800CB7091F8CE2091F8C9304FF4617610FB14
:107B1800056510FB07600095019091F8CC00029074
:107B2800C8314548497903912146013402F097FA52
:107B38000C2CDCD17CE00DF00DFB0B28044672DC2C
:107B48003C4B701C1D68202100238DF817300DF068
:107B58009CFA064680B1013630460DF0FBFA032840
:107B68009FBF062303FB045383F8CE009DF817300C
:107B78009CBF01338DF81730304620210DF085FA6F
:107B8800074680B1013738460DF0E4FA0D289FBF4B
:107B9800062303FB045383F8C9009DF817309CBFE4
:107BA80001338DF8173006266643A9193846CA31BD
:107BB8000DF11702FFF76CFD20210DF066FA07465C
:107BC80070B1013738460DF0C5FA14289FBF9DF8EB
:107BD80017307619013386F8CC0098BF8DF8173026
:107BE800384620210DF051FA78B101300DF0B2FA83
:107BF8000D289FBF062303FB045383F8CD009DF88F
:107C080017309CBF01338DF817309DF81730062BBD
:107C18000ED0062202FB04500021C9300DF0FFF9F6
:107C2800FFF7E4FD04E0054800210B22FFF75BFDA8
:107C380007B0F0BD901100203E9A0108CC990108C8
:107C48002DE9F341047880464CB9204601A907F094
:107C580041FB0134FFF7F4FF122CF6D169E00DF077
:107C680079FAC6B2112E5FD8334C06F1D00704EB6F
:107C7800470308F1010020219D780DF006FA18B994
:107C8800AA1E5542554139E04378682B06D0732B1C
:107C980007D0612B13D14FF0000804E04FF0010822
:107CA80001E04FF00208A8F102035D4200F1010073
:107CB8004FF020015D410DF0E8F9D8B115B9FFF793
:107CC80095FD36E001300DF045FA40F2ED2380B223
:107CD800984205DD40F6CA039842A8BF184601E05D
:107CE80040F2EE2004EB4703A0F2EE20192290FBAD
:107CF800F2F0D87004EB470383F8028004EB4704E2
:107D08000E4AA378D25C55B1E3780D4840F2EE24D0
:107D18001925314605FB034302F0A1F909E0314674
:107D2800084802F09CF904E0074800211122FFF7F7
:107D3800DAFC02B0BDE8F08194240020CC79010877
:107D48005E9A0108709A01084FA5010810B504460B
:107D58002046FEF711FF18B90A20FEF766FEF7E77E
:107D680010BD002207490C2303FB02135968814206
:107D780004D10022C2621A725A6070470132042A82
:107D8800F0D17047A82200202DE9F04F87B088462F
:107D98009DF8444011461A469DF84030814600251A
:107DA8000C206843814E87198057484505D197F8BC
:107DB80008A0BAF1000F04D0F3E00135042DEFD18B
:107DC800EFE0B9F1010F00F0DA8006DCB9F1000F3D
:107DD80040F0E78000947648D6E0B9F1020F00F051
:107DE800D180B9F1140F40F0DC80724FBB6943F0C9
:107DF8000103BB617B694FF0904443F400337B611E
:107E0800012603224FF4805B04A94FF090408DF8BF
:107E180015200392CDF810B08DF814608DF8166017
:107E28008DF817A004F020F9A4F828B0C820FEF7B0
:107E3800FCFDC4F818B07B69039A43F400337B61F6
:107E480020464FF4C0534FF0020B04A904938DF859
:107E580015208DF814B08DF816A08DF817A004F031
:107E680003F9636A23F470436362636A43F460430B
:107E78006362636A23F470236362636A43F4602372
:107E880063624D4B4D4C4FF480221A6002F18042E0
:107E9800A2F53F3212232363082384F83530136890
:107EA80084F8366023F480231360536823F4802316
:107EB800536094F8343003F1804303F582331A6831
:107EC80042F480221A60226B3D4B22F01F0002F020
:107ED8001F02C15806FA02F221EA0202C250226BBE
:107EE800384922F01F0002F01F0250F801E006FA9C
:107EF80002F22EEA02024250226B22F01F0102F027
:107F08001F02C85806FA02F20243CA502E4B2F4AE3
:107F1800C3F800A0FB6943F40003FB612C4B04A8E1
:107F2800DA608DF810908DF811B08DF812A08DF8E8
:107F3800136008F0ABFD2A238DF810309DF813303C
:107F48008DF811608DF812A01BB104A808F09EFDF1
:107F580004E0204B4FF48062C3F884201E4A1F4B74
:107F6800136002221A721E4A1E4B13601E4A1F49D2
:107F78001B68116098471E4B2360104807E0009467
:107F88001C4801E01C48009405F094FC48B1074BDC
:107F980080F804900C2202FB053585F8088068609B
:107FA80000E0002007B0BDE8F08F00BFA822002045
:107FB80000380140001002401404014098150020C8
:107FC800080401400C040140D80042420005FA05AB
:107FD80000ED00E000E100E094210020982100205D
:107FE800BC200020B4000020B8200020140000208D
:107FF800D0790108004400400048004010B5084B03
:108008001968002201EBC20393F90240844201D1AE
:10801800981C10BD0132042AF4D1002010BD00BF05
:10802800A4220020F0B5027887B08AB94A4C04F13E
:10803800200694F8F22100234849595650B281424B
:108048006ED00C33302BF7D10834B442F1D181E033
:10805800002204920592451C0DF07CF8C4B260B26F
:10806800FFF7CCFF074618B18DF81040012400E057
:108078000446284620210DF008F8054638B1013598
:1080880028460DF067F80134ADF81200E4B2002676
:10809800284620210CF0F9FFB0B3451C28460DF006
:1080A80059F800222E4951F8223083425FFA82FEA5
:1080B80004D00132082AF5D1002300E0734651F8B4
:1080C8002320824220D1022E0FD0032E12D05A1E16
:1080D800012ED2B204D0042A13D88DF814300EE041
:1080E800042A0ED88DF8153009E0052B09D88DF82B
:1080F800173004E09A1E052A03D88DF8163001348B
:10810800E4B20136042EC3D1052C04D807B0BDE86B
:10811800F040FFF76BBB04AB03CB3860796019E024
:1081280094F8F7010E4B94F8F65153F82000B4F880
:10813800F421009094F8F90153F82000019094F884
:10814800F80153F82000029053F82530054801F053
:1081580086FF79E707B0F0BD94240020A82200200C
:10816800F88201087F9A010838B1438811EA0300B0
:1081780003D08B420CBF01200220704730B50B4B57
:108188000B491C6891F83820032A0BD8134604EBD6
:10819800C303551CEAB29D882842F5D081F83820DF
:1081A800981C30BD81F83820002030BDA422002062
:1081B80098150020024B002283F83820DEE700BF24
:1081C800981500202DE9F047877890F803C0214DD5
:1081D800BBB2C7F1640E03EB83065C42C3F17800BF
:1081E8005FFA8EFE7600CCF16408A4B280B2A3B226
:1081F8000FFA83F9B9F1000F05DC002B14BFBA465A
:108208004FF0010A00E0F24613FB03F303FB0CF204
:108218001AFB0AF392FBF3F3434403FB09F30A2224
:1082280093FBF2F333449BB225F8023FB1F8009078
:108238004A880A34C9EB020AA4B21AB202FB0AF24B
:108248004FF47A73844292FBF3F34B442B80CED1E4
:10825800BDE8F087D01500202E4B2F4A1B68126806
:1082680010B51A602D4A1168596051689268DA6031
:108278002B4A996011681961516892689A61294A74
:1082880059611168D961516892685A62264A19621F
:1082980011881985518859859188D288DA85234AA9
:1082A8009985118819865188598692889A86204A14
:1082B8001188D986518819871946928821F83A2F4A
:1082C8001C4A10780022824206DA1B4C34F812400D
:1082D80021F8024F0132F6E7184A1288A3F8642001
:1082E800174A1288A3F86620164A1188A3F86C105A
:1082F80051889288A3F87020134AA3F86E10126868
:108308009A66124A1288A3F87220114A5289A3F871
:108318005E2010BD942C0020302F0020181A002059
:10832800241A0020301A0020341200207411002072
:108338001E12002080130020941100201C19002018
:108348002C1000207A11002028120020B0110020E3
:10835800801100202DE9F8430E4B93E88003054671
:108368000E460024B44213DA7B1933F9140008EBE3
:10837800050333F9142009EB050333F914301344CA
:10838800022293FBF2F3C01A08F051FB0134E9E72B
:10839800BDE8F883942C002070B5472008F096FAC1
:1083A800174B1B681B0307D5164B174A5B681068E9
:1083B8001B68C01A08F02CFB144E154C154D30786C
:1083C80008F026FB23682868C01A08F030FB6368A9
:1083D8006868C01A08F02BFB0F4B188808F018FBC8
:1083E8000E4B188808F014FB0D4B188808F010FB8A
:1083F800337823742B68A3606B68E36070BD00BF9B
:10840800002E0020942C0020302F00205A1200202B
:10841800802C00205C1200205812002056120020E8
:10842800B81100207FB5254C254E264D2649274AF0
:10843800274B20B127480088B0F5805F30D23088BC
:10844800ADF8040028781D4D897912788DF806005A
:108458008DF807108DF808201B788DF8093001A8D1
:10846800294606220CF0C0FD28B30198BDF8083053
:108478002860AB80532008F029FA208808F0C8FA51
:10848800A07808F0C5FAE37801932379029301A84C
:108498006379039308F022FA0E4B00221A800AE04F
:1084A800308820808979287812781B78A070E1704C
:1084B80022716371DEE704B070BD00BFEC150020C7
:1084C80018130020541200207C0E0020AB0E002050
:1084D800100F0020202E0020A0F17D03012B70B585
:1084E80004460D460A4E05D830687D21FEF750FB3C
:1084F80084F0200430682146FEF74AFB35B12B880A
:108508001C4404EB142404F0FF042C8070BD00BF4D
:10851800081300200A4A138801331380094A136894
:1085280001331360084A138801339BB2202B01BF23
:1085380000231380054A138808BF0133138070474E
:10854800202E0020082E00200C2E00200E2E0020A9
:1085580038B53A4B1B78083B012B05460C466BD8BF
:10856800452008F0B3F9284608F0B0F90C2D23D0BF
:1085780004D80A2D0AD014D835B138BD0E2D4BD0E9
:108588002ED3FF2D50D038BD206849E0207808F060
:108598009DF962796378002A14BF8020002018436F
:1085A80000E0207808F092F9A07808F08FF9E078D8
:1085B80008F08CF920793BE0B4F9000008F01EFAC5
:1085C800A07808F083F9E07808F080F9B4F904009D
:1085D80008F014FAB4F90600BDE8384008F00EBAFD
:1085E800637820788BB180F0800008F06FF9A46878
:1085F800E0B208F06BF9C4F3072008F067F9C4F398
:10860800074008F063F9200E12E008F05FF960688F
:10861800BDE8384008F00BBA206808F0F9F960683E
:10862800BDE8384008F0F4B9054808F02DF90020F5
:10863800BDE8384008F04AB938BD00BF702C0020AA
:108648009E9A01082DE9F04FB74BB84F1A888BB0A6
:108658000193002A40F0A380B7F8D207B44E42F243
:108668000103C21A50425041FFF7DCFEFFF7F4FD48
:108678003468492008F02AF9AE4B2546186808F0F6
:10868800C7F955F8040B08F0C3F9284606F078FD39
:1086980004F1100006F074FD04F11C094FF01008F5
:1086A800A54D01232A6803FA08F3134203D0D9F829
:1086B800000008F0BCF908F10108B8F1130F09F13E
:1086C8000409EDD104F1280006F04AFDB7F8443159
:1086D800B4F92E00C01A08F09BF92B68DB0408D502
:1086E800964BB4F864001B88181AC0F30D0008F004
:1086F8008FF92B68980403D5B4F8660008F088F958
:108708002B68590503D504F16C0006F029FD2B6888
:108718001A0502D5A06E08F08AF92B681B0403D548
:10872800B4F8720008F074F904F13000A04606F0BD
:1087380017FD04F1360006F013FDB7F8443138F997
:108748003C0FC01A08F064F901277D4B1B789F4243
:1087580008DA38F9020FB4F93C30C01A08F067F9A2
:108768000137F2E72B68980505D5B4F95E00A0F249
:10877800DC5008F05CF9326872487260B260121A14
:108788009110714A4A43531C032293FBF2F202EB05
:1087980042029A1A742303FB02033360C9E16B4B4C
:1087A8006B4A1B6811688B4206D00AA9002041F861
:1087B800203D1360FFF7CCFE019B97F8D2171B886A
:1087C80097F8D3070B44013BB3FBF0F200FB1233DD
:1087D8008B4280F07981564C0120FFF723FEFFF78A
:1087E8003BFD50202668656808F070F8A268236889
:1087F80010681B68626803441068A3EB400008F027
:1088080016F96A6873689B1A0293AA68B3689B1A78
:108818000393EA68F36802A89B1A049306F0B0FC75
:108828002A6933699B1A02936A6973699B1A0393CD
:10883800B369AA6902A89B1A049308F04FF806F1D5
:108848001C0905F11C0B1027A0463B4801210368B1
:10885800B9401942824606D0D9F80000DBF800304A
:10886800C01A08F0E4F80137132F09F104090BF1D5
:10887800040BEAD106F1260005F12601002331F99F
:10888800024F30F9022F121B02AC44F823200133A7
:10889800042BF4D10322002702ABBF0053F8223087
:1088A800FFB26BB103F108010F2902D847F00107A5
:1088B80006E08033FF2B94BF47F0020747F0030719
:1088C80012F1FF32E8D2384608F000F800240DF122
:1088D8000809A34607F00302022A10D0032A17D07A
:1088E800012A4AD1BBF1000F41D0D9F8000000F0AD
:1088F8000F00204307F0EAFF4FF0000B3DE0BBF10B
:10890800000F0CD0D9F80000C0F3031020432CE06E
:10891800BBF1000F1ED199F8010007F0D7FF99F8B5
:10892800000007F0D3FF28E00C2E0020942400203C
:10893800942C0020082E0020002E0020FC2D002062
:1089480080130020A02C002035C2724F142E002066
:10895800102E0020D9F80000C0F30330204307F0A0
:10896800B5FFD9F80000C0F3071007F0AFFFD9F83A
:1089780000402401E4B24FF0010B09F1040906ABF1
:1089880099454FEA9707A5D1BBF1010F02D12046BF
:1089980007F09CFFDAF8003013F480541FBFB6F8D4
:1089A8006420B5F86410521A029218BF0124990481
:1089B8000AD50AAA02EB8401B5F86600B6F8662063
:1089C800121A41F8202C01345A0513D502AA02EBD9
:1089D800840E06F16A0705F16A00002237F9021FC2
:1089E80030F902CFCCEB01014EF822100132032AF4
:1089F800F4D103341F0508D50AAA02EB8400A96E36
:108A0800B26E521A40F8202C013418040BD50AAB68
:108A180003EB8402B5F87210B6F872305B1A42F8AC
:108A2800203C013400E0F4B1012C03D1029807F096
:108A3800FEFF18E0631E002002AA400052F823201F
:108A4800C0B20AB140F0010013F1FF33F4D207F0CD
:108A58003DFF002702AB53F8270008B107F0E7FFF6
:108A68000137A742F6DB30200321FFF773FC3620DD
:108A78000321FFF76FFC314B3C201978FFF76AFCA4
:108A8800DAF80030990506D5B6F95E00B5F95E301A
:108A9800C01A07F0CCFFD8F800202948D8F80430CD
:108AA800C8F80420121A9110264AC8F808304A4318
:108AB800531C032293FBF2F202EB42029A1A74232C
:108AC80003FB0203C8F800301F4B1B681A0630D599
:108AD8001E4C1F4D22682B689A420BD162686B6846
:108AE8009A4207D1019B1B88102B11D1194B1B8867
:108AF8005B060DD1482007F0E9FE206807F097FFD4
:108B0800606807F094FF23682B6063686B600EE071
:108B1800114A0F4B11782A7C914208D10F4A996863
:108B28001068884203D15268DB689A4201D0FFF787
:108B380033FC07F09BFE0BB0BDE8F08F80130020DC
:108B4800A02C002035C2724F34240020BC11002014
:108B5800802C00200E2E00205A1200205C120020CB
:108B68002DE9F84F0C9E3A4CC2EB030B0B9BF61AFF
:108B78006368002914BF4FF0060A4FF0040A013356
:108B88000546904613D1236853455ED2314A324890
:108B980052F82320032B98BF294607F085FE636807
:108BA800013363602D4B002205469A7113E00025BE
:108BB80011E02B4A1278954240DA0B9BE3B109FB8E
:108BC80006F2995C01228A40264909680A4213D1B3
:108BD800636801336360D4F804900A9B1C4F99457D
:108BE800E7DB2BD10A2007F071FE3B6801333B60BD
:108BF8004FF0FF337B6021E0184A917921B12C2096
:108C080007F064FE013501E001219171226809FB3A
:108C18000BF308EB030752B958F8030007F034FECA
:108C280097F904104B1C0544D2D00F4802E03A448F
:108C38000E48117907F038FE0544C9E72068504509
:108C48002CBF00200120BDE8F88F0020BDE8F88F78
:108C5800182E0020A87E0108A99A0108EC1500200A
:108C680014010020002E0020B89A01087BA20108F8
:108C780030B585B004AC002524F8025D0091ADF84C
:108C8800060021461020FFF727FC9DF80600214624
:108C9800FFF722FC9DF807002146FFF71DFC9DF811
:108CA80000002146FFF718FC9DF801002146FFF758
:108CB80013FC9DF802002146FFF70EFC9DF8030007
:108CC8002146FFF709FC9DF80E00C043C0B22946B3
:108CD800FFF702FC05B030BD10B5054C2068FDF764
:108CE80054FF18B12068FDF74DFFF6E710BD00BF2F
:108CF800D812002013B5044601A9006808F000FF47
:108D0800132008F039FFBDF9040008F023FF1B20E9
:108D180008F032FFBDF9060008F01CFF232008F018
:108D28002BFF2368002BB4BF53204E2008F012FFFE
:108D380001A9606808F0E4FE122008F01DFFBDF9E3
:108D4800040008F007FF1A2008F016FFBDF9060016
:108D580008F000FF222008F00FFF6368002BB4BF63
:108D68005720452008F0F6FE02B010BD82B01B4B1C
:108D78001B4A8DF807101968106860B31268052A35
:108D880029D1184A106810BB9DF808109DF80730C3
:108D980043EA012314490B80144B1968144B89B218
:108DA8000B445B0019680121196013680B441360B8
:108DB800104A136823F4E04323F040039BB283F086
:108DC800300343F4004343F08003136003E01A6860
:108DD800521A312AD5D902B0704700BF5824002052
:108DE8003C2F0020F821002080610040505C0040AA
:108DF8000A300020045C0040014B1868C0B270477C
:108E0800B4210020012070477047704707EE900A90
:108E1800F8EEE77ADFED0C6A9FED0C0AF5EEC07A02
:108E2800F1EE10FAD4BFB1EE677AC7EEA67A08B5AC
:108E3800D8BFC7EE267A27EE800A01F0A1F9044BC5
:108E480083ED000A08BD00BF8096184B35FA8E3CAA
:108E580078000020F7B51C4B1A680AB91C6800E0B6
:108E680001241A490E780022D0B2A04202F1010270
:108E780007D202AD2F18164D3544285C07F8040CAC
:108E8800F2E71A68121B1A600A781D6822440A70F1
:108E98009DB90320402102F0CFFD0E4A136823F448
:108EA800804323F070039BB283F4405343F40043A0
:108EB80043F080031360054B1D70002CCBD09DF848
:108EC800040003B0F0BD00BFB4210020F415002059
:108ED800B82100200C5C004013B5062204466B46FE
:108EE80003211E20FBF7ECFE9DF800209DF80130C1
:108EF8009DF8021043EA02231BB21B4A07EE903A80
:108F080092ED007AF8EEE77A67EE877A92ED027AC8
:108F1800FDEEE77A17EE903A23809DF8033043EA96
:108F280001231BB207EE903AF8EEE77A9DF8041099
:108F380067EE877A92ED017AFDEEE77A17EE903ABE
:108F4800A3809DF8053043EA01231BB207EE903A4F
:108F5800F8EEE77A67EE877AFDEEE77A17EE903A51
:108F6800638002B010BD00BF380000201FB5044662
:108F780002210C2001220DF10703FBF7A1FEC8B363
:108F88009DF80730DB0735D50321062202AB0C20FC
:108F9800FBF796FE0C20092101220DF10703FBF7D0
:108FA8008FFE38B39DF8073013F00C0F22D19DF8CF
:108FB80009209DF8083043EA0223C3EB83339B0062
:108FC8009DF80B2023809DF80A3043EA0223C3EB67
:108FD80083339B009DF80D2063809DF80C3043EA95
:108FE8000223C3EB83339B00A3800C200A210122B8
:108FF800FBF7E2FE04B010BD07B50A2100220C20E1
:10900800FBF7DAFE1420FDF710FD0A210F220C20D1
:10901800FBF7D2FE0A20FDF708FD01AB1021032261
:109028000C20FBF74DFE0A20FDF7FFFC0A21002269
:109038000C20FBF7C1FE0A20FDF7F7FC0DF1030336
:10904800022101220C20FBF73BFE0DF1030309214D
:1090580001220C20FBF734FE0A2101220C20FBF729
:10906800ABFE03B05DF804FB2DE9FF41634B1B68C1
:1090780093B11A681AB16249486902434A619A88E9
:10908800ADF8042002228DF807209868002201A973
:109098008DF80620FBF7FEFC3220FDF7C6FC002108
:1090A80011221E20FBF788FE012160221E20FBF7FB
:1090B80083FE6420FDF7B9FC02A8FFF70DFF00242A
:1090C8000A2726462546022101221E20FBF774FEA8
:1090D8003220FDF7AAFC02A8FFF7FEFEBDF9082022
:1090E800BDF90A10BDF90C308A421444A8BF0A46DB
:1090F80093421D44A8BF134613F5805F0E440ADD52
:10910800404A938A9BB283F48043013F9382DAD129
:109118004FF0010801E04FF000081E200021122244
:10912800FBF74AFE0A27022101221E20FBF744FE14
:109138003220FDF77AFC02A8FFF7CEFEBDF9082021
:10914800BDF90A10BDF90C308A42A4EB0204A8BF8D
:109158000A469342A5EB0305A8BF134613F5805FA3
:10916800A6EB010608DD274A938A9BB283F4804365
:10917800013F9382D7D101E04FF0000807EE904AF3
:109188009FED217A214FF8EEE77A0021C7EE277A82
:1091980070221E20F0EEE77AC7ED007A07EE906A9B
:1091A800F8EEE77AC7EE277A9FED197AF0EEE77ABC
:1091B800C7ED017A07EE905AF8EEE77AC7EE277AFC
:1091C800F0EEE77AC7ED027AFBF7F6FD01212022DF
:1091D8001E20FBF7F1FD1E2002210022FBF7ECFD0B
:1091E8006420FDF722FCB8F1000F04D14FF07E5344
:1091F8003B607B60BB6004B0BDE8F0810C030020DD
:10920800001002400008004800406F463800002067
:1092180001C05E46F8B59B4B1B680546187818B127
:10922800012800F06581DCE2242D974C0CD006D88B
:109238000A2D00F0D8800D2D00F0D58042E12A2DAE
:1092480006D02C2D04D03DE16070A070E0704BE199
:109258008E4BA17867788C4A002058542FBB197818
:109268001771472921D1597850291ED19978472952
:1092780007D1D978472904D11979412901D1012188
:1092880011719978814A522903D1D1784D2900F07A
:10929800AA8299787D4A472907D1D178532904D1E0
:1092A8001279562A04BF032222712279764E022AA5
:1092B80038D0032A4BD0012A40F08380BA1E072AEF
:1092C8007FD8DFE802F004080F131A257E2A07F07A
:1092D800B5FDA06075E01B78532B72D1A3685B4283
:1092E800A3606EE007F0AAFDE0606AE01B78572BE8
:1092F80067D1E3685B42E36063E01B78302B644B23
:109308001A788CBF42F0020222F002021A7058E06A
:10931800002007F0F3FD207453E0002007F0EEFD75
:1093280060824EE0072F06D0082F4AD1012007F0AF
:10933800E5FDF08245E0012007F0E0FD41F2184329
:1093480058434FF47A73B0FBF3F0B08239E0022F40
:1093580007D0032F0AD1002007F0D0FD4D4B18701D
:109368002FE0002007F0CAFD30762AE029D93A1FFD
:109378009210337E0132D2B2013B02EB8303DBB29F
:10938800102B1ED8F91EC2F1010201EB8202D2B2E3
:10939800012A0BD0042A11D100205E1E07F0AEFD71
:1093A8003D4B98553D4B00229A5507E05E1E3C4ABE
:1093B8000020935507F0A2FD3A4B9855E369013315
:1093C800E361314B2A2D18BFDA7807F101074FF016
:1093D80000000CBF012255406770A0700CBF83F8D5
:1093E8002020DD7080E094F82000002846D02E4B25
:1093F80013F8012D2D495A708B42F9D1234A224D79
:1094080013785278402B85BF373B1B011B01DBB219
:1094180098BF03F0F003402A8CBF373A303AD2B2F3
:109428001344E278DBB29A4225D121230B702879C4
:109438006B6A1E4A013301286B620AD002281CD1CC
:10944800722313701A4BAA8A1A801A4BEA8A1A8056
:1094580013E0672313700E4B1B789F070ED5164B2E
:10946800AA681A60EA685A60144B2A7C1A70144B6E
:109478006A8A1A8002E03F230B700020002384F8D8
:10948800203031E008080020F41500206024002076
:1094980054120020D011002001120020F1110020E8
:1094A800D1110020E11100202C0300201803002016
:1094B80056120020B81100205C1200205A12002019
:1094C80058120020A37894F820000E2B9FBFAA4AB8
:1094D800591C9170A94A98BFD554A74A18B9D3788E
:1094E8005D40D57000E00020003018BF0120F8BDB5
:1094F800A14B93F828100022082900F27281DFE8B6
:1095080001F0050C101A2B3B5F7B8800B52D40F04D
:10951800688183F8292001224FE0622D08BF0222CA
:109528004BE0032283F8282083F82A5083F82B5035
:1095380083F82C5055E1042283F8282093F82B2037
:1095480093F82C1083F82D502A44D2B283F82B209C
:109558000A4483F82C2044E1052283F8282093F854
:109568002B2093F82C10DD852A44D2B283F82B20C7
:109578000A4483F82C2034E1062283F8282093F843
:109588002B2093F82C102A44D2B283F82B200A44BB
:1095980083F82C20DA8D02EB0525ADB2B5F5AC7F4A
:1095A80088BF754ADD8584BF012182F82910002211
:1095B8001A86002D40F01581072283F8282010E133
:1095C80093F82B2093F82C102A44D2B283F82B203E
:1095D8000A4483F82C201A8EB2F5AC7F3CBF66494A
:1095E800891802F1010238BF81F83450D98D92B23E
:1095F80091421A86E0D9F4E0082283F8282093F8EB
:109608002B30AB4200F0ED805B4B012283F8292020
:109618000FE05B4C83F8282014F8012D6270594A3A
:109628009442F9D193F82C10534AA94206D03F230B
:109638002370554A536801335360D2E0516A92F857
:1096480029000131516210B13E232370C9E0212164
:10965800217092F82D10062941D004D8022907D08C
:10966800032923D0F8BD122959D0302967D0F8BD75
:10967800502121704549946B4C60D46B0C60516C3F
:109688004FF47A7491FBF4F1414C218092F88C11DB
:10969800404A19B1117841F0020102E0117821F035
:1096A80002011170012283F88D218CE05321217071
:1096B80092F83910CE0705D592F83820D51E6A429F
:1096C8006A4100E0024602F0010183F88C11002A89
:1096D80079D130490A7822F002020A7073E04F21EA
:1096E800217092F83F10CC0705D592F83E20D11E84
:1096F8004A424A4100E0024602F0010183F88C1117
:1097080022B924490A7822F002020A70224A93F800
:1097180063101170214AB3F86010118053E056218C
:1097280021701F49946C0C8042F21074D16C91FB2B
:10973800F4F11C4C2180012182F88E1143E049216B
:10974800217092F83810184A102988BF102111701A
:10975800164914780022A24232D2154D0E7A565577
:10976800144D4E7A5655144DCE7A5655134D11F860
:109778000C6F56550132EEE7F415002060240020E6
:109788002C03002018030020E80700205C120020AA
:1097980058120020541200205A1200200A010020FA
:1097A80056120020B8110020D011002028160020E1
:1097B800D1110020E1110020F11100200112002038
:1097C800DA690132DA6193F88D310B4A93B192F874
:1097D8008E317BB1002182F88D1182F88E111846E6
:1097E800F8BD0020F8BD1279432A7FF452AD022259
:1097F80022714EE5F8BD00BFF41500200449054B61
:109808000968187000225A6199611A77704700BF79
:1098180058240020E807002010B5121A07EE902AF5
:109828005B1A2DED028BF8EEE78A07EE903A184B9B
:10983800059CB8EEE78AD3ED007A28EE278A28EE51
:10984800080AA8EEA80A0CF09FF8DFED127A049B2C
:1098580020EE270AF0EE480ABCEEC00A83ED000AA3
:10986800B1EE680A0BF0ECFEDFED0B7A9FED0B7A98
:10987800E0EE077ABDEC028BFDEEE77A17EE903A40
:10988800002BBCBF03F50C43A033236010BD00BF01
:10989800780000202C7D8E3F00A00C46A00CB3451C
:1098A80044F25063984203DDA0F50C40A03870479D
:1098B800034B9842BCBF00F50C40A030704700BF76
:1098C800B0B9FFFF73B51A4C036823600B68636077
:1098D800184D0068184EFFF799FA184B009395E851
:1098E800030094E80C000196FFF796FF144B3268CA
:1098F8001A606868636813491B1A07EE903A124B9E
:10990800286893ED007A23681B1A0B600F4BF8EE5A
:10991800E77A1A600E4B67EE877A1B68FDEEE77AE6
:10992800DA880C4BC1ED017A1A8002B070BD00BF15
:10993800342100205C120020402100203C2100201E
:109948007C21002044210020780000207421002080
:10995800800F0020702100204279DFED2A5A2A4B1F
:109968009FED2A5A07EE902AF8EE677AC27BC7EE77
:10997800A57AB2EE047AC3ED007A07EE902AF8EEE3
:10998800677A234ADA60C7EEA57AC3ED017A81794E
:10999800204B07EE901AF8EE677A017CDA60C7EE82
:1099A800877AC3ED007A07EE901A817E06EE101AC8
:1099B800F8EE677AB8EE466AC7EEA57A86EE056ACB
:1099C800C3ED017A83ED026AC179134B06EE901A52
:1099D800417CDA60F8EE666AC6EE876A07EE101A0E
:1099E800C17EC3ED006A07EE901AB8EE477AF8EE2A
:1099F800677A87EE257AC7EE857A83ED017AC3ED1B
:109A0800027A70470000C8424C21002000007A44C6
:109A18000000FA445C2100208021002010B50C4C85
:109A280023789B0713D50B4B1B78042B0FD90A4AB5
:109A38000A4B106852685A601860FFF7E7F9084B3C
:109A48001A88084B1A80237843F00103237010BD4D
:109A5800541200205A1200205C120020BC11002071
:109A68002C120020902100201C4B1B681B0307B5FB
:109A780030D51B4A1B4BD2ED007A1B788DF800308D
:109A8800B2EE047A67EE877A174B9FED187A1B7847
:109A98008DF80130FCEEE77A0A2017EE903AD2ED05
:109AA800017A8DF8023067EE877A6946FCEEE77A2C
:109AB80017EE903AD2ED027A8DF80330FCEEE77A91
:109AC80017EE903A8DF80430094B1B788DF8053065
:109AD800FEF73EFD03B05DF804FB00BF3424002010
:109AE80048240020262400204424002000007A4432
:109AF8002A240020054A137883F001031370044ACE
:109B080000231360034A1360AEE700BF2A24002035
:109B1800402400203C240020F0B50124B0FBF4F5DB
:109B28008D4201D34C43F9E70026D4B1B0FBF4F5DC
:109B380004FB1500B4FBF1F41EB9002D01DC002C68
:109B4800F3D1092D03F1010EEFB204DD002A14BF91
:109B58003725572500E030253D441D7001367346F2
:109B6800E3E71C70F0BDF0B50124B0FBF4F58D42BD
:109B780001D34C43F9E70026D4B1B0FBF4F504FB5C
:109B88001500B4FBF1F41EB9002D01DC002CF3D153
:109B9800092D03F1010EEFB204DD002A14BF3725A9
:109BA800572500E030253D441D7001367346E3E734
:109BB8001C70F0BD03685A1C0260197070472DE9CB
:109BC800F843089E002B07468846144614BF4FF0FA
:109BD80030094FF02009334613F8012B0AB92546FE
:109BE80003E0002CFBDD013CF6E7002D04DD3846E0
:109BF8004946C047013DF8E724EAE4743546A01B0E
:109C0800284415F8011B11B13846C047F7E7BDE8ED
:109C1800F883024B1868FCF7BBBF00BF3810002060
:109C280090ED017A07EE901AB5EE407AF1EE10FA4F
:109C380001BFF8EEE77A9FED0E7A67EE877AB7EE06
:109C4800007A04BFC7EE277AC0ED017A90ED017A59
:109C5800D0ED007A30EE877A30EE670AC0EE870AD8
:109C6800E0EE807AB0EE670AC0ED007A704700BF78
:109C7800DB0FC94010B50278202A034600F1010025
:109C8800F9D0092AF7D02D2A03D10346BFEE000ADE
:109C980004E02B2A08BF0346B7EE000ADFED387A46
:109CA8001A46134612F8010BA0F13001CCB2092C68
:109CB8000AD807EE101AB8EEC77AF2EE046AA7EED1
:109CC800A67AF0EE477AECE72E2816D1F2EE046A6F
:109CD8001146B0EE666A0B4611F8012B303AD0B245
:109CE80009280AD807EE102AB8EEC77A87EE267A2E
:109CF80066EE866A77EE877AEDE71A7802F0DF0279
:109D0800452A35D15A782D2A02D10233012004E0A0
:109D18002B2A14BF013302330020013B002213F821
:109D2800011F3039CCB2092C03D80A2404FB0212D3
:109D3800F5E7B2F59A7F28BF4FF49A721346B7EE4B
:109D4800007A072B05D9DFED0F6A083B27EE267A44
:109D5800F7E702F007032BB1F2EE046A27EE267A42
:109D6800013BF8E7F0EE476A20B1C7EE877A03E0D7
:109D7800F7EE006A67EEA67A20EE270A10BD00BF4C
:109D88000000000020BCBE4C30B52DED028B87B022
:109D9800B0EE408A0C220021054603A80BF03FF9DB
:109DA800B5EEC08ADFED2A7AF1EE10FACCBF38EEB4
:109DB800278A38EE678ADFED277A28EE278A6946F0
:109DC800FDEEC87A17EE904A84EAE470A0EBE470DE
:109DD80005F080FA002CACBF20232D2368468DF8AF
:109DE8000C300BF060F9012807D130238DF80D30C5
:109DF8008DF80E308DF80F300CE0022805D1302395
:109E08008DF80D308DF80E3004E0032804BF3023A0
:109E18008DF80D30694603A80BF028F903A80BF05C
:109E280042F90338C4B2224603A928460BF068F960
:109E380000232B55284608490BF018F903AB284690
:109E480019190BF013F9284607B0BDEC028B30BD89
:109E58006F12033A00007A44DC9A010870B506468E
:109E680015460846B6FBF2F414B12046FFF7F6FF94
:109E780005FB1464024B1B5D00F8013B70BD00BF7D
:109E8800DE9A01082DE9F04F814689B08A461646C8
:109E98001C4600253178002900F0DD80252902D0F4
:109EA8000136484675E07278302A08BFB278A2F1C8
:109EB800300319BFB71C4FF0000BF71C4FF0010B14
:109EC800092B4FF0000819D8A2F13003D9B209299B
:109ED80005D80A2202FB083817F8012BF4E7A2F18B
:109EE8006103052B02D8A2F1570305E0A2F1410353
:109EF800052B03D8A2F137030A2BEADD6C2A31D1EE
:109F08003A78642A07F1010600F083800BD8252AE5
:109F18003DD003D8002A00F09E80BBE7582A0CD019
:109F2800632A19D0B6E7732A22D002D86E2A37D00E
:109F3800B0E7752A5CD0782AACD1271D2068A2F139
:109F4800580462424FF01001624155E02CD9582A5A
:109F580032D0632A2AD13E4648462178271DD04769
:109F680001350FE0642A64D00ED9732A14D13E4615
:109F7800236800934846514642460023FFF71FFED8
:109F8800271D05443C4685E7252ADFD13E4648463D
:109F98002521D04701357DE70AD86E2A06D13E46ED
:109FA800236804341D6075E7002A54D03E4671E7E3
:109FB800752A26D0782AF9D1A2F1580304F1040CA5
:109FC8005A422068CDF80CC04FF010015A4105AB39
:109FD800FFF7A2FDDDF80CC03E46644605AB0093D2
:109FE8004846514642465B46FFF7E9FD054451E7BE
:109FF8002068271D0A21002205ABFFF7B4FD3C4667
:10A00800ECE704F1040CCDF80CC020680A2100220A
:10A01800DDE72068002804F1040708DA2D238DF80D
:10A02800143040420DF115030A210022E5E705AB83
:10A03800FAE72068002804F1040C0ADA2D238DF8C9
:10A04800143040420DF11503CDF80CC00A2100224E
:10A05800BEE705ABF8E7284609B0BDE8F08F0FB4B6
:10A0680013B50B4904AB08680A4953F8042B09686F
:10A078000193FFF707FF0446074B1868FCF77CFDC0
:10A088000028F9D0204602B0BDE8104004B070475F
:10A098008C010020880100203810002080EAE0733D
:10A0A800A3EBE0738B4206DB002801DD401A704702
:10A0B80002D00844704700207047FDEEC07A17EEC2
:10A0C800903A2033402B43D8DFED237AB4EEE70AE9
:10A0D800F1EE10FA04DDDFED217A30EE670AF3E7DE
:10A0E800DFED1F7AB4EEE70AF1EE10FA04D5DFEDE2
:10A0F8001B7A30EE270AF3E7DFED1A7AB4EEE70AA7
:10A10800F1EE10FA04DD30EE670A37EEC00A0AE015
:10A118009FED157AB4EEC70AF1EE10FA44BF30EE9F
:10A12800270A37EE400A60EE007ADFED106A9FEDED
:10A13800107AA7EEA67ADFED0F6AE7EE876A9FED41
:10A148000E7AA7EEA67A20EE276AA6EE070A7047CF
:10A158009FED0A0A704700BFDB0F4940DB0FC9407B
:10A16800DB0F49C0DB0FC93FDB0FC9BF9A7C2E3616
:10A17800FAAF4FB93587083CA4AA2ABE00000000F0
:10A18800DFED027A30EE270A97E700BFDB0FC93F01
:10A1980038B52DED068B90ED008AB0EE480A0C46D6
:10A1A8000546FFF7EDFFB0EE40AAB0EE480AFFF70C
:10A1B80084FFD5ED018AB0EE409AB0EE680AFFF749
:10A1C800DFFFB0EE408AB0EE680AFFF776FFD5ED04
:10A1D80002AAF0EE408AB0EE6A0AFFF7D1FFF0EE6D
:10A1E800409AB0EE6A0AFFF768FF60EE0A6A69EE05
:10A1F800297AF0EE665AE7EEA85A29EE8A6A29EE1D
:10A20800007A69EE889A29EE489A28EE400A28EEE4
:10A218000A8AC4ED035AF0EE465AE7EE685AE6EEAB
:10A22800A87AA6EE687AC4ED009AC4ED028A84ED95
:10A23800059A84ED088ABDEC068B84ED010AC4ED0D
:10A24800045A84ED067AC4ED077A38BD10B52DEDB1
:10A25800048B8AB090ED009AD0ED028A90ED018AC5
:10A268000446084601A9FFF793FFDDED047A9DED4A
:10A27800017A68EE277AE9EE077A9DED077AE8EE2B
:10A28800877A9DED027AC4ED007ADDED057A68EEF5
:10A29800277AE9EE077A9DED087AE8EE877AC4ED29
:10A2A800017ADDED067A28EE278ADDED037AA9EE3C
:10A2B800278ADDED097AA8EEA78A84ED028A0AB01A
:10A2C800BDEC048B10BD074B1A8822EA00009042AF
:10A2D80010B518801C4602D00120FCF7FBFB208833
:10A2E80010BD00BF18130020064B1A881043904277
:10A2F80010B518801C4602D00120FCF7EBFB208823
:10A3080010BD00BF18130020024A936823EA00001A
:10A31800906070479424002008B5104B1A780023E9
:10A32800D9B2914207D20E4951F82310096800208A
:10A3380008600133F4E73220FCF777FB094B1B6810
:10A348005A0309D5084B9B685B0305D440F2DC50DF
:10A35800BDE80840FCF769BB08BD00BF80130020BA
:10A36800501300203424002094240020454A6923F7
:10A378002DE9F34113704FF4FB635380BE2313712F
:10A38800EF2382F8D537002382F8D63719461646C8
:10A39800F25C0133B3F5FB6F81EA0201F8D1394B66
:10A3A80083F8D617384B1A69120604D5374A5A600B
:10A3B80002F188325A6004270020013F17F0FF0796
:10A3C8004FD0314B3422DA60002444B1002356F8D0
:10A3D8000480019304F04EFF0428EED117E004F046
:10A3E80049FF0428E9D1284D2B6943F002032B616A
:10A3F800274B6B612B6943F040032B6104F03AFF54
:10A408002B69042823F002032B61DFD0D5E71E4D0A
:10A418002B6943F001032B6104F1006303F57E33DC
:10A428001FFA88F21A8004F025FF042810D1194B6E
:10A4380023440193019B4FEA1848A3F8008004F0D5
:10A4480019FF2B69042823F001032B6105D0B4E719
:10A458002B6923F001032B61AFE70434B4F5FB6FDC
:10A46800B3D1094A1369042843F08003136102D168
:10A4780005F03CFF10B90A20FCF744FB02B0BDE828
:10A48800F08100BF9424002000200240230167458A
:10A4980000F8030802F8030810B50E4C2068FCF712
:10A4A80023FA2068047A002202FB02F3193B634373
:10A4B80003F6C4135343192193FBF1F3064921F81A
:10A4C80012300132072AEFD10449BDE81040FDF7E8
:10A4D80079BE00BFB411002008100020D825002044
:10A4E8002DE9F04105F002FF10B90A20FCF70AFB3C
:10A4F800A44CA549A54D4FF4FB6220460AF084FD03
:10A5080094F8AC37022B84BF002384F8AC3794F856
:10A51800AC274FF4CC7101FB02F3E018234400F59B
:10A528003970286093F8380303F54C73022801FB4F
:10A53800024284BF0020187292F83833944A13708C
:10A548000C2202FB0343934A03F2AE731360A36821
:10A5580046F209021A401AB98A4A43F40053936032
:10A56800A368D80703D54FF40050FFF7CDFEA368C2
:10A57800590409D50820FFF7C7FE4FF40050FFF72C
:10A58800C3FE0120FFF7C0FEA3681A0706D54FF4E3
:10A598000050FFF7B9FE0120FFF7B6FEA3689B0441
:10A5A80002D54020FFF7B0FE94F8DC21754B2AB1A4
:10A5B80093F8E02112B1002283F8E021764B774E20
:10A5C8001E604FF0000C674604EB0C03B3F8F4E18F
:10A5D8004FEA5E0101F077314FEA9E0303F033330F
:10A5E800C1EB0E00C11A4FEADE0303F01133CB1A98
:10A5F80003EB23131EF0010803F00F324FF0FF03A3
:10A6080092FBF3F3C3EB032318BF0137A2EB030359
:10A6180018BFFFB2012B0ADD022B40F0B080B8F161
:10A62800000F00F0AC801EF0BC0F00F0A8800CF109
:10A63800080CBCF1200FC7D1013F012F00F29F8009
:10A64800FFF72AFF302200215548564F0AF0E7FC51
:10A65800554BD5F800801F60544B002108F1790054
:10A66800C3F80080FCF780F9514B80F001001870A6
:10A67800504B07F126021A604F4B07F1D0021A60BF
:10A6880098F8000002F07CFD28684C4B00F5C57274
:10A698001A60FFF761F94A4BDFED4A6A07F1940245
:10A6A8001A60494B00221A809A71484B07F12C0214
:10A6B8001A602B68464A93ED187A03F21911116053
:10A6C800444A03F289111160434A07F108011160F5
:10A6D800424A1760424A07F19C011160414A07F15A
:10A6E800A60111604049536167EE266A0E60B6EE16
:10A6F800007AB4F8661187EE267A101D07EE901AD4
:10A70800B4F86811F8EE677AC2ED027A07EE901A8B
:10A7180093F85C10117193F87810517194F8DF1167
:10A728001174F8EE677AB3F81611C2ED037A07EEE2
:10A73800901A2E492E4A086003F1640111602D4ACF
:10A748002D4982ED007AF8EEE77A9FED2C7A2C4AB3
:10A758000B60C7EE277A2B499FED2B7A67EE877A35
:10A76800C2ED007A03F168020A60284903F2111366
:10A778000B60274B1F60274B1A60BDE8F08104F07F
:10A788004DFD5DE79424002000F803089011002097
:10A79800E0230020B41100201C2F00201E260020DA
:10A7A8003C0F0020D8250020700F0020740F0020D7
:10A7B80003000020BC14002058060020800F002051
:10A7C800300F0020DB0F49407C0E002018150020B8
:10A7D800DC170020A80900202414002028140020D9
:10A7E800BC08002084170020800900204C15002098
:10A7F8008415002080150020E40700200000614433
:10A80800B8080020D80700204C3D0F44A8080020B5
:10A81800B0080020E406002008B5FFF7A7FDFFF701
:10A828005FFE0120BDE80840FCF754B938B50024A4
:10A838000B4D6059254405F043FB696811B109487F
:10A84800FFF70DFCA96811B10748FFF708FC074896
:10A85800103405F035FBB4F5D87FE9D138BD00BF19
:10A86800C07E0108039B0108099B010821A3010878
:10A87800F0B585B004460AF016FC082826D1621EF9
:10A88800E01D1F4912F8013F09681944497801F091
:10A898000301022908BF203B82421370F1D12546EB
:10A8A80004F1080715F8016B164831460AF0EDFB6C
:10A8B80020B1284631460AF0E8FB10B1FCF796FFB4
:10A8C8001CE0BD42EED1204604F0E6FC0E4805F03F
:10A8D800F7FA00230D4A1A4404A992F88A210A4477
:10A8E8000849595C02F80C1C0133082BF2D10023EB
:10A8F80007488DF80C3001A9FFF7B1FB05B0F0BD92
:10A9080018010020C9A101080F9B01089424002008
:10A9180063A20108234B244C1D68206880B5FDF70D
:10A9280015FA2846FDF712FA206841798B0704D4F6
:10A93800036841F002015B6998471C4B4FF40042E1
:10A948009A614FF480429A612068FCF71EF9A0B121
:10A95800164E4FF400433385134B1868FCF712F971
:10A968000746FEF757FC08B103F084FE284639462F
:10A97800FCF70EF94FF40043B3612846FCF705F9DC
:10A988000028E1D0094ED4F800804FF4804737857D
:10A998002846FCF7F7F801464046FCF7F9F8B76196
:10A9A800D2E700BFFC2300209C17002000080048C5
:10A9B8002DE9F04705460AF076FB314E0446D6F8F5
:10A9C800088090B92F4805F07BFA2F4B53F82410D4
:10A9D80049B10123A34013EA080F02D02B48FFF71F
:10A9E8003EFB0134F1E72A4822E02846294922465D
:10A9F8000AF062FB58B92848284C05F061FA54F867
:10AA0800041F0029EFD02148FFF729FBF7E72B782F
:10AA18002D2B03BF013504F1FF344FF0010A4FF02D
:10AA2800000A4FF00009184B53F8297027B91C4841
:10AA3800BDE8F04705F044BA2846394622460AF0F0
:10AA48003BFBC8B9012000FA09F0830501D5154878
:10AA5800EEE7BAF1000F03D0FFF756FC124803E007
:10AA680040EA0800B060114805F02AFA3946104853
:10AA7800BDE8F047FFF7F3BA09F10109D3E700BFD2
:10AA880094240020159B0108708001081F9B010871
:10AA980021A30108239B0108289B01086C80010859
:10AAA800239A0108349B0108429B01084B9B01082B
:10AAB80062A2010810B5084805F002FA074B002405
:10AAC8001C715C63064B1C70FCF7E4F905F0DCFBB9
:10AAD800044B1C6010BD00BF539B01089C1700204D
:10AAE800582F0020FC23002070B5064600240B4B8D
:10AAF800E518AA8816420AD0E1580948FFF7AFFAC4
:10AB08002846002105F069F9064805F0D9F91434FA
:10AB180040F694439C42EAD170BD00BF58850108B5
:10AB28007F9B010821A30108F0B504788BB0054686
:10AB38000CB1002436E04A4B19680E2303FB0411BC
:10AB480001F58C70B1F91D51B1F91921B1F91B3119
:10AB5800009591F82051019591F82151029590F9AD
:10AB68000700039001F590713E4891F90210049195
:10AB780021460134FFF773FA082CDCD16DE02D2B48
:10AB880014D1072C1BDC28460AF0E4FA0AAB661C31
:10AB980003EB440424F8100C15F8013F303B092B53
:10ABA800FAD934462B78002BE9D104E0A3F130021E
:10ABB800092A09D8E5E7082CBDF8182009D00BB0F8
:10ABC800BDE8F040FCF712BE202BF8D1013526462F
:10ABD800E7E7072AF3D8BDF81A00214BA0F2EE21C7
:10ABE80089B240F2DC55A9421B68E8D8BDF81C10B0
:10ABF800A1F2EE24A4B2AC42E1D8BDF81E7004B2B2
:10AC08003EB2A642DBDB0DB2AE42D8DCA542D6DBB3
:10AC1800BDF92440642CD2D1BDF8266034B2112C81
:10AC2800CDDCBDF82050B42DC9D8BDF82240B42CD5
:10AC3800C5D812B24FF00E0E0EFB0233A3F81B114B
:10AC48006421A3F81901A3F81D7183F8205183F832
:10AC5800214183F81F1183F822610BB0F0BD00BFBA
:10AC680090110020899B0108F0B504468FB020465A
:10AC78000AF019FAC5B225BBAC48AD4C05F020F96D
:10AC880094F8D61009B9AB4854E049B294F8D420E6
:10AC980094F8D530009194F8D710019194F9D81010
:10ACA800029194F9D910039194F8DA100491A2480A
:10ACB80029460135FFF7D3F9102D04F10704DFD138
:10ACC800E1E720469D4905220AF0F6F90546B8B99C
:10ACD80029469B4870220AF0A2F99A4B196828461F
:10ACE8000E2303FB001301300022082883F82321D8
:10ACF80083F8242183F8252183F82621F0D113E154
:10AD08002046914904220AF0D7F905462046002D2D
:10AD18004AD120210AF0B9F9002800F00581461C23
:10AD280030460AF0C0F92C460746884B53F82450A1
:10AD38002DB987480FB0BDE8F040FFF790B930460D
:10AD48002946FAB20AF0B8F901340028EDD1784A58
:10AD580002F170011646002382F8DA3082F8D63004
:10AD680082F8D53082F8D43007328A42F3D1794953
:10AD780001EBC40191F80822934210DAD1F80C7261
:10AD8800C3EBC302B0183A4400F1D4011768C0F805
:10AD9800D4709088888092798A710133E7E72946D0
:10ADA8006D48FFF75CF990E06C4907220AF084F9D6
:10ADB80005462046002D4AD120210AF066F90646AC
:10ADC8000AF071F9C4B274BB6548FFF748F9214627
:10ADD80064480134FFF743F90E2CF8D15548FFF7C2
:10ADE8003EF9002460482146FFF739F90025554A05
:10ADF8005E4811680E2202FB04120123D2F82321B7
:10AE08005B49AB4013425B4B05F1010508BF19468E
:10AE1800FFF725F90E2DEAD146480134FFF71FF94F
:10AE2800082CDFD180E0304653490AF097F92C46C8
:10AE380000284CD0022C4FD00AF08CF906AB4E49B2
:10AE480043F8240000200AF089F90134F0E74A4960
:10AE58000AF084F9002460B1082C38D00AF07AF995
:10AE680006AB454943F8240000200AF077F901347D
:10AE7800F1E7082C2BD1069B0F2B28D8DDF81CE016
:10AE8800BEF1070F23D8089F0D2F20D8099E06F181
:10AE98006402C82A1BD80A9DFF2D18D80B9864286D
:10AEA80015D80C99642912D8884210DA0D9C032C05
:10AEB8000DD8324AC3EBC303134483F804E05F712F
:10AEC8009E71DD71187259729C722D4CCFE60FB0CD
:10AED800BDE8F040FCF78ABC069B072B20D80799F1
:10AEE8000D291DD80278722A0DD06E2A18D1154A5C
:10AEF80012680E2000FB032301228A40D3F8231195
:10AF080021EA020209E00F4A12680E2000FB03231F
:10AF180001228A40D3F823110A43C3F8232101E010
:10AF2800FCF764FC0D4CA2E60FB0F0BDB19B010824
:10AF38009424002021A30108DC9B0108F39901084F
:10AF480068250020901100201E9A0108EC91010844
:10AF5800239A0108C07E0108329A0108A99B0108BA
:10AF68000D9B0108F89B01087BA20108FD9B0108C5
:10AF780082A601083CA70108019C0108642500205D
:10AF8800929701082DE9F743047805468CB9324DAC
:10AF980095F8A712B5F8A42295F8A6322F48009183
:10AFA80021460134FFF75BF8102C05F10405EFD1B9
:10AFB8004EE00AF0CFF80F28044636DC2846202158
:10AFC8000AF063F8264EE4B2D6F83880451CA4008F
:10AFD800002728460AF0BEF85FFA87F9B9F1010F91
:10AFE80083B208D0B9F1020F0BD0B3F5B47F24D2E5
:10AFF800B26B13530AE0FF2B1FD8B36B234498702E
:10B0080004E0FF2B19D8B36B2344D87028462C21B1
:10B018000AF03BF8054608B1013502E0B9F1020F24
:10B028000BD10137032FD4D112E00E4800210F2293
:10B0380003B0BDE8F043FCF756BB08EB0400002161
:10B04800042209F0ECFF03B0BDE8F043FCF7CEBBE7
:10B0580003B0BDE8F08300BF94240020039C0108DE
:10B068009C170020CC9901082DE9F04304788FB093
:10B078000546002C59D17C4B0021142209A807AEA3
:10B08800D3F83C8009F0CBFF07223046002109F0B5
:10B09800C6FF05A80023A700059308EB07058380D2
:10B0A8001A467249B5F802E031F813C01CEA0E0FCF
:10B0B8000AD00DF1380C0E3102F1010E6244595CD0
:10B0C80002F81C1C5FFA8EF20133072BE9D100212C
:10B0D8000B46674AB5F802E011F802C01CEA0E0FE9
:10B0E8000AD00DF1380C063203F1010E63448A5C74
:10B0F80003F8242C5FFA8EF301310629E9D118F8F8
:10B1080007305C498DE841006A78029209A81A095B
:10B1180003F00F0305F018FF2146574809AA013428
:10B12800FEF79DFF202CA6D19BE00AF013F81F28FC
:10B13800044600F3898028462021E4B209F0A5FFDF
:10B148001F2C02D9FCF752FB8BE0474BDB6B03EB60
:10B158008404451C00212046042209F060FF0027D2
:10B16800464B09AE304600210A2217F803905FFAD1
:10B1780087F809F054FF002315F8012B32B10A2B88
:10B1880004D04A4502D0F2540133F5E74A4561D16B
:10B1980008F1FF33032B09D8DFE803F0100502425A
:10B1A8000DF1230037E00DF123011FE0304609F0CF
:10B1B800D1FF2378C0B243EA001006E0304609F018
:10B1C800C9FF237800F00F001843207034E00133E2
:10B1D800062B0BD02A4800F2F3269E5D9642F6D144
:10B1E800034493F8ED2263881343638011F8012F19
:10B1F80012B30023EEE70133072B0CD0204A02F2EA
:10B20800E6269E5D8E42F6D102EB4303B3F8D822C0
:10B2180063881343638010F8011F69B10023EDE7C9
:10B22800304609F097FF0F2804DC304609F092FFFA
:10B23800607001E0002363700137052F90D101246D
:10B2480003F0BEF96CB97DE70E4800211F22FCF718
:10B258004AFA06E020460021042209F0E0FE002414
:10B26800EEE70FB0BDE8F0839C1700209881010835
:10B27800AD810108179C0108269C0108B9810108C5
:10B28800C07E0108CC9901082DE9F0412DED048B11
:10B29800B2498AB0044609F0CBFEB14900282046DD
:10B2A8000CBF0126072609F0C3FEAE490028204638
:10B2B80008BF022609F0BCFE002808BF0426F107D3
:10B2C80040F10581A848A94C04F0FAFD002004F0DB
:10B2D80003FCA74804F0F4FDA64804F0F1FD6379E7
:10B2E800A54AA648013B254652F82310FEF7B7FEAB
:10B2F800A348FEF7B4FE4FF00008274695ED058AEF
:10B30800B5EE408AF1EE10FA04D19E48FEF7A7FE8A
:10B31800002570E09C48D5ED069A95ED079AD5ED85
:10B32800088A4146FEF79BFEB5EEC08AF1EE10FA98
:10B3380002D5202004F0BCFDB0EE480A06A8FEF7AE
:10B3480023FD01469148FEF78AFEF5EEC09AF1EE1C
:10B3580010FA02D5202004F0ABFDB0EE690A06A869
:10B36800FEF712FD01468948FEF779FEB5EEC09A50
:10B37800F1EE10FA02D5202004F09AFDB0EE490A49
:10B3880006A8FEF701FD01468048FEF768FEF5EEC7
:10B39800C08AF1EE10FA02D5202004F089FDB0EE43
:10B3A800680A06A8FEF7F0FC08F10108014678488B
:10B3B800FEF755FEB8F10C0F05F110059ED1A4E774
:10B3C80049B294F8D42094F8D530009194F8D71065
:10B3D800019194F9D810029194F9D910039194F835
:10B3E800DA1004916B4829460135FEF738FE102D16
:10B3F80004F1070403D094F8D6100029E0D1002501
:10B408004FF00E0808FB05F80024634A126C42440A
:10B418000123D2F80A20A340134240F0948001345B
:10B428000E2CF2D10135082DEAD15C485C4C04F0B1
:10B4380047FDD7F8088054F8041F19B15948FEF79A
:10B448000EFEF8E70D46584B53F8254054B101233A
:10B45800AB4013EA080F03D054482146FEF7FFFD1E
:10B468000135F0E7524804F02BFD21467B180AAA63
:10B4780093F88A3113444F4A8A5C03F8102C01313F
:10B488000829F3D1002306A94B488DF82030FEF790
:10B49800E6FD4A4804F014FD4948FCF7C3FD494855
:10B4A80004F00EFD4648FFF7DFFD474804F008FDAD
:10B4B8004348FFF767FD4548FEF7D1FD4020FFF7F9
:10B4C80013FB434804F0FCFC3D48FCF7B9FBB2070A
:10B4D80026D5404804F0F4FC3F4804F0F1FC384815
:10B4E80004F03AFB3D4804F0EBFC3548FCF708F95A
:10B4F8003B4804F0E5FC3248FCF7F4FA3948FEF71B
:10B50800AEFD2F48FCF778F9374804F0D9FC2C48F1
:10B51800FFF70AFB2D48FEF7A2FD8020FFF7E4FAAB
:10B52800730716D5314804F0CBFC314804F0C8FC49
:10B53800234804F0EBFA2548FEF791FD4FF480709C
:10B54800FFF7D2FA05E0294622462A48FEF787FD8A
:10B5580065E70AB0BDEC048BBDE8F081329C0108B8
:10B5680042A00108399C01083F9C0108942400204E
:10B578004D9C01085F9C0108EC9101086B9C010837
:10B58800769C0108839C0108909C01080C9B01088B
:10B5980063A20108989C01089C170020B79C010829
:10B5A8006C800108C79C010870800108D59C0108BF
:10B5B800E29C0108C9A10108EE9C0108F79C01085A
:10B5C80092970108069D0108129D010821A3010810
:10B5D800209D01082D9D0108409D01084E9D0108F0
:10B5E800589D0108679D0108759D0108819D010806
:10B5F800929D0108A49D010810B5214A18B9136845
:10B6080002221A8210BD1F48146800230380217883
:10B6180011F07F0102460DD1637A990644BF0221D9
:10B62800017013F0400F037814BF43F0010323F0B7
:10B63800010315E0012921D002291ED1637913F0F5
:10B64800800F03F00F034FEA830303F1804303F5F0
:10B65800B8431B6806D003F03003102B07D1012331
:10B66800137004E003F44053B3F5805FF6E7064B2C
:10B678001B681B699847034810BD184610BD00BFDA
:10B6880094210020E0170020B820002010B5064CB7
:10B6980018B9236801221A8210BD044B1B689B68E5
:10B6A800984720680C3010BD94210020B820002055
:10B6B80010B5064C18B9236801221A8210BD044B34
:10B6C8001B681B68984720680A3010BD9421002029
:10B6D800B820002003788B4283BF034B03EB410162
:10B6E80048880020704700BFE017002070B500228E
:10B6F8001346244914180C44A47E83EA042308241E
:10B7080013F4004F4FEA430318BF83F4815304F145
:10B71800FF3418BF83F0010314F0FF049BB2EFD18C
:10B728000132192AE5D100F1190200F11A050A447B
:10B738000D44967EAA7E02EB062292B29A421FD14F
:10B74800104B93F83B50E2B2AA4216D2431C03EBCB
:10B758004203DBB2CA1801330B44927E9B7E03EB93
:10B7680002239BB24FF4AF6253431B13064A03F5FF
:10B77800487322F814300134E5E7012381F83C309E
:10B7880070BD00BFE0170020E217002003788B424D
:10B798000BD9074B1A78074B89001944086C02B17A
:10B7A800400800F5777080B270470020704700BFEE
:10B7B800A0220020E017002007299DBF034B03EBC0
:10B7C8008101B1F870000020704700BFE017002029
:10B7D800034B03EB4101B1F89000C008704700BF6C
:10B7E800E017002070B5334C0546FBF7F7F8D4F89E
:10B7F800B030C4F8B000C31AB3F5FA5FC4F8B43077
:10B8080082BF002384F8B83084F8B93094F8B8308F
:10B818002BB9A12D02BF274A012182F8B91094F84B
:10B82800B910244A29B1D118EDB201338D7682F8C6
:10B83800B83094F8B85094F8BA30AB4239D11D4BAF
:10B8480093F8BB30052B02D0062B03D02CE0002048
:10B85800FFF74CFFE37E1E2B26D100200246C1B223
:10B868006B1E994219DA21448B7E0821DBB283EAE8
:10B878000206F60744BF83F01803C3F3460301F139
:10B88800FF3154BF5B0843F0800311F0FF01C2F39E
:10B898004702ECD101301A46E1E723449B7E9A42E5
:10B8A80002D10320FFF722FF002384F8B93084F87F
:10B8B800B83070BDE017002010B50446FBF78EF8CD
:10B8C8000F4BD3F8BC20C3F8BC00821A41F2883170
:10B8D8008A42C3F8C02084BF002283F8C42093F8AA
:10B8E800C420074913440F2AE4B218BF013283F871
:10B8F800C54012BF81F8C420012381F8D53010BD9E
:10B90800E017002010B50446FBF768F80F4BD3F892
:10B91800D820C3F8D800821A41F288318A42C3F885
:10B92800DC2084BF002283F8E02093F8E020074958
:10B938001344142A18BF013283F8E14012BF81F87A
:10B94800E020012381F8F63010BD00BFE017002089
:10B958002DE9F843324F3D682A8A2E7AB2B9042E6F
:10B9680014D1304C30482378012B0BD12F4B196858
:10B978002F4B89B20B445B0019681A60302303808F
:10B98800227048E010230380072644E0AC8AAB69A4
:10B99800A24294BF04260226944228BF14461FFAE6
:10B9A80084F840469847214A13689BB203F1005334
:10B9B80003F540535B0004F1010E1B689BB203F1D1
:10B9C800005303F540534FEA6E0E5B0000217145AA
:10B9D80000F1020009D010F8019C10F802CC4CEAE2
:10B9E800092C23F821C00131F1E71268104B92B2FB
:10B9F80013445B001A681C602B8AC8EB03032B8274
:10BA08006B8A9844084BA5F8128030221A80094B9B
:10BA18004FF440521A803B681E72BDE8F88300BF9D
:10BA280094210020592F0020B2200020505C0040B3
:10BA380002300020B02000200E4B0F4A1B689BB23A
:10BA480003EBC00002443E294FEA420209D94B09E0
:10BA5800C80604BF03F1FF339BB29B0243F40043C3
:10BA680004E04B08C90748BF01339B021168136003
:10BA7800704700BF505C00400630002010B5454BB1
:10BA88001A68107810F07F0004D1537A23F020034D
:10BA9800537210BD02287AD15388002B78D11379BC
:10BAA800002B75D1537923F08000840004F1804184
:10BAB80001F5B84113F0800F096814BF01F0300197
:10BAC80001F44051032862D8002960D0927A002AF4
:10BAD8005DD004F1804404F5B8441906226825D5E0
:10BAE80002F03002102A4CD103F07F039B0003F1CF
:10BAF800804303F5B8431A68510641BF196840F6F8
:10BB08000F720A4042F4004244BF42F0C0021A6079
:10BB18001A6822F4E04222F0400292B282F0300227
:10BB280042F4004242F080021A602AE002F44052D5
:10BB3800B2F5805F25D128B9174B93F82C10FFF781
:10BB48007BFF11E09B0003F1804303F5B8431A68BB
:10BB5800520441BF196840F60F720A4042F440424D
:10BB680044BF42F080021A60236823F4804323F024
:10BB780070039BB283F4405343F4004343F08003C3
:10BB88002360064B1B685B699847002010BD0220A4
:10BB980010BD00BF94210020B4000020B820002070
:10BBA8000023036043608360838103614361836191
:10BBB800C36103624362836270478A68036810B591
:10BBC8000C6A14430A6914434A6914438A69144382
:10BBD800CA6914434A6A14438A6A23F4FF4323F068
:10BBE80070032243134303608B8943600B688360AF
:10BBF8004B68C36010BD02684FF6FE7313400360C4
:10BC08000023036043608360C360294B984201D1DD
:10BC1800284A27E0284B984201D1264A2AE0274B98
:10BC2800984201D1234A2DE0254B984201D1214A5F
:10BC380030E0244B984201D11E4A33E0224B98420F
:10BC480004D11C4A536843F470032EE01F4B9842FA
:10BC580004D1184A536843F0706326E01C4B98429D
:10BC680004D11C4A536843F00F031EE01A4B984254
:10BC780004D1184A536843F0F00316E0174B984272
:10BC880004D1144A536843F470630EE0144B98428D
:10BC980004D1104A536843F4704306E0114B9842AC
:10BCA80004D10C4A536843F470235360704700BFB3
:10BCB80008000240000002401C0002403000024020
:10BCC80044000240580002406C00024080000240DC
:10BCD80008040240000402401C04024030040240F0
:10BCE8004404024058040240084BDA68D10709D4DA
:10BCF800DA68D20608D4DB6813F0040F14BF0320F7
:10BD0800042070470120704702207047002002403D
:10BD1800036A23F001030362036A70B54468826909
:10BD28000D6822F4803222F0730215438A8923F0C9
:10BD3800020313438A881343134A90420FD002F533
:10BD4800006290420BD002F54062904207D002F5A3
:10BD58008062904203D002F5806290420DD1CA8978
:10BD6800CE8823F0080313430A8A24F4407414434A
:10BD78004A8A23F00403334314438A684460856184
:10BD88004263036270BD00BF002C0140994A5368AA
:10BD980003F00C03042B2DE9F04105D0082B06D045
:10BDA80095490160B3B916E0934B036012E05368FC
:10BDB8005468C3F38343991CE30349BFD36A8F4B89
:10BDC8008D4C03F00F0344BF0133B4FBF3F34B4333
:10BDD800036000E000235168894FC1F303117D5CC3
:10BDE8000168EDB221FA05F444605668C6F30226EC
:10BDF800BE5D24FA06FEC0F808E05668C6F3C226FF
:10BE0800BE5DF6B2F440C460D2F82C80C8F30418C2
:10BE180008F00F0C07EB4C0C18F0100FBCF810C012
:10BE28001FFA8CFC07D0BCF1000F04D0B3FBFCFC5C
:10BE3800C0F810C000E00161D2F82CC0CCF3442C4B
:10BE48000CF00F0807EB48071CF0100F3F8ABFB231
:10BE580004D01FB1B3FBF7F7476100E04161176BEE
:10BE6800FF065ABF644F87618161176BBF065ABFCF
:10BE7800614FC761C161176B7F065ABF5E4F07628A
:10BE88000162176BFF0506D5994204D1AE4202D173
:10BE98004F00476200E04462176BFF0406D59942E1
:10BEA80004D1AE4202D14F00876200E08462176B72
:10BEB800BF0506D5994204D1AE4202D14F00C762F0
:10BEC80000E0C462176B7F0506D5994204D1AE42E3
:10BED80002D14F00476400E04464176B3F0506D564
:10BEE800994204D1AE4202D14F00876400E08464D5
:10BEF800176BBF0406D5994204D1AE4202D14B005C
:10BF0800C36400E08464156B3A4BAD0701D1046348
:10BF180015E01C6B04F00304012C01D101630EE051
:10BF28001C6B04F00304022C02D14FF4004305E01B
:10BF38001B6B03F00303032B01D12F4B0363146B1B
:10BF48002C4B14F4403F02D1C0F834E018E01C6BCD
:10BF580004F44034B4F5803F01D1416310E01C6B18
:10BF680004F44034B4F5003F02D14FF4004306E036
:10BF78001B6B03F44033B3F5403F01D11E4B4363C1
:10BF8800146B1C4B14F4402F02D1C0F838E018E0B1
:10BF98001C6B04F44024B4F5802F01D1816310E0B8
:10BFA8001C6B04F44024B4F5002F02D14FF4004375
:10BFB80006E01B6B03F44023B3F5402F01D10E4B71
:10BFC8008363146B0B4B14F4401F02D1C0F83CE0A0
:10BFD80020E01C6B04F44014B4F5801F01D1C16348
:10BFE80018E01C6B04F44014B4F5001F0AD14FF498
:10BFF80000430EE00010024000127A0000093D00E4
:10C00800440000201B6B03F44013B3F5401F01D11B
:10C01800134BC363126B134B12F4400F03D1C0F8D8
:10C0280040E0BDE8F0811A6B02F44002B2F5800FDF
:10C0380002D10164BDE8F0811A6B02F44002B2F546
:10C04800000F02D14FF4004306E01B6B03F44003DA
:10C05800B3F5400F01D1024B0364BDE8F08100BF86
:10C0680000127A0000100240F0B500230E681C464A
:10C078000125A54005EA060EAE452BD10F797A1E9B
:10C08800012A15D8856803229A4025EA02028260AF
:10C098004D7982689D4015438560828892B222EA74
:10C0A8000E0282808A798588A2402A4392B28280D1
:10C0B800032205689A40D2431540056005689F40F1
:10C0C8002F430760C7681740CA7902FA03F547EAA1
:10C0D8000502C2600134102C03F10203C8D1F0BD7F
:10C0E80038B52DED048B4A4C0368C4F8F8308388C2
:10C0F800A4F8FC30013A0D46072A42D8DFE802F0DE
:10C10800040A101822292F35B4F8F8300B80B4F837
:10C11800FA3013E0B4F8FA300B80B4F8F83005E0E0
:10C12800B4F8F8305B420B80B4F8FA305B4205E0B3
:10C13800B4F8FA305B420B80B4F8F8306B80B4F88E
:10C14800FC301DE0B4F8F8305B420B80B4F8FA30EC
:10C1580012E0B4F8FA300B80B4F8F8300CE0B4F818
:10C16800F8300B80B4F8FA3005E0B4F8FA305B42E6
:10C178000B80B4F8F8305B426B80B4F8FC305B425B
:10C18800AB80244B93F83030002B3ED1B5F900300A
:10C1980094ED430AD4ED407A09EE103AB5F902302D
:10C1A80008EE103AB8EEC88AB5F90430B8EEC99A64
:10C1B80028EE000A08EE903AA7EE890AF8EEE88A17
:10C1C800D4ED467AA7EEA80A09F038F994ED440AA6
:10C1D800D4ED417A288028EE000AA7EE890AD4ED2A
:10C1E800477AA7EEA80A09F029F994ED450AD4ED93
:10C1F800427A688028EE000AA7EE890AD4ED487AC8
:10C20800A7EEA80A09F01AF9A880BDEC048B38BD7E
:10C21800E017002044000020094B1A68137844F600
:10C22800FB7103EB431300FB03135078C0EB0030A2
:10C23800B3FBF0F39078B3FBF0F080B2704700BF27
:10C248003C12002008B50A4890F8253100EB43035A
:10C258000A22B3F8341189B2A0F83C1100F5A07095
:10C26800FAF799FC80B2FFF7D7FF024B188008BD98
:10C27800E0170020401200202DE9F04F2DED028B31
:10C2880085B007460293A04B1B889807934636D57E
:10C29800109B9E48DC89B0F900301B1B03F2F31594
:10C2A80040F2E632954203D8002BB8BF5B4201E06A
:10C2B8004FF4FA73B0F90220121B02F2F31440F2A1
:10C2C800E630844203D8002AB8BF524201E04FF456
:10C2D800FA729342B8BF1346C3F5FA73052293FB6B
:10C2E800F2F30A22643B53433A7FD2105343642249
:10C2F80093FBF2F3134423EAE373DBB200E0642315
:10C308000093CB1C0193B8460024019BDFF824A2BC
:10C3180013F8016F0193022C4FEA440905D1BAF9C9
:10C3280004301B365E43761146E079493AF814200A
:10C3380031F91410022012FB0011CBF100029142D6
:10C3480003DB59450A46A8BF5A467249029B31F990
:10C358000950551B33F91420154404F0E5FF88B142
:10C3680007EE905A6C4AB8EEE70AB2EE048A105DFE
:10C3780080EE080A04F0D4FB20EE080AFDEEC07A2D
:10C3880017EE905A604A1288D10712D43AF9093048
:10C398001B365E4393074FEA26160DD5BB7C5D43DB
:10C3A8009DF900305D43642395FBF3F506EB2516F4
:10C3B80002E03E7A75432E11584B042533F90930B3
:10C3C80093FBF5F5564BE25C924698F80120751BF5
:10C3D80051466A434A43642192FBF1F297F851109F
:10C3E800D21108EE102AA9B1022CB8EEC80A08D159
:10C3F8004A0803D09142A8BF114600E001214948EC
:10C4080002E0181D00EBC400D3ED070AFDF708FC95
:10C41800BDEEC08ADFF808E1434B98F80B60188836
:10C428000EF1200300FB05F253F82410D21206FB8C
:10C438000216B6F5001F3D4AA8BF4FF400169642F3
:10C44800B8BF16460EF12C0243F8246052F8243087
:10C4580042F82450EB1A0EF138014FF6FF7200092A
:10C46800B2FBF0F043430EF1440051F8245050F869
:10C47800242040F824509B112A4441F8243097F88E
:10C4880050101A444FEA840C761300EE102A79B142
:10C498000EF15000B8EEC00A00EBC400DEED070A4A
:10C4A800CDF80CC0FDF7BCFBDDF80CC0BDEEC00A32
:10C4B80098F8153010EE102A18EE101A5A43534601
:10C4C80053431A463144642392FBF3F3184A1B1270
:10C4D800194422F8091018EE100A02F10801013473
:10C4E8004CF8010002F114012032032C4CF80160D1
:10C4F8004CF8023008F101087FF407AF05B0BDEC35
:10C50800028BBDE8F08F00BF1813002070240020B4
:10C51800502F00202C2400207C8201087411002058
:10C52800A8190020BC190020481100200000E0FFD5
:10C53800101A0020341200202DE9F04F2DED028B47
:10C5480085B080460393BC4B02911C88019204F08D
:10C558000204A4B294B1B94BB3F90240B3F9003064
:10C56800002CB8BF6442002BB8BF5B429C42B8BFE6
:10C578001C46B4F5007FA8BF4FF40074C2460025DE
:10C58800AF4AAE4B32F9152033F81510AD4882EAA0
:10C59800E27EAEEBE27E0BB2BEF5206F4FEA4509B4
:10C5A8004FEA43034FEA850750F8256012DC4FF045
:10C5B800040E92FBFEF29A1A1644B6F57A5FA8BFEB
:10C5C8004FF47A56A04A9642ACBF40F8256040F82E
:10C5D800252002E0002240F82520C6599AF80B20B1
:10C5E800F61156439AF801205343934A12884FEAAA
:10C5F800A31B93074FEAA61654D0944A019B32F91D
:10C608000920022011FB00215A42914203DB8B4290
:10C61800A8BF0B461A468E49039B39F90110511AD7
:10C6280033F915208B1808EE103A04F07DFE68B136
:10C63800B8EEC80A874AB2EE048A80EE080A505D4E
:10C6480004F06EFA20EE080ABDEEC08A82488349DB
:10C658003A5818EE103A42F2107E1A447245A8BFB2
:10C6680072468A42B8BF0A463A5098F8081098F8B5
:10C678001C00594300EB8000C911C0F1000E714540
:10C6880003DB8142A8BF01468E4698F812104A4340
:10C698001213CEEB0B03B61A6643634302EB66260E
:10C6A8000EEB632B664A39F90210042291FBF2F172
:10C6B8006B4A02F19C00405D4143ABEBA11398F833
:10C6C800511008EE103A51B1101DB8EEC80A00EB2F
:10C6D800C500D2ED070AFDF7A3FABDEEC08ADFF860
:10C6E80080E1574B0EF1A00139F8030039F9012018
:10C6F80029F801000FFA80FC0EF1A4010EF1AC003C
:10C70800C2EB0C023B584FF0040C92FBFCF257F8BA
:10C7180001C07A50634498F8501047F800C0134499
:10C7280000EE103A59B10EF15000B8EEC00A00EB15
:10C73800C500DEED070AFDF773FABDEEC00A4849E9
:10C7480001F1B40210EE103A525D53435A1118EE3B
:10C75800103A01F1680E9819801A01F1700329F84E
:10C768000E0018EE100AF85001F17C035242FE50F8
:10C7780001F188030AF1010AFA500B460DB90125A7
:10C78800FEE62E4A9C6AB2F90410029A92790F3298
:10C7980052004A4352112A49002AB1F904104FF0B5
:10C7A800040091FBF0F0A2EB0000B8BF5242322A1D
:10C7B80098F80D100BDC2B4A01FB00418A42A8BFF8
:10C7C8000A4629498A42ACBF9A62996201E000226E
:10C7D8009A6298F8031001FB00F2244909780329AA
:10C7E8004FEAA2120CD9B8F84E10B1F5FA7F07D269
:10C7F8004842824203DB8A42A8BF0A4600E002465A
:10C80800996A9A6741F34F31B1F5807FA8BF4FF419
:10C8180080716FF0FF008142B8BF014650180022B6
:10C82800A3F86C00C3F88410C3F8902005B0BDECE1
:10C83800028BBDE8F08F00BF1813002034120020CF
:10C8480074110020C819002080C1FFFF502F00205C
:10C858002C2400207C8201083C1A0020F0D8FFFF1D
:10C86800A8190020FEFFFF0F020000F0801300202F
:10C878002DE9F04F2DED028B87B000260593C54BAF
:10C888000491B3F90280B3F900300392B8F1000FB4
:10C89800B8BFC8F10008002BB8BF5B429845B8BFC5
:10C8A8009846B8F5FA7F0746A8BF4FF4FA78009083
:10C8B800B1460196B3463446B74D2B88990758D0F0
:10C8C800B44BB64A33F8143032F91420022013FB63
:10C8D8000022039B5B429A424FEA440103DB039B1D
:10C8E8009342A8BF1346AE4A31F902A0059A32F91D
:10C8F8001420CAEB030303EB020A04F015FD88B108
:10C9080007EE90AAA74BB8EEE70AB2EE048A185DC4
:10C9180080EE080A04F004F920EE080AFDEEC07A59
:10C9280017EE90AA3B7A642203FB0AF393FBF2F317
:10C938003A7F6FF0040101FB02FB5B4505DB02EB6C
:10C9480082029342A8BF13469B46974A52F8241086
:10C958000AEB010342F210718B42A8BF0B469349C0
:10C968008B42B8BF0B4642F82430BA7C53431B13A2
:10C9780001932D8805F00303012B38D0854B8C4992
:10C9880033F91490009B51F824E093F801C0894BC7
:10C9980033F9140080EAE073A3EBE073B3F5206F7A
:10C9A8004FEA840616DC09EB89031A0192FBFCF3B3
:10C9B800042290FBF2F0181A8644BEF57A5FA8BFED
:10C9C8004FF47A5E7C4B9E45ACBF41F824E041F8B9
:10C9D800243002E0002341F824308B597D2693FB54
:10C9E800F6F6009BDB7A7343402693FBF6F6AA071C
:10C9F80011D5019BC8F5FA7208FB09F008FB06F58A
:10CA08004FF4FA7102FB0B0002FB035590FBF1F0A7
:10CA180095FBF1F505E0EB074DBF019D354648460E
:10CA28005846644B33F91420042392FBF3F3634A0A
:10CA380002F19C014FEA440A615C4B436FF04F01DD
:10CA480093FBF1F397F85110C31808EE103A51B15F
:10CA5800101DB8EEC80A00EBC400D2ED070AFDF7B6
:10CA6800DFF8BDEEC08ADFF854E1524B0EF1B80191
:10CA78003AF803003AF901302AF8010002B20EF13F
:10CA8800BC010EF1C400D31A042293FBF2F2A300F6
:10CA980051F824C0029350F8243041F8242063440C
:10CAA80097F8501040F824C0134400EE103A59B1DA
:10CAB8000EF15000B8EEC00A00EBC400DEED070A24
:10CAC800FDF7AEF8BDEEC00A3C4A02F1B40110EE23
:10CAD800103A095D01FB03FE18EE101A02F1680016
:10CAE80029444FF0200C9EFBFCF3C91A2AF80010C9
:10CAF800029902F1700E084618EE101A40F80E104E
:10CB080002F17C015B42455002F188014350009BD1
:10CB1800013300930CB90124CEE61E4B946AB3F995
:10CB28000410049B9B790F335B004B435B11214935
:10CB3800002BB1F904104FF0040091FBF0F0A3EBC7
:10CB48000000B8BF5B42322B797B0BDC1C4B01FB2E
:10CB580000418B42A8BF0B461A498B42ACBF936277
:10CB6800916201E000239362F97801FB00F3164912
:10CB7800097803294FEAA31329D9B7F84E10B1F55C
:10CB8800FA7F24D24842834220DB8B42A8BF0B465F
:10CB98001DE000BF3412002018130020502F002081
:10CBA8002C2400207C8201083C1A0020F0D8FFFFCA
:10CBB800C81900207411002080C1FFFFA8190020A7
:10CBC800FEFFFF0F020000F0801300200346916A69
:10CBD800936741F34F31B1F5807FA8BF4FF480715F
:10CBE8006FF0FF008142B8BF014658180023A2F831
:10CBF8006C00C2F88410C2F8903007B0BDEC028B0C
:10CC0800BDE8F08F2DE9F04F2DED0A8B85B08346F6
:10CC1800039390F85030029101921BB1322BA8BFB8
:10CC2800322300E0012307EE903AF8EEE7BADFED91
:10CC3800DE7ADE4B9FEDDECA1B88C7EEABBA002B4F
:10CC480008BF012307EE903AB8EEE7AAD94B2AEEBF
:10CC58000CCA1B887BEE8CBA9807CCEE2BBA27D56A
:10CC6800D54AB2F90030B2F9022083EAE37182EAC8
:10CC7800E270A1EBE371A0EBE27088420446B8BF12
:10CC88000C46B4F5E17F16DA88429FEDCCBA05DD93
:10CC9800002AD8BF524207EE902A04E0002BD8BFE2
:10CCA8005B4207EE903AF8EEE77A87EE8BBA04E03B
:10CCB8009FEDC3BA01E0B7EE00BAC24EDFEDC09AED
:10CCC800CDF800B006F1080806F1100906F11C05B8
:10CCD8000024F0EE69AABC49DFF8D8A231F9143073
:10CCE800B54909EE103AB8EEC99AF5EE047A29EE7C
:10CCF800279A31F91430BAF80010BDEEC99A08EE37
:10CD0800103AF8EEC97A9FEDB19A89074FEA4407BD
:10CD180027EE899AB8EEC88A00F08180AC4931F9CB
:10CD2800143007EE903AF8EEE77AB0EE007AE8EEC3
:10CD3800077A019B5842FDEEE77A17EE901A814276
:10CD480003DB8B42A8BF0B461846A249039B795EBA
:10CD5800401A33F91410084407EE900AF8EEE78AEF
:10CD680004F0E2FA48B19C49F2EE049A88EEA90A66
:10CD7800085D03F0D5FE60EE298A9BF81C30DFEDD4
:10CD8800976A0AEE903A9BF8083007EE903AF8EE68
:10CD9800677AF8EE6AAA68EEA77AB1EE047A67EEC7
:10CDA800A67A2AEE877AFDEEE77A17EE901AF1EE68
:10CDB800477AFDEEE7AA1AEE903A994208DBFDEEB3
:10CDC800C7AA1AEE903A8B42A8BF0B460AEE903AD1
:10CDD800D5ED007AE8EE8C7ABBEE0E7AF4EEC77ADF
:10CDE800F1EE10FAF8EEEAAA09D4B3EE0E7AF4EEF0
:10CDF800477AF1EE10FAC8BFF0EE477A01E0F0EE9C
:10CE0800477AC5ED007A9BF8123009EE903AF8EEB1
:10CE1800699A67EEA97ADFED729A67EEA99ABAF86D
:10CE28000010CA0753D46848385E0028B8BF40428B
:10CE3800B0F5206F03DD0020C9F8000026E0009B54
:10CE48009FED687A5B7868EE077A07EE103AB8EEDD
:10CE5800477A87EE877AD9ED007A37EE497AE7EE96
:10CE68000C7A9FED617AF4EEC77AF1EE10FA09D4E4
:10CE78009FED5E7AF4EE477AF1EE10FAC8BFF0EE55
:10CE8800477A01E0F0EE477AC9ED007A009BD9EDC8
:10CE9800007ADB7A08EE903AF8EE688A8B0768EE3B
:10CEA800A77ADFED538A67EEA88A14D538EE6A8A26
:10CEB800F0EE6A7AEBEE087A78EEE98AB0EE678AE5
:10CEC800F0EE697AEBEE287AF0EE678A03E0F0EE8E
:10CED800698AB0EE6A8A474B9FED477A03F19C0155
:10CEE800625C9BF8511007EE902AF8EEE77A67EE3D
:10CEF800C97AA7EE878A51B1181DB0EE480A00EB2F
:10CF0800C400D3ED070AFCF78BFEB0EE408A96ED1D
:10CF1800007ADFF8E0A0D8ED007AA6EC019A39EEA5
:10CF2800477A0AF1B40187EE0C7A635C09F10409C7
:10CF3800043509EE103A37EE677AB8EEC99AEBEE87
:10CF4800877A38EE280AE8EC017A67EE897A9FED4D
:10CF58002B9A27EE899A30EE490A08F06FFA0AF1FF
:10CF68006801BDEEC88AC85318EE103A0AF170017C
:10CF7800FDEEE88AB1EE499A41F82430BDEEC99A2F
:10CF88000AF17C0118EE903A41F8243019EE103A73
:10CF98000AF18801574641F82430009B0133009379
:10CFA80074BB012497E600BF83F9223E4811002094
:10CFB800BD37863518130020341200200000E143E5
:10CFC80000000000741A002074110020CDCC4C40E1
:10CFD800502F00202C2400207C8201086F12033C73
:10CFE8000AD7A33D0000A043000040C3000040430F
:10CFF8000AD7233CA8190020A69B443BF7CC9238BB
:10D00800029A584B9479B3F90430640028345C438D
:10D01800554BB3F9043000EE103ABAEECF0A08F0D7
:10D028000DFA6411201A002C07EE900AB8BF64426A
:10D03800322CF8EEE76A03DD0023CAF8283029E02D
:10D04800BDEECAAA1AEE103A23F0030307EE903A8F
:10D05800B8EEE7AADFED457A9BF80D30CAEE277ADD
:10D0680007EE103AB8EE477ADAF8283026EE877AD3
:10D0780067EE277AFDEEE77A17EE902A13443C4ACA
:10D088009342A8BF13463B4A9342ACBFCAF8283024
:10D09800CAF82820BB6A5B13B3F5807FA8BF4FF49A
:10D0A80080736FF0FF029342B8BF134607EE903AC1
:10D0B800F8EEE78AFDEEE67A9BF8032017EE903A41
:10D0C80053439B1107EE903A2B4B1B78032BB8EE7A
:10D0D800E78A14D9BBF84E20B2F5FA7F0FD2FDEEDD
:10D0E800C87A534217EE901A994204DB914217EE20
:10D0F800903AA8BF134607EE903AB8EEE78A9BF835
:10D10800511079B14B0803D09942A8BF194600E0E5
:10D118000121B0EE480A1948D7ED070AFCF780FD4F
:10D12800B0EE408A38EE280ABDEEC00A8DED000A3E
:10D13800BDF9003000EE103AB8EEC00A08F07EF9EA
:10D14800BDEEC88AFDEEE88A0023A7F86C0087EDDB
:10D158001E8AC7ED218AC7F8903005B0BDEC0A8B4E
:10D16800BDE8F08F341200207411002000803B4588
:10D17800FEFFFF0F020000F080130020BC19002002
:10D1880001380A4B042804D8DFE800F00507090B2A
:10D198000D00074A08E0074A06E0074A04E0074A84
:10D1A80002E0074A00E0074A1A6070470C010020B5
:10D1B8005513010881C200088116010841C50008FD
:10D1C80079C800080DCC00082DE9F74FA74CF9F7EE
:10D1D80005FC26686568A768861BF643451BC71BC0
:10D1E800ED43FF43F60F8046ED0FFF0F2EB93FB911
:10D1F800002D00F08682B9462CE04FF0000929E0A6
:10D20800B14627E003EB8A0BBBF802301A050ED4AF
:10D2180013F4805F1DBF964A9BF801101268954A67
:10D22800954B14BF52F82120126843F82A20BBF806
:10D238000230D80516D499050AD5904B1B7813F0FF
:10D24800040F0CBF8E4A8F4A8B4B126843F82A2072
:10D2580009F10109207B8C495FFA89FA82450B683C
:10D26800D0D326E0894A5046594601F039F9884B0F
:10D278001B885A0603D550465946864A16E0580771
:10D2880003D550465946844A10E0190703D550463D
:10D298005946824A0AE09A0703D550465946804AB9
:10D2A80004E0DB07D4D57F4A5046594601F018F907
:10D2B800CEE7DFF808E20093BEF906307822A3F53E
:10D2C8007A7353434FF47A7293FBF2F303F22B13FE
:10D2D80001930022F3465FFA82FE864517D2009B2F
:10D2E80003EB820EBEF802E01EF4806F0DD0DFF86B
:10D2F8008891019B39F822E040F2671A9E449EFB10
:10D30800FAFC0AFB1CEE29F822E00132E3E74DB3F0
:10D3180008F5C333A0336360637B544A13BB93732C
:10D32800614B1B6813F0020F0AD0DFF894E19EF8F6
:10D3380000E0BEF1000F03D04FF0010E82F80EE0BE
:10D34800DA0506D5594B5B791BB1A37B43F0020381
:10D35800A3734A4B1B7813F0050F02BFA37B43F05E
:10D368000403A37394F80EE0BEF1000F03D13F4B02
:10D378005B7B002B4FD094F80DC01CF0010FACF173
:10D388000C031DD1BCF1030F07D8DFF8E8903C4A25
:10D398001EF0040F08BF4A4600E0364AACF1040C00
:10D3A800BCF1070F05D8DFF81CC11EF0010F18BF2C
:10D3B8006246DBB2032B0ED81EF0020F3C4B06E090
:10D3C800DBB2032B06D82F4B2A4A1EF0020F18BFD8
:10D3D8001A4600E0274A4FF0000C5FFA8CF38342AC
:10D3E8000DD20B6803EB8C035B881B0642BF224BF4
:10D3F800D2F8009043F82C900CF1010CEDE785B1C0
:10D40800BEF1000F08D0637B184A0133DBB2142B3E
:10D4180006D1002304E025B1637B002BF3D100E0A3
:10D428005373002E52D0234AB2F90250B2F90020A9
:10D43800002DB8BF6D42002A4FF03203B8BF5242E8
:10D4480095FBF3F592FBF3F2EDB2D3B2AB4238BFE2
:10D458002B46194A13B192FBF3F300E013464344F9
:10D468002360E37B014A7BBB01232EE0981A00204E
:10D47800D417002040940108F20D0020562F0020F8
:10D488007893010868930108D81700207E82010864
:10D4980018130020848201088A82010890820108FA
:10D4A800968201089C820108342400207C0E00200A
:10D4B8008093010834120020400D030070240020DE
:10D4C800A0120020889301080023D3738E4D8F4B40
:10D4D8002D78E27BADB9002F00F00E818C4B267BB6
:10D4E8001A788C4B8C4D93F800C08C4BD3F800E025
:10D4F8000B6802F004020021D2B203EB86060F4645
:10D50800B5E01AB9864A1A61002508E0854AFAE7A3
:10D518000A68AB00D6187688760604D40135EBB2D3
:10D528008342F5D3D7E7804EB6F90060192E25DD82
:10D5380012F803E094F814C026690EF00F09E145CB
:10D548000CDCDFF8C8C19CF815C0BCEB1E1FDEBFA1
:10D55800DFF8D8E1D6F800C043F80EC012F803E0AF
:10D5680094F816C00EF00F09E14533DBDFF89CC1D3
:10D578009CF815C0BCEB1E1F2CDC26E0193629DAF6
:10D5880012F803E094F814C026690EF00F09E1457B
:10D598000CDCDFF878C19CF817C0BCEB1E1FA2BFDB
:10D5A800DFF888E1D6F800C043F80EC012F803E0AF
:10D5B80094F816C00EF00F09E1450BDBDFF84CC1FB
:10D5C8009CF817C0BCEB1E1F04DBD6F800E0574ED2
:10D5D80043F806E0544EB6F90260192E1BDD12F826
:10D5E80003C094F814E026690CF00F09F1450CDC2F
:10D5F800DFF8189199F81590B9EB1C1FDEBFDFF81A
:10D608002CC1D6F8009043F80C90D25C02F00F0CB5
:10D61800F4451EDD82E7193680DA12F803C094F863
:10D6280016E026690CF00F09F1450CDBDFF8DC90F9
:10D6380099F81590B9EB1C1FDEBFDFF8F0C0D6F8DB
:10D64800009043F80C90D25C02F00F0CF445FFF602
:10D6580065AF94F817E0BEEB121FA2BF334A3668D5
:10D668009E505BE75888000504D404330435B34260
:10D67800F8D122E04AB101EB0C0A06209AFBF0F936
:10D6880000FB19A001280DDC01E057B9012793F828
:10D6980001900EEB89003EF829A090F80290C0781E
:10D6A80003E01746002081468246013125F802AC86
:10D6B80085F800906870C9B2D7E7164A1378013B1D
:10D6C80013F0FF0308BF06231370114B1B785B0789
:10D6D80041BFBBF90630A3F57A7303EBC3034FF4DC
:10D6E8007A7243BF93FBF2F30133DBB20123104A92
:10D6F80092FBF3F34344A36003B0BDE8F04FF7F7A0
:10D70800EBB803B0BDE8F08FAB0E0020981A0020EC
:10D71800562F002076000020F40D0020D41700209A
:10D72800849301084094010834120020F20D00206F
:10D73800400D0300026BC168034610B5406942B151
:10D748001A6C8C1A013A005D08BF0A46C0B21A6406
:10D7580010BD1A6A805C01328A4228BF0022C0B21A
:10D768001A6210BD436B13B190F844007047836A86
:10D77800406A1B1A584258417047036B13B15B68E3
:10D78800016C01E0C369016A8B423CBFC2689B1807
:10D79800581AC0B27047836A8169426B1944D160D4
:10D7A800416A99429DBF0169CB1A5360CB1A96BF53
:10D7B8000023536083624FF0000380F844301368FD
:10D7C80088BF816243F0010313607047436A82692E
:10D7D800D154436A02690133934228BF002343624C
:10D7E800436B1BB11B68DB0705D4D4E7026D1368D4
:10D7F80043F08003136070474171F6F70BBF8160F7
:10D80800F6F708BF026D036B70B50446D5699BB97E
:10D81800A90611D5C36A1BB1908C80B298470BE05A
:10D82800E169928C40694E1CD2B2E6614254E169CA
:10D83800E268914228BFE361616BA1B92A0612D55B
:10D84800636AA26A9A42236D09D0501CA669A06235
:10D85800B25C1A852369984205D3A16203E01A686D
:10D8680022F080021A602B0742BF236D08221A6239
:10D8780070BD0D4B0D484FF400525A600C4A1168A8
:10D888004FF6FE730B401360426B11684FF6FE7340
:10D898000B401360426A836A9A4200D07BE70123F7
:10D8A80080F84430704700BF000002408C230020FD
:10D8B800440002402DE9F0471E46A24B8CB0984226
:10D8C800894690469DF850507ED19F4B9F4A1A60DA
:10D8D8009F4A5A6102F580729A614FF48072DA6049
:10D8E8001A619C4A1A63143A5A63A2F54842203ACC
:10D8F800DA6404329A64C3F808801865964B9A690A
:10D9080042F480429A615A6942F001025A61022344
:10D918008DF80830032315F0010A8DF809304FF00F
:10D9280000038DF80A3014BF022301232C078DF859
:10D938000B3017D5894C102701978AF001038DF811
:10D948000A30236A23F470232362236A43F4E02312
:10D958002362204601A9FEF787FBBAF1000F23D105
:10D96800A76121E0B0070ED50CA9102341F82C3D82
:10D978007A48036A23F470230362036A43F4E023BA
:10D988000362FEF771FBF1070ED50CA9202341F8BD
:10D998002C3D7248036A23F470030362036A43F45C
:10D9A800E0030362FEF760FB0E238DF800300022CF
:10D9B800012368468DF801308DF802208DF8033078
:10D9C800614C03F063F80CE1654B984276D1654BE6
:10D9D8005E4A1A604FF48072DA601A61624A5A61CC
:10D9E80002F580729A615C4AC3F808801865D369A9
:10D9F80043F40033D36102238DF80830032315F074
:10DA0800010A8DF809304FF000038DF80A3014BF71
:10DA1800022301232A078DF80B3019D54FF09044C3
:10DA28004FF4804701978AF001038DF80A30636A42
:10DA380023F070636362636A43F0E06363622046C5
:10DA480001A9FEF711FBBAF1000F27D1A76125E064
:10DA5800B30710D50CA94FF4804341F82C3D4FF083
:10DA68009040436A23F070634362436A43F0E06383
:10DA78004362FEF7F9FAF70710D50CA94FF40043F3
:10DA880041F82C3D4FF09040436A23F070434362C5
:10DA9800436A43F0E0434362FEF7E6FA26238DF833
:10DAA80000300022012368468DF801308DF80220ED
:10DAB8008DF803302B4C02F0E9FF92E02B4B984293
:10DAC80040F010812A4B214A1A604FF48072DA60C4
:10DAD8001A61284A5A6102F580729A611E4AC3F88F
:10DAE80008801865D36943F48023D36102238DF835
:10DAF8000830032315F0010A8DF809304FF00003B0
:10DB08008DF80A3014BF022301232C078DF80B303F
:10DB180034D5194C4FF4806701978AF001038DF8CA
:10DB28000A30636A23F470636362636A43F4E063F0
:10DB38006362204601A9FEF797FABAF1000F41D1B6
:10DB4800A7613FE0003801408C230020A48201082F
:10DB5800B01A002058000240001002400008004897
:10DB68000044004038230020B01C0020004800403A
:10DB7800E4220020B01E002000040048B0070FD5A2
:10DB88000CA94FF4806341F82C3D5848436A23F4AC
:10DB980070634362436A43F4E0634362FEF764FAE6
:10DBA800F1070FD50CA94FF4006341F82C3D4F48FD
:10DBB800436A23F470434362436A43F4E043436295
:10DBC800FEF752FA27238DF8003000220123684619
:10DBD8008DF801308DF802208DF8033002F056FFE1
:10DBE800434CC4F82C900027012384F84430276262
:10DBF800E761A76267626671C4F80880A57120466C
:10DC0800F6F708FDF20734D5236B002B2AD001A8BC
:10DC1800FDF7C6FFE36C01934FF480530A9380230A
:10DC28000693E368ADF8103020230993206B6369ED
:10DC380002930B970597079708970397FDF7DBFF64
:10DC480001A9206BFDF7B9FF236B216D1A6842F01B
:10DC580001021A608A6842F040028A605B689BB2DF
:10DC6800236406E0236D20221A621A6842F020021B
:10DC78001A60B3072FD5636B43B301A8FDF790FF74
:10DC8800A36C01934FF480530A938023069323696E
:10DC9800ADF8103000251023606B03930B950595A4
:10DCA800079508950995FDF7A6FF606B01A9FDF793
:10DCB80084FF636B1A6842F002021A60226D5D608D
:10DCC8005D60936843F08003936004E0226D1368FD
:10DCD80043F080031360226D136843F0010313605F
:10DCE800204600E000200CB0BDE8F08700040048A2
:10DCF800E4220020704708B50B4B002093F82C1045
:10DD0800FDF79AFE094B1B68187A082801BF084BD3
:10DD18004FF480521A80102208BF5A80A0F10903DC
:10DD28005842584108BD00BFB4000020942100208B
:10DD3800B0200020024B4FF480221A60704700BFC9
:10DD480014040140704770477047FEE7FEE7FEE79E
:10DD5800704730B50024E3B293420DD2030F092B6C
:10DD680094BF3033373301F8143001EB44030025F6
:10DD780000015D700134EEE730BD30B5002202F1DC
:10DD8800805303F5B8539B0042F400441D6840F6E5
:10DD98000F7144F08004294001322143042A19609C
:10DDA800EDD1024B40F08000186030BD4C5C004063
:10DDB8002DE9F347884D894C2B68894E9BB2A38087
:10DDC800A28831880A40970507D54FF6FF53854A40
:10DDD8002B6013780133DBB21370A3880B4018044F
:10DDE80040F100830023ADF802302B687B4F9AB2D4
:10DDF8001804A28040F1F682BB8803F00F03BB71C0
:10DE0800002B40F0C182784A13689BB23B803B8864
:10DE180003F030037B803B8803F440533B80116858
:10DE28004BF6BF730B4083F4005383F0200343F495
:10DE3800004343F080031360BB88D90621D41168DE
:10DE480048F60F730B40694913600B681A7A022A67
:10DE5800884601D0042A02D1FDF77AFD5AE2062A43
:10DE680040F06B825A78052A08D11A78520605D1F3
:10DE7800D878FFF782FFBB681B6A9847E3689B68FE
:10DE88005AE213689BB2ADF80230BDF802301F05A4
:10DE980040F1D0811168554F40F68F730B405449BB
:10DEA80013600A68534B92B213445B0088461A68A1
:10DEB8003B68187A092817D092B2520002F18042C2
:10DEC80002F5C04211781970517859709188C8B21A
:10DED800090A41EA002159801189C8B2090A41EAB0
:10DEE800002199809289DA8001221A72DA8893F8DF
:10DEF8000190002A40F0DC801A7812F07F024AD1A3
:10DF0800B9F1090F0FD1DA78012A00F2B8809978AF
:10DF1800002940F0B4809988002940F0B0809A72B6
:10DF2800A3685B68A9E0B9F1050F10D193F9032044
:10DF3800002A01DA0823B9E09A78002AFAD19A88E7
:10DF4800002AF7D19B7A002B00F0A280F2E7B9F102
:10DF5800030F0ED1DA78012A40F091809A88002ABE
:10DF680040F08D805A7A42F020025A72A368DB6929
:10DF780083E0B9F1010F40F08280DA78012A7ED17E
:10DF88009A88002A7BD15B7A980678D5FDF776FDCA
:10DF980000287DD073E0012A2ED1B9F10B0F6ED184
:10DFA800E26858799269D97890473B689A7A002A4A
:10DFB80065D0002863D11A79002A60D19B78002B9C
:10DFC8005DD1064B9B68DB689847084B1B685A79FC
:10DFD800DA72DA781A735BE0445C0040B020002003
:10DFE800FC2100205A2F0020005C004094210020D2
:10DFF800505C004004300020022A40D1B9F1010FE2
:10E00800C4D0B9F1030F3AD1587920F0800E4FEA05
:10E018008E0202F1804101F5B84110F0800F0968C5
:10E0280014BF01F0300101F44051BEF1030F26D8AE
:10E03800B3F802E0BEF1000F21D101B39B7AF3B12E
:10E0480002F1804202F5B842010613684BBF23F47F
:10E05800E04323F4804323F0400323F070034BBFD5
:10E068009BB29BB283F0100383F4805343F40043C4
:10E0780043F080031360A3689B69984708E0E3684E
:10E0880048465B69984703280FD000287FF452AFB1
:10E09800D8F80020A14B92B213445B001A68002202
:10E0A8001A6030236380062300E009233A6847E1B9
:10E0B800B9F1060F12D11A78520678D19B78012B44
:10E0C80002D1E368DB6967E0022B02D1E3681B6ACF
:10E0D80062E0032B6BD1E3685B6A5DE0B9F1000F86
:10E0E80038D15988002962D15A6822F47F42B2F5A2
:10E0F800003F5CD11A7812F07F0204D19B88002B74
:10E1080000F0D58153E0012A08D1E2685879926974
:10E11800904700284BD13B689B7A17E0022A46D1EA
:10E128005A7902F00F010BB29B0003F1804303F50B
:10E13800B84312F0800F1B6814BF03F0300303F4D8
:10E148004053032933D812F0700F30D1002B40F020
:10E15800AE812CE0B9F1080F04D11B785B0600F002
:10E16800A88124E0B9F10A0F21D11A7802F07F02C0
:10E17800012A1CD19A7AD2B15988C1B95A6822F4B5
:10E188007F42B2F5803F12D1E26858799269904790
:10E19800002800F090810AE04BB13A684FF000087F
:10E1A800A2F8128093614046984740460BE0E36826
:10E1B8003A681B6950789847032804D1584B1B6864
:10E1C80009221A72BDE03A68138A4FF6FF718B4232
:10E1D80001D10923B4E0022800D00BB90823AFE02D
:10E1E80092F9001000291FDAD18801910198834221
:10E1F80002D9019B138210E08B420ED2E16891F89C
:10E208002C00834201D2002105E093FBF0F100FBD2
:10E21800113313B90121434B1970E36893F82C307B
:10E228009382FDF795FB8CE0032313724FF4405360
:10E23800238086E0BDF802301BB2002BBFF6D5ADB7
:10E24800116840F68F730B401360354A17683B7AA4
:10E25800022B904671D0042B6FD0032B01D0052BD5
:10E2680066D1BB693A8A8BB9398A00293BD04FF409
:10E27800405323802C4B1A68284B92B213445B00FE
:10E288001A6800221A60302363802CE0002AEBD041
:10E29800B7F81490914528BF91461FFA89FA50465D
:10E2A80098473B8ACAEB03033B827B8A53447B82B1
:10E2B8001D4B1A681D4B92B213445B0009F1010211
:10E2C8001B689BB203F1005303F5405352105B00E7
:10E2D8004FF0000E9645C7D053F82E1020F81E10A8
:10E2E8000EF1010EF6E7BB8A8B42D8F8003001D850
:10E2F800032201E011B105221A720BE006221A72FC
:10E30800094B1A68054B92B213445B001A681960EE
:10E3180030236380D8F800301B7A0FE002300020E9
:10E3280094210020592F0020505C00400430002028
:10E33800072B02D1E368DB6898470823D8F8002048
:10E348001372FFF7D8FC5E4B1A684BF6BF73134085
:10E358002288D704228848BF83F4805390046288B7
:10E3680048BF83F40053D106628848BF83F0100386
:10E37800920648BF83F0200343F4004343F0800330
:10E388004F4A9BB213602DE09A0002F1804202F5D9
:10E39800B842116889B2ADF80210BDF8021009B28E
:10E3A800002909DA106840F68F7101401160013BBD
:10E3B800444A52F823309847BDF802301F067FF5CB
:10E3C80014ADA1798B0003F1804303F5B84348F6F7
:10E3D8000F72186802401A603A4B03EB81039B697D
:10E3E800984702E5A28833881340590505D54FF6AA
:10E3F800FF332B60344B5B689847A28831880A400A
:10E40800920444BF4DF6FF732B60A3882F4A0B403C
:10E41800DB0452D54EF6FF732B6000231374137C74
:10E42800052B41D8DFE803F0030D1418222D63698A
:10E43800264D1BB900F0DCFF062300E005232B74F2
:10E448003BE000F0D5FF042323740123636134E02B
:10E4580002236374032328E0637C013BDBB263740B
:10E46800637C53BB194B04221A7426E0184A1368BC
:10E478009BB243F010031360052323740A236374CB
:10E488001BE0637C114A013BDBB26374637C03F0DD
:10E49800FF0093B90E490C684FF6EF7323400B60E9
:10E4A80006231374506108E00623237405E0094B22
:10E4B80073E6094B71E6094B6FE602B0BDE8F087D9
:10E4C800005C0040BC820108B4000020B02000209D
:10E4D800405C004001B60008B9B6000895B60008CF
:10E4E80010B54B88DC0641BF2F4B14791B6853F8D5
:10E4F800244044BF2D4B43F820404B889B0641BF26
:10E50800294B54791B6853F8244044BF274B43F8E0
:10E5180020404B881C070ED5254B0C781B78B3EB95
:10E52800141FA1BF204BD4781B6853F82440A4BF04
:10E538001E4B43F820404B889B070ED51D4B0C788B
:10E548001B78B3EB141FDFBF174B54781B6853F8C5
:10E558002440DCBF154B43F820404B88DC070FD51F
:10E56800154C0B78247803F00F03A342DFBF0E4B42
:10E5780014781B6853F82440DCBF0C4B43F8204048
:10E588004B885B070FD50B780C49097803F00F030C
:10E598008B42A1BF044B92781B6853F82220A4BF7A
:10E5A800024B43F8202010BDD4170020F20D0020A4
:10E5B800AF1A0020AD1A0020AC1A0020AE1A0020B5
:10E5C800254A264826490023F0B5156803700B70C4
:10E5D8001C461A462E1976884EB92F5D3FB903702E
:10E5E80000230A704B7007781C461A460CE0360563
:10E5F80048BF013204F1040403F1010348BFD2B259
:10E60800802CDBB2E6D1EAE7E0B2B8420CD215F8CA
:10E61800240006099E4200F00F00A8BF731C904218
:10E62800A8BF421C0134EFE78A704B70C2F3470160
:10E6380002F001020A444C1E0A490B480A70C3F34F
:10E64800470203F00103134404700849501E084AA6
:10E6580008701370F0BD00BFD8170020A41A00205E
:10E66800C8200020AE1A0020AC1A0020AF1A0020E3
:10E67800AD1A00202DE9F04FC24BDA682DED028B60
:10E688001A61C14A1168D960C0490B6843F0200378
:10E698000B60BF4B1978012990460CBF002201225C
:10E6A8001A70BC4B1A78910789B040F13D83BA497A
:10E6B8000978042940F23883B849097801F004013F
:10E6C80001F0FF0011B922F001021A701B78DB0774
:10E6D80002D408B1FBF7A2F9B149CA78531C052244
:10E6E80093FBF2F202EB82029A1AAE4BCA701B78C5
:10E6F800039392000023AC4CDFF8CCC2DFF8D89229
:10E708005CF8231091FBF9F504F1080004F11006F8
:10E7180040F82350A54844F8231000FB051142F2A5
:10E72800107091FBF0F080B226F813004FF0140E31
:10E7380004F1140604F13C0A0EFB036E5AF8236038
:10E748005EF802704EF80210F61B314444344AF861
:10E758002310052691FBF6F109FB051144F8231057
:10E76800039C012C4FEA830BE24605D10238B0F531
:10E77800797F98BF4BF80C100BB90123BBE7884C85
:10E78800D8F80030226D9FED8A7A8A4E8A4D9B1AFE
:10E7980007EE903AF8EE677AD8F800302365C7EEAE
:10E7A800877A7C4B1B78B7EE008AF4EEC87AF1EED4
:10E7B80010FA58BFF0EE487A13F00103C4ED157A49
:10E7C80012D005AA00927D4B06AA01920CCB9AE8BA
:10E7D8000300FBF721F86421059A069BB2FBF1F2CE
:10E7E80093FBF1F3328000E033802B8094F85830AB
:10E7F8006B48002B3BD0D0ED157AC26DDAF80030AB
:10E80800C8EE276A9B1A026E022507EE103AB8EE88
:10E81800C77ADAF8043027EE267A9B1AFDEEC77A13
:10E82800B0F9662017EE901A07EE903A644BB8EEEE
:10E83800E77AD3ED007A67EE277A67EEA67AFDEEDF
:10E84800E77A17EE903A02FA83F3B0F9642093FB63
:10E85800F5F302FA81F29BB292FBF5F292B2A0F8BC
:10E868006A30A0F86820A0F86630A0F86420012378
:10E8780084F85830534BDAF804101B88DAF8000093
:10E88800474D514E216603F03003E065002B00F040
:10E898004B8205F17403009305F178030193EA6E46
:10E8A8002B6FFAF7B9FF72682B6F9B1A07EE903A35
:10E8B800434B326893ED007AEB6EF8EEE77A9B1AD9
:10E8C800EB67384B67EE877A1B78FDEEE77A012B0A
:10E8D800C5ED207A03D0022B00F0DF8024E2D5EDCD
:10E8E800287A3A4BD5ED215A95ED255A95ED156ABA
:10E8F80095ED264AD5ED274A35491D68B1EE677A68
:10E90800BDEEC77AFDEEE77A17EE10EA17EE90CA69
:10E918000020304A91ED007A52F8207007EE907A84
:10E92800F8EEE77AA2F1140367EEA57A33F81060DF
:10E93800FDEEE77A283217EE903A9B1B9BB222F83D
:10E9480010301BB207EE903AF8EEE77A3B4467EED8
:10E95800857A4400FDEEE77ACDED037A07EE903A2A
:10E96800F8EEE77ABDF80C8067EE847AA7EE867A2F
:10E97800FDEEC77A17EE902A724531DB6245A8BFD3
:10E9880062462EE0E807002058240020501200209C
:10E99800BA110020541200205A120020562F0020CD
:10E9A800C82000207C0F0020CC200020806967FF51
:10E9B80000007A44CE120020D0120020BC110020A2
:10E9C80078000020181300205C120020800F00201F
:10E9D800B00F00204421002080969800DB0FC9402A
:10E9E800724607EE902AF8EEE77A5FED046AC1ED09
:10E9F800007AFDEEE77A313617EE903A43449AB240
:10EA0800AB78D1ED027A07EE103AB8EE477A4B6848
:10EA18004F6027EE267AFB1A88EE077AB6B2622E86
:10EA280006EE903AF8EEE66A37EE067AC6EE866AA1
:10EA380086EE077A76EEE76AE7EE267AC1ED047A83
:10EA4800C1ED027A0FD964EEA77ABA4EFDEEE77AE5
:10EA580017EE903AB3F5FA6FA8BF4FF4FA63B342D2
:10EA6800B8BF334600E0002313441BB240F6B83267
:10EA78009342A8BF1346B04A9342B8BF1346AF4A61
:10EA8800A352AF4A142303FB002351F8142B1A6036
:10EA9800002840F0498101203BE7AA4BD5F8748053
:10EAA8001F68D4F878903E89DFEDA78A4FEA5803AB
:10EAB8009E4228BF1E46B5F8A8301AB29642C3BF78
:10EAC800D5ED157A9FEDA17A67EE877AB6B2C1BF08
:10EAD800FDEEE77A17EE906AF618B6B2C8BFA5F849
:10EAE800A860D4F8AC50C5EB09052846FAF7D8FE5B
:10EAF8000028D8BF404241F293129042CCBF002078
:10EB0800012088B307EE905AB8EEE70A20EE280AEB
:10EB1800FBF7D3FA07EE908AF8EE677A40F6B83337
:10EB280020EE270AFDEEC07ACDED037ABDF80C2061
:10EB3800A4F8B02012B29A42A8BF1A467E4B9A4255
:10EB4800ACBF09EB02034B4448F6A042934203DDF5
:10EB5800A3F50C43A03B04E0002BBCBF03F50C431A
:10EB6800A033C4F8B43001E0C4F8B490D4F8B45079
:10EB7800C5F50C53283307EE903AF8EEE77A67EEBE
:10EB8800A88AB0EE680AFBF7FBFA8DED070AB0EE2B
:10EB9800680AFBF792FAD4ED317AD4ED2E4AD4ED17
:10EBA800155A94ED2F4A94ED305A65498DED060AB1
:10EBB800B1EE677ABDEEC77AFDEEE77A0DF1180E71
:10EBC80017EE10AA17EE90BA0020614AFEEC016A0F
:10EBD80032F91030DFF88C9107EE903A07EE106AA0
:10EBE800F8EEE77AB8EEC77A3C32D6EE877A4FEA83
:10EBF800400CFDEEE77ACDED037ABDF90C30B3F5A4
:10EC08007A7FA8BF4FF47A734B45B8BF4B461FFABB
:10EC180083F922F810900FFA89F207EE902AF8EE9D
:10EC2800E77A27EEA47ABDEEC77A8DED037A27EE50
:10EC3800847AD1ED007ABDF80C90E7EE257AFDEEE6
:10EC4800E77A17EE902A524503DB5A45A8BF5A4681
:10EC580000E0524607EE902AF8EEE77A9FED3D6A0B
:10EC6800C1ED007ABA7891ED027A06EE902AF8EEB4
:10EC7800666A4A684B6066EE866A9A1AC8EE266A21
:10EC8800143106EE102AB8EEC66A76EEA56A86EE4C
:10EC9800256AC5EEA66A36EE476AA6EE867A01EDC3
:10ECA800017A01ED037A25EE077ABDEEC77A17EEF1
:10ECB800103ABDEEE77A4B4417EE102A13441BB204
:10ECC80040F6B8329342A8BF13461B4A9342B8BFD6
:10ECD80013461A4A2CF802301F4A142303FB002358
:10ECE800C3ED007A08B901206FE73B7923B16423AB
:10ECF80095FBF3F5194B1D803B8898450DD9D4F841
:10ED0800AC30A06FC01AFAF7CBFD80EAE072A2EB34
:10ED1800E07242F210739A4206DD114B01221A701A
:10ED28000E4BB4F8C8201A8009B0BDEC028BBDE8C0
:10ED3800F08F00BF30F8FFFF48F4FFFF04100020F9
:10ED4800D80F0020800F0020D30237390000C842B6
:10ED580030210020DB0FC940B00F0020780F0020C1
:10ED68007C0F002018FCFFFF20B9034B1B6808220A
:10ED78001A82704701487047942100207C000020C7
:10ED880020B9034B1B6808221A8270470148704754
:10ED9800942100207C00002021B901288CBF02208A
:10EDA800002070470220704710B5094B1A68D378C5
:10EDB800042B0BD8074C518ADB00234418B99B89D4
:10EDC8005B1A138210BD9B68581810BD002010BD37
:10EDD800942100207C000020054B1968054B4A8AC5
:10EDE80018B99B8D9B1A0B827047986A104470471C
:10EDF800942100207C000020054B1968054B4A8AA5
:10EE080018B99B8E9B1A0B827047186B1044704779
:10EE1800942100207C000020074B1B681B7803F01E
:10EE28007F03212B06D100F0DF00022814BF022047
:10EE3800002070470220704794210020212810B537
:10EE480008D1114B1B681B7803F07F03212B10D0CE
:10EE5800022010BD2028FBD10B4B0C4A1B681070F8
:10EE68001B7803F07F03212B094B18BF00230BB934
:10EE7800EEE7084B044A1268002493615482204646
:10EE88009847204610BD00BF942100205B2F00202A
:10EE980071ED000889ED00087047034B1A78202AA5
:10EEA80004BF00221A7070475B2F0020014B042218
:10EEB8001A6070473C2F0020034B9B7B13B1034B18
:10EEC80005221A60704700BF942100203C2F0020C3
:10EED8000D4B0E491A680E4B92B213445B000D4A53
:10EEE8001B68C3F3090310B51362136A9BB201339D
:10EEF8005B1000229A4206D0074851F8044B20F8CC
:10EF080012400132F6E710BD505C0040206200401C
:10EF18001E30002094210020B8210020014B00223F
:10EF28005A667047942100202DE9F843664B674ED6
:10EF38001B68DFF8B881664A00254FF0C0099D724A
:10EF480083F80990DD723560D8F8003023F4EC437B
:10EF580023F0700343F400739BB2C8F80030D8F86C
:10EF6800003023F4E04323F040039BB248F28004CE
:10EF780083F010032343C8F80030336812FA83F390
:10EF88005B0040271A681F6033689BB203F1005387
:10EF980003F540535B0028461A6880221A60D8F8A7
:10EFA800003023F4F8731B051B0D2343C8F8003009
:10EFB800484B93F86410FCF73FFDD8F80030464AF8
:10EFC800464923F4804323F070039BB283F44053F3
:10EFD8002343C8F80030136823F4EC4323F070038C
:10EFE8009BB21360336811FA83F35B00032019683E
:10EFF800C3F8009013683A4923F4E04323F0400330
:10F008009BB283F0200323431360136823F48043E7
:10F0180023F0700323439BB21360536823F4EC433B
:10F0280023F0700343F4C0639BB25360336811FA52
:10F0380083F35B0019684FF480711960536823F4F7
:10F04800804323F0700323439BB25360536823F437
:10F05800E04323F040039BB283F020032343536033
:10F06800D8F80C301F4A23F4EC4323F070039BB20A
:10F07800C8F80C30336812FA83F35B0039461A6813
:10F088004FF488721A60FCF7D7FCD8F80C3023F4D8
:10F09800804323F070039BB283F440532343C8F8A2
:10F0A8000C30D8F80C3023F4E04323F040031C4321
:10F0B800A4B2C8F80C402846FEF75FFE0A4B0122AE
:10F0C8001A60BDE8F88300BF94210020505C00401E
:10F0D800043000207C000020045C00400830002040
:10F0E800103000201C3000203C2F0020005C004025
:10F0F800134A144B50681B68181810B5146808D0C8
:10F1080011490822FEF725FE204610490422FEF781
:10F1180020FE0F480268002393720E4A01211160F5
:10F128000D4913604FF4E0540B6014600B604FF40A
:10F138003641A0F868101160084A136010BD00BF7E
:10F14800B0F7FF1FACF7FF1FE6000020F600002015
:10F1580094210020405C0040445C00403C2F00208B
:10F1680010B50446B0F9000001F061FCB4F90200E2
:10F1780001F05DFCB4F90400BDE8104001F057BC93
:10F1880010B50446006801F052FC606801F04FFCBD
:10F19800A068BDE8104001F04ABC2DE9F74F0120F6
:10F1A800F9F708F8002488B3012C2FD8194E4FF02E
:10F1B8004C0909FB04FA06EB0A0808F1B407BD7804
:10F1C80015B10134E4B2EEE790F9003090F804E0AC
:10F1D8001846114B03228DE8240001212A4653F8D2
:10F1E8002E30F8F7D1FD834660B106F16C0050442B
:10F1F80029464A4605F013FF01231C44C8F86CB0A1
:10F20800BB70E4B20120F8F7B9FFCCE703B0BDE862
:10F21800F08F00BF94210020F882010800212222EB
:10F2280010B5114805F0FBFE104B00221946104896
:10F238000424105C83F8F2010132052083F8F741B9
:10F24800042A4FF0000483F8F60183F8F94183F8A3
:10F25800F80103F10803EAD10123A1F8F43152239C
:10F2680081F8F03110BD00BF8426002094240020CE
:10F27800C5A1010810B5FCF737FD4FF4302401286B
:10F2880006D11CB1FCF730FD013CF8E7052010BDA4
:10F29800002C08BF052010BD70B50646441E14F8A2
:10F2A800011F89B1094D284605F0EFFE0028F6D068
:10F2B80005F1080398423FBF054B401BC018A31B2C
:10F2C80038BF80F88A31EAE770BD00BFC9A10108DC
:10F2D80094240020031EB8BF2D2210B5B8BF584291
:10F2E8000C46B8BF01F8012B0A22FAF7B7FD002334
:10F2F8000370204610BD07B51C4B03F58472C3F894
:10F3080004211B4A92F892215AB1012A14D10321EF
:10F3180083F80A11072183F80C2183F80B110C22BA
:10F3280008E0022183F80A11032183F80C2183F8ED
:10F338000B11072283F808210E4B0F4AC3F88420CB
:10F348004020F8F737FF70B10122002390F9000040
:10F3580040218DE80C00094A4FF4E133F8F714FD19
:10F36800003018BF012003B05DF804FB9421002091
:10F37800942400207C00002095B70008C1B800083C
:10F388000120002100F0F6BCF0B5184A92F80D31C2
:10F39800D2F810711546032B11D807EBC3025E1C77
:10F3A800941CF6B209D013469288D10705D51042AD
:10F3B80003D008E00131042908D13346EBE785F88A
:10F3C8000D310020F0BD93F802E00021074C0C221B
:10F3D80004F58A7C02FB01F31CF803209645E9D169
:10F3E800234484F80D61D3F81801F0BD942100205E
:10F3F8000A4B10B519684FF6FB720A401A60084AA2
:10F40800927B1C46074B0AB1052200E001221A60D4
:10F4180001F0DEF94FF43643236010BD405C004034
:10F42800942100203C2F00206C4B6D4A2DE9F04FB1
:10F438005E8914684FEA062AB4EB0A0A9C884FEAE8
:10F4480004481C894FF000054FF0000B65EB0B0BCF
:10F45800A4FB0A6704FB0B77F40944EA476418EB3A
:10F4680004065C884FF000094FEAE7154FEAC438F4
:10F47800DC8849EB050787B0CDE90467A4FB0A6778
:10F4880004FB0B77340A44EA076418EB04064FEAD6
:10F4980027259C894FF0000949EB0507CDE900674E
:10F4A800AAFB046704FB0B77F40D44EA472414F520
:10F4B800FA664FEAE75545F10007B6F5FA6F77F1B6
:10F4C8000003CDE90267964667DAA4FB046704FBEC
:10F4D80005F34FF0050C07EB4307DDE90489A6FBAC
:10F4E8000C230CFB07335F104FEA3206B8EB060813
:10F4F8004FEA920669EB070946EA83769F10DDE931
:10F508000023921B63EB0703DDE90267CDE90023C3
:10F51800344A4FF0FF33964277EB0303CDE9048971
:10F5280028DA40F6AC52A4184FF000035D4104FB02
:10F5380005F3A4FB044505EB43056FF0060266429C
:10F5480002FB0566A4FB0223334418EB020649EBD1
:10F558000307CDE904670B26A4FB062306FB053346
:10F56800DDE900455B104FEA3202A41A65EB03059A
:10F57800CDE900450AFB0BF3DDE90245AAFB0AAB1E
:10F588000BEB430B4FEADA7242EA4B02A41A4FEA3A
:10F59800EB7365EB0305CDE90245DEF80440009BFB
:10F5A800019DA4FB032304FB05334FEA52584FEA9D
:10F5B800635948EAC328DDE90423B8EB020269EB82
:10F5C80003039946D30B43EA494300B1036009B1E9
:10F5D800029B0B6007B0BDE8F08F00BFFA02002065
:10F5E800D822002024FAFFFF024B4FF480521A80E1
:10F5F800704700BF04000020772048210122F5F75A
:10F60800DBBB772058210122F5F7D6BB07B50021CF
:10F6180001AB03227720F5F753FB9DF805309DF8E1
:10F6280004001B0243EA00439DF80600184303B098
:10F638005DF804FB08B5FFF7E9FF014B586008BD0A
:10F64800D822002008B5FFF7E1FF014B186008BD7C
:10F65800D822002038B54FF09043154610221A855D
:10F6680040F080000C4601F0E9F9164B9B894FF4F5
:10F678007A73E5B1134A1289900706D4013B9BB20D
:10F688004FF6FF729342F5D10CE00F4AFF2111703B
:10F698000C490989C9070FD4013B9BB24FF6FF718A
:10F6A8008B42F5D1094A138801339BB213804FF07E
:10F6B800904310229A6138BD12780CB1227001343F
:10F6C800013DD6E7003001400C30014024240020E1
:10F6D80013B501220DF1070104463820FFF7BAFFE0
:10F6E8000520F7F797F99DF8073003B10123237038
:10F6F80002B010BD13B50622044669464320FFF741
:10F70800A9FF9DF800209DF8013043EA02232380D9
:10F718009DF802209DF8033043EA022363809DF898
:10F7280004209DF8053043EA0223A38002B010BDEF
:10F7380013B50622044669463B20FFF78BFF9DF868
:10F7480000209DF8013043EA022323809DF802201F
:10F758009DF8033043EA022363809DF804209DF856
:10F76800053043EA0223A38002B010BD70B54FF004
:10F77800904410250E46258501F060F9304601F0C9
:10F788005DF9A56170BD08B580216B20FFF7EEFF1C
:10F798006420F7F74AF900216B20FFF7E7FF6420A0
:10F7A800F7F743F96B200121FFF7E0FF1B20182131
:10F7B800FFF7DCFF1C201021FFF7D8FF044B1A20AD
:10F7C8001978FFF7D3FF19200021BDE80840CDE7DD
:10F7D800000000202DE9F0410369C76805460E4680
:10F7E8001F40002F35D0B7FA87F24FF00043D340BF
:10F7F800DB432B611F40A2F11B03042BF1D8DFE888
:10F8080003F0221F1C190300746A24B1013C002371
:10F81800A4B2736201E0EC6AA4B2D6F82080B8F111
:10F82800000FDED0D8F80030404621469847D8F877
:10F838000480F4E73068696B07E07068A96B04E03E
:10F84800B068E96B01E0F068296C036889B29847F1
:10F85800C7E7BDE8F08173B51E4C237A6BBB1E4920
:10F868004A6942F400324A611026032201254FF00A
:10F87800904069468DF805208DF806308DF80730E0
:10F8880000968DF80450FCF7EFFB4FF09043134AB5
:10F898009E61138823F04003B340F340138013881C
:10F8A80023F03803B340F34043F008031380138870
:10F8B8009BB243F0400313802572752069460122EC
:10F8C800FFF7C8FE9DF80000A0F1700358425841A8
:10F8D80002B070BDD8220020001002400030014064
:10F8E8000148024976E700BF00400140FC130020B0
:10F8F800014802496EE700BF00040040D41300200D
:10F908004FF08040004965E7AC13002001480249E8
:10F9180060E700BF002C0140841300200148024921
:10F9280058E700BF002C014084130020224B10B57B
:10F93800224C5A43224BB3FBF2F203880139013AB5
:10F94800A04289B292B29BB20ED004F50064A042E4
:10F958000AD0B0F1804F07D0A4F59834A04203D064
:10F9680004F58064A04202D123F070039BB2154CC9
:10F97800A04206D004F58064A0421CBF23F4407363
:10F988009BB203800D4BC162984202850FD003F5EC
:10F99800006398420BD003F54063984207D003F503
:10F9A8008063984203D003F58063984201D1002315
:10F9B80003860123436110BD40420F00002C014023
:10F9C80000A24A04001000400B4B800A98420DD058
:10F9D80004D8B0F5801F0BD101207047074B98421F
:10F9E80008D00533984203D103207047022070479E
:10F9F800FE20704700207047010010004B001000E7
:10FA0800F8B50468064620460F461546FFF7DCFFA2
:10FA180003284BD8B27A910847B902238B40D4F80F
:10FA28000CE0DB439BB203EA0E03E3600A23204A9F
:10FA380003FB001342F82370043342F823501546A1
:10FA48003FB1B17AE268890802238B409BB2134325
:10FA5800E360282202FB00522032EFF31286502383
:10FA680083F3128803B203EB8303DB0003F10C0179
:10FA78001C3329442B4451F8047F17B117600A68D6
:10FA880004329942F7D100231360F3B283F311884B
:10FA9800282303FB0050036A1BB1E36843F001030A
:10FAA80003E0E2684FF6FE731340E360F8BD00BF61
:10FAB800841300200148FDF7A5BE00BFE422002002
:10FAC8000148FDF79FBE00BF382300200148FDF71D
:10FAD80099BE00BF8C23002007B5064B0093064B48
:10FAE80001930649064A074B0748FAF7B8FA03B0E4
:10FAF8005DF804FBA494010879940108FEA10108AB
:10FB08000BA2010898940108DEA1010808B5037842
:10FB180033B90C4B0C481978BDE80840FAF79FBA7E
:10FB280005F018FB02280CD8064B1870074B0C225E
:10FB380002FB0030064B06301860FAF7ADFC0548AA
:10FB4800E5E708BDE023002012A201083C2C0020B4
:10FB5800B41100209297010808B503783BB90B4B04
:10FB68000B4893F8AC17BDE80840FAF778BA05F0E7
:10FB7800F1FA022808D8054B83F8AC07FAF7F6FB28
:10FB8800FAF7AEFC0348E8E708BD00BF942400205C
:10FB980016A201089297010838B5037803BB214BD8
:10FBA8001B6801330F2B07D81F490C2202FB0312D5
:10FBB8001C4695682DBB00E01C4601340F2C01DD66
:10FBC800002400E005D818490C2202FB04129568AD
:10FBD800BDB99C42F1D11548BDE83840FAF73FBAA3
:10FBE80005F0B8FA0F28044605D80F4A0C2303FB82
:10FBF80000239D682DB921460D48BDE83840FAF725
:10FC08002EBA084B1C60F6F72FFF21462A460948F2
:10FC1800FAF725FA0C235C43034B185DBDE838401E
:10FC2800F6F736BF04010020B883010823A20108B3
:10FC380039A2010851A2010873B5037813B9F7F77F
:10FC4800D5FD3DE01F4901AA05F0E5FA002401466B
:10FC58002646254699B134B1012C08D1084605F04D
:10FC680079FA064603E0084605F074FA0546154990
:10FC7800002001AA05F0CFFA01340146EAE70B2D6E
:10FC880002D911480C220BE0022C10D1A6F57A7388
:10FC9800B3F57A7F07D90D484FF47A714FF4FA62B9
:10FCA800F7F721FD0CE00A4B03EB45035E80084B98
:10FCB800084803EB45032946B3F90220FAF7CFF9C0
:10FCC80002B070BD019C0108CC990108649F01082D
:10FCD800E023002068A2010838B50D4C2368834250
:10FCE800054606D1F8F73DF8204600214C2205F0DC
:10FCF80096F9E36CAB4209D12846F8F732F8054883
:10FD080000214C22BDE8384005F089B938BD00BF54
:10FD1800002200204C220020034B1A68D379591C7A
:10FD28001344D171187A7047F812002010B5FFF704
:10FD3800F3FF84B2FFF7F0FF04EB002080B210BDA0
:10FD480010B5FFF7F3FF0446FFF7F0FF04EB0040A0
:10FD580010BD064B10B5044621461868F6F718FF83
:10FD6800034B1B6898796040987110BDFC12002005
:10FD7800F812002038B5044624200D46FFF7E9FFA5
:10FD88004D20FFF7E6FF002C084C14BF21203E2031
:10FD9800FFF7DFFF2368002228469A71FFF7D9FF93
:10FDA800236893F84900BDE83840D2E7F8120020EC
:10FDB80001460020DEE710B50446C0B2FFF7C9FFD0
:10FDC800200ABDE81040C4E710B5044680B2FFF72A
:10FDD800F2FF200CBDE81040EDE737B58288836854
:10FDE800044610060D4641BF2B4991F8AC174FF455
:10FDF800CC7000FB0133D10544BF2849097802F0D3
:10FE08003F0244BF01EB410103EB8103042A12D0F6
:10FE180006D8012A0DD0022A32D193F9001030E019
:10FE2800102A0AD0202A0AD0082A29D1B3F90010AA
:10FE380027E0197825E0198823E0196821E093ED77
:10FE4800000A6846F9F7A0FF01461548FAF707F9CE
:10FE580005B3D4ED037A6846B8EEE70AF9F794FFDC
:10FE680001461048FAF7FBF894ED040A6846B8EE24
:10FE7800C00AF9F789FF01460A48FAF7F0F809E0DD
:10FE880000210948FAF7EBF825B10848E16822692A
:10FE9800FAF7E5F803B030BD94240020E0230020F1
:10FEA8000C9B0108059B01087BA2010877A20108A9
:10FEB800024B0146D869F6F76BBE00BFE02300206D
:10FEC80010B5441E14F8011F21B1034BD869F6F789
:10FED8005FFEF7E710BD00BFE0230020F7B52B4910
:10FEE8002B4B08782B4D1C682B4B05EB80001A8890
:10FEF8002A4BD0F8C0101B78294800914FF47A712A
:10FF0800B4FBF1F1FAF7ABF826484821FAF7A7F85D
:10FF1800254B1F680026F3B205EB8302D2F8D010F8
:10FF2800E9B101249C403C4217D0220715D01F4A52
:10FF3800D25C0B2000FB0323164A1D4802EB830307
:10FF4800D3F8F020FAF78BF8022C06D1194B93F866
:10FF5800281011B11848FAF782F80136DBE717487C
:10FF6800FFF7AEFF164B17481A68174B9A420CBF9B
:10FF7800164B174B1A88174B198892B24FF4FB632C
:10FF880003B0BDE8F040FAF76AB800BFA01200203D
:10FF980058240020B88301084012002008010020DE
:10FFA8007EA20108C1A20108501200201001002001
:10FFB800D1A20108E0230020D9A2010821A3010849
:10FFC8004C110020DDA2010800540040501100200F
:10FFD80052110020481100202DE9F04100248046EC
:10FFE80025460F4EA7594146384605F09BF858B1AB
:08FFF80039460C48FAF733F812
:020000040801F1
:1000000030190021FFF7EDFE0948FFF75DFF0135CC
:10001000143440F694439C42E7D11DB90548BDE82D
:10002000F04151E7BDE8F08158850108839B010844
:1000300021A30108239A01082DE9F04F2DED028B31
:1000400083B0054605F033F8064620B1012818D1E3
:100050002B782A2B15D15C48FFF736FF00245B4D27
:100060005B486159F9F7FFFF28193146FFF7B9FEE0
:100070005848FFF729FF143440F694439C42EED1D0
:100080009CE028463D2105F004F8002800F08F8010
:100090000346994613F8012D202AFAD0441C204625
:1000A00005F05CF880462046F9F7E8FDC5EB090944
:1000B000B0EE408A0026DFF834A1142202FB06F4D9
:1000C0000AF5D07B54F80B70384604F0F0FF034675
:1000D0001A4628463946019304F0F2FF019B002896
:1000E0005BD15FFA89F29A4257D10AEB0402D2ED52
:1000F0006B7AF8EEE77A0BEB0405B4EEE78AF1EEE3
:1001000010FA48DBD2ED6C7AF8EEE77AB4EEE78AC3
:10011000F1EE10FA3FD8B2F8A431D2F8A82113F0CA
:10012000200F08BF08EE108A1C0641BF2A4991F82B
:10013000AC174FF4CC7404FB0122D90544BF274906
:10014000097803F03F0344BF01EB410102EB810258
:10015000042B18EE100A0BD004D8013B012B0ED84B
:1001600010700CE0102B05D0202B06D0082B06D1E8
:10017000108004E082ED008A01E082ED008A3946B9
:100180001748F9F770FF2846002103B0BDEC028B39
:10019000BDE8F04F25E6134803E00136A12E8AD1D1
:1001A000114803B0BDEC028BBDE8F04F8CE6284649
:1001B00003B0BDEC028BBDE8F04F11E703B0BDEC1E
:1001C000028BBDE8F08F00BF0FA30108588501081E
:1001D000839B010821A3010894240020E023002030
:1001E00024A301082FA30108239A0108B88301085A
:1001F00070B50546284604F05AFF064658B9194B13
:1002000019485A79194B03EB8203BDE87040D3F8C3
:10021000301EF9F728BF28461549324604F050FF32
:1002200060B91448144CFFF74FFE54F8041F19B17D
:100230001248F9F718FFF8E7114805E00024114BC0
:1002400053F8241019B91048BDE870403CE6284620
:10025000324604F035FF01340028F0D1014B0B4D3C
:100260005C71C7E7942400204FA30108B8830108FC
:10027000239B01085BA30108E89101081F9B01086B
:1002800021A30108EC910108239A01089297010823
:1002900008B50748FFF718FE064BD869F7F75AFD6F
:1002A000F6F7D8FDFAF73CF8034B044ADA6008BDCC
:1002B0006EA30108E023002000ED00E00400FA0531
:1002C00008B50548FFF700FE00F036F8FAF752F8D7
:1002D000BDE80840DCE700BF7AA3010808B5044880
:1002E000FFF7F2FDFAF746F8BDE80840D0E700BF97
:1002F00090A301080E4B1A78692A16D15A88B2F5D4
:10030000FB6F12D11A79BE2A0FD193F8D527EF2AA5
:100310004FF000000BD113F8012B5040054A9342D7
:10032000F9D1B0FA80F0400970470020704770475B
:1003300000F80308D8FF03082DE9F04FEF4C002127
:100340004FF4FB6285B0204604F06DFEEC4B04F5E3
:1003500039721A60EB4B00221A70EB4B04F2AE714B
:100360001960692323700323637140F20113A360B2
:100370004FF41673A4F86631FA23A4F86831BC234D
:10038000A4F864314FF4FA732021A4F86E310123EC
:1003900084F8623184F86A1184F87E316E2184F821
:1003A0008631052384F87C1184F823320A2140F237
:1003B000DC5384F87D11A4F898312B2140F24C4392
:1003C00084F87F11A4F89A31212140F26C7384F8EB
:1003D0008011A4F89C31232140F2753384F88111F7
:1003E000A4F89E314FF4C87140F64303A4F8A0313D
:1003F000A4F8821123469918023200254FF01E09F5
:10040000242ABE4C81F8A25181F8A391F3D14FF474
:10041000FA6340F27E4040F27E57DFF8E4B2A4F87F
:10042000C831A4F8CC31A4F8D031A4F8D431A4F860
:100430004401052340F23A70A4F84C7140F2EA57A7
:1004400001264FF47A78C82219214FF0320A84F835
:10045000DE31A4F846014FF4C87340F2DC50A4F832
:100460004E7140F2B457A4F8E221039284F89591BA
:1004700084F8DD6184F8DF11019184F8E06184F88B
:10048000E16184F8E461A4F8E63184F8EA61A4F853
:100490004A010290A4F85071A4F8543184F8ED6137
:1004A000A4F8C681A4F8CA81A4F8CE81A4F8D281A8
:1004B000A4F84881A4F852A1A4F856A1FEF7B2FE10
:1004C000DBF8003026744FF0170E83F815E083F840
:1004D00016E04FF0550EE673A573A58183F803E08F
:1004E0004FF00F0E83F805E00199D9714FF0220EFD
:1004F00083F806E021214FF00E0E83F80B9083F86D
:100500000C9083F810E059744FF0350E53214FF0E2
:10051000640928274FF02D0C83F81AE0D9764FF0A4
:100520005A0E0A2183F81C904FF0780983F80DC009
:1005300083F808E0997483F80A901D705F709F70CB
:10054000DD7583F804A09D731D76DD735D765F72A3
:1005500083F814C04FF4FA7CA3F84EC0DFF8C0C192
:10056000C3F838C0C3F83CC0DFF8B8C1C3F828C02E
:100570004FF07E5CC3F834C0F7EE087ADFF8A8913C
:10058000DFF8A8C1C3ED087AC3F82C90C3ED097A4F
:10059000C3F83090C3F848C0F1EE047A02989E7711
:1005A0004FF04B0C4FF0000983F8501083F8525075
:1005B00083F85170C3F84090C3ED117A83F84CC0B2
:1005C00084F8AEE7A4F8B8074FF0410E042084F891
:1005D000AFE784F8B0A784F8B15784F8B55784F82A
:1005E000B65784F8B25784F8B35784F8B45783F8F1
:1005F0005C0015200191A3F85850A3F85A50A3F8B5
:100600005650C3ED187A83F868004048D8664048D1
:1006100018674048586783F878603F4883F86470EB
:1006200083F86570FEF73CFEDBF800300199039A11
:1006300083F814614FF4487083F8115183F8125114
:1006400083F8137183F81851A3F816015E4684F8F5
:10065000D81184F8D921A4F8DA8119460E2202FBB8
:1006600005326FF0170082F81901032082F81A0191
:100670006FF02F0082F81B01072082F81C016FF039
:10068000230082F81D01052082F81E0101355A2041
:1006900081F8200181F821016422FF20082D81F8D2
:1006A0001F2181F8220101F10E01D7D1002183F829
:1006B0008911C821A3F88A11142183F88C11A3F899
:1006C00090211E214FF4967283F88D11A3F8922188
:1006D00001212822A3F8942183F88E11074B03F1FE
:1006E000C0021F46C3F8149010339342FAD10B484E
:1006F0000021402204F097FC1AE000BF942400205F
:1007000090110020E0230020B41100209A99193F95
:10071000F6287C3F3D0A773F45AE01083827002088
:100720008FC2F53C00002040CDCCCC3E00004040C4
:100730000023264D264C5959FA1804330868C2F88C
:10074000A402382BF5D104F509700021802204F0B1
:100750006AFC05F13801702204F5097004F058FCB8
:10076000FDF732FF366800230125314604F27C4054
:100770004FF4CC7284F8D43784F8D25784F8D35726
:1007800004F046FC04F2146031464FF4CC7204F0DD
:100790003FFC104B1B681A68C4F8BA275A68C4F8A3
:1007A000BE279A68C4F8C2271A68C4F8C6275A68D0
:1007B000C4F8CA279A68C4F8CE27022384F8D05414
:1007C00084F8683605B0BDE8F08F00BFB492010828
:1007D00094240020B41100201549D1F8883043F446
:1007E0007003C1F88830134B1A6842F001021A6096
:1007F0005868114A02405A601A6822F0847222F442
:1008000080321A601A6822F480221A605A6822F430
:10081000FE025A60DA6A22F00F02DA62186B074AA7
:1008200002401A6300229A604FF000638B607047A9
:1008300000ED00E0001002400CC07FF8CCFC00FF8F
:1008400038B5094B93F8D45765B9084C2068F7F7C9
:100850008CFA074B25601B78022B03D1BDE838408A
:10086000FEF79FBC38BD00BF942400207C2C0020E4
:10087000782C0020044B93F8D4371BB9034B18682D
:10088000F6F77EB900207047942400207C2C0020CD
:1008900038B505460446204614F8011B21B1034B28
:1008A0001868F6F779F9F6E7401B38BD7C2C002074
:1008B0000FB407B504AB064953F8042B019300208D
:1008C000F9F7E4FA03B05DF804EB04B0704700BF39
:1008D0003F0A0108024B01461868F6F75DB900BFF0
:1008E0007C2C0020F8B5011F06460023083051F883
:1008F000042F02F120043F2C3AD802F108040F2CF7
:1009000006D80232032A04D9002B08BF012300E0D5
:1009100002238142EBD1012B30680ED0022B1AD07A
:10092000736803F003039B0000F0030043EA001028
:10093000B36803F00303184317E000F00F0040F022
:100940004000FFF7C7FFB068736800F00F0040EA8F
:100950000310C0B209E000F03F0040F08000FFF754
:10096000B9FF3079FFF7B6FF307ABDE8F840B1E75C
:1009700006F10C0734463A46002552F8043D03F1CF
:100980008001FF294FEA850510D903F50041B1F533
:10099000803F02D245F0010508E003F50003B3F102
:1009A000807F34BF45F0020545F00305B242E4D133
:1009B00065F03F00C0B2FFF78DFF05F00303022B87
:1009C000207807D0032B0CD0012B13D1FFF782FF27
:1009D00060780FE0FFF77EFF6078FFF77BFFA0787D
:1009E00008E0FFF777FF6078FFF774FFA078FFF764
:1009F00071FFE0780434FFF76DFFBC424FEAA505B4
:100A0000DBD1F8BD10B50446C0B2FFF763FFC4F3F5
:100A10000720BDE810405DE710B504467F2C06D9DD
:100A200064F07F00C0B2FFF755FFE409F6E7E0B2DB
:100A3000BDE810404EE7430083EAE070ECE708466B
:100A400048E700BF40F2E9330F4A1289920704D405
:100A5000013B9BB2002BF7D10BE00C4A40F2E9338B
:100A6000107009490989C9070AD4013B9BB2002BC0
:100A7000F7D1074A138801339BB21380FF207047D8
:100A80001078C0B2704700BF003001400C30014008
:100A9000242400200C4B0D49DA684378D243C2F37A
:100AA0000222C2F10402934002781B010A44DBB225
:100AB00082F8003303780122580903F01F0302FA79
:100AC00003F341F82030704700ED00E000E100E062
:100AD00073B50546002100680122FEF72BFF2A6846
:100AE00013889BB243F001031380EB7A8DF8043036
:100AF0000124002601A88DF805408DF806608DF8C8
:100B00000740FFF7C7FFEB7A1B2B0BD1192301A876
:100B10008DF804308DF805408DF806608DF807409B
:100B2000FFF7B8FF02B070BDF0B5BE4CA3782DED55
:100B3000028B013B012B85B000F26F81E578854285
:100B400040F06B812379022B00F06781B64B5B5D2F
:100B50006371A3796D00F2EE048A1BB16319B3F9D6
:100B6000083009E06319D4ED037AB3F90830F1EEE7
:100B7000677AC4ED037A5B4208EE103A2369A94E06
:100B8000B8EEC88A1A0388EE288A35D5D6ED037ADE
:100B9000FDEEE77A28EE280A17EE903AD6ED057AB0
:100BA0008DF80A30FDEEE77A17EE903A8DF80B30AB
:100BB00004F08EFCFCEEC07A96ED060A17EE903A31
:100BC00020EE280AADF8083004F082FCFCEEC07A72
:100BD00096ED070A17EE903A20EE280AADF80C3091
:100BE00004F076FCFCEEC07A0C2017EE903A02A9D5
:100BF000ADF80E30F7F7B0FCD4ED077A894BF5EE7F
:100C0000407AF1EE10FA60D1D3ED067AB4EEE78ABD
:100C1000F1EE10FA04DDDA6883ED068A5A61E8E045
:100C2000F5EEC07AF1EE10FA40F3E38093F820205D
:100C300042B1022A00F2DD805A6B83ED078AFA3254
:100C40009A63D6E0D3ED037A38EE678AF7EE007A3E
:100C5000B4EEE78AF1EE10FAACBF01210021D3ED2A
:100C60000A7A69B19FED717A27EE877ADFED707AA3
:100C7000B4EEE77AF1EE10FA58BFF0EE477A03E0EF
:100C80009FED6C7A67EE877AC3ED0A7A2369654A2D
:100C90001B0311D58DF808105379116B0B440B20F1
:100CA0005A788DF80920DA7A8DF80A205B7D8DF864
:100CB0000B3002A9F7F750FC0123226B84F8203097
:100CC000637913440022DA7291E0B4EEE78AF1EE20
:100CD00010FA48BF83ED078AA16B636B94ED067A27
:100CE000D4ED076A591AC943C90F77EE667A59B924
:100CF000B7EE006AF4EEC67AF1EE10FA79DDB4EEE2
:100D0000E68AF1EE10FA74DDD4ED056A454BB4EED7
:100D1000E67AF1EE10FACCBF0126002666B1D3EDDB
:100D2000097A9FED427A67EE877A9FED427AC3EDAA
:100D3000097AD3ED0B7A0AE0B0EE007AF4EEC77AC6
:100D4000F1EE10FA08DDD3ED0B7A9FED387A67EEFD
:100D5000877AC3ED0B7A07E0D3ED097A9FED357AF8
:100D600067EE877AC3ED097AD4ED097A206B627950
:100D700067EEA87A1044FCEEE77ACDED017A9DF893
:100D800004304370D4ED0B7A2769FCEEE77A3F0319
:100D9000CDED017A9DF8042042750ED546EA410159
:100DA0008DF808108DF80930C37A8DF80A300B20C1
:100DB00002A98DF80B20F7F7CFFB94F82020194BF0
:100DC000022A11D1D3ED0A7A9FED1B7A196B67EED7
:100DD000877A002283F82020FCEEE77A5A7917EE12
:100DE000903A0A44D37202E0022283F82020F8F7F6
:100DF00085FEA2790B4B0AB1104A00E0104ADA6076
:100E00002544D4ED037AB5F9083000EE103AB8EE77
:100E1000C00A80EE280A37EEC00A05B0BDEC028B8E
:100E2000F0BD00BF242400208C930108EC51783FD2
:100E30006F12833A0AD7833F00007A440000A04132
:100E40000000A0C12B4BF0B52B4D1E6805F1100022
:100E50002F78F3192C46597801F00401013501F07F
:100E6000FF0219B18542F3D10020F0BD224D631B72
:100E7000022B0ADD1AB102EB82025200D2B215F83F
:100E8000013B303B1A44D2B2F1E70021AC420AD90F
:100E900019B101EB81014900C9B215F8013B303BA2
:100EA0001944C9B2F2E72E2F16D1013404200023D1
:100EB0002578771903EB83037F785B007F079BB26C
:100EC00044BF303D5B1900F1FF3044BF01349BB299
:100ED00010F0FF00ECD100E00023084841436420FB
:100EE00000FB03130620B3FBF0F3054800FB0230C0
:100EF000F0BD00BF180100206024002040420F0018
:100F00008096980030B500231A4610498C1894F842
:100F10003C40BCB12E2C06D1013298B18C1804444F
:100F2000002584F83C5011440A2491F83C10634396
:100F3000A1F13004092C9CBF303B5B180E2A03D86A
:100F40000132E2E7184630BD002030BD24240020E5
:100F50000EB40FB50749019006AB01A8064A0393EA
:100F6000F8F794FF019B00221A7004B05DF804EBBF
:100F700003B07047BD9B0008179C01080B4A13691A
:100F800013F4805FB2F9523006D0B2F80822111A79
:100F90008B4208DD104401E0B2F80A028342B4BF7C
:100FA0000020012070470120704700BF242400204A
:100FB0002DE9F04FAB490B7813F0010F87B003F028
:100FC000040200F07181002A40F07B8103F00200EE
:100FD00000F0FF04002840F0678143F004030B7029
:100FE000A14BA24F1A88A24B1A803B681B0340F109
:100FF0001981A04B80201C70FEF7CAF908B1FEF7DA
:101000006FFE9D4C2678012E40F00C819B4B93F88F
:10101000D21721B193F8D3270AB1914203D3012209
:1010200083F8D2270FE01546084635B190FBF5FE50
:1010300005FB1E0E28467546F7E791FBF0F183F895
:10104000D21792FBF0F283F8D32793F8D4271AB182
:101050008A4A002182F8D417626893F8D45702EBC9
:10106000C20241F669018A4284BF40F2E241B2FB0A
:10107000F1F283498CBFD2B204220A70FDB98020FC
:10108000F7F79CF88046D0B18021F7F771F898F80F
:1010900006207C4B207253F8223098F90000DFF8CC
:1010A000D881B3F5613F0CBF0222002202218DE8F6
:1010B000060080212A46F6F76BFEE06008B900239F
:1010C000AFE008F110002946142203F0ACFF08F14C
:1010D0003003C8F8243008F1A403C8F8283008F514
:1010E0008C73C8F82C30684B68491B88A8F88C3181
:1010F000624B086893F8D2C7597993F8D32793F8CD
:10110000869193F89431A1F1190E944528BF4FF0C0
:10111000000C3A6838BF4FF0010CDEF1000747EBD6
:101120000E07012914BF39460121594F0491002BA4
:10113000584BD7F800E01B78039302F40068C2F321
:10114000400BC0F3800AC2F3C032C0F3C00018BF26
:1011500001220597711EC9B24B1E132B3DD8DFE843
:1011600003F00C0C0C0C0C0C0C0C0AAAAC292B3F39
:1011700037121212393F049BA0E0039B8B42B4BF8D
:101180000023012328E09EF80030022B0BD10EEB48
:10119000810353ED027AF5EE407AF1EE10FA14BFB6
:1011A0000123002318E00EEB01035B79003318BF25
:1011B000012311E05B4681E0B8F1000F04D009F192
:1011C000FF377B427B4100E0434603F0010375E0BB
:1011D000134673E0634671E013B101238B401D4356
:1011E000142E02D80136F6B2B4E7059BC4F890512C
:1011F000186819217930F5F7BBFB0023C4F8983142
:10120000A4F89C31A4F89E31C4F8A831224BD4F83C
:10121000A4211B68C4F8AC3184F89401C4F8A0215F
:10122000022323701C4B154A1B6892F8DE214FF4F1
:101230007A7101FB0233194A13600C4B1B681A06C2
:1012400009D5174B1B789B0705D5164B1B78042B2C
:1012500001D9062000E0052007B0BDE8F04FF5F702
:101260001BBC00BF562F00202C120020342400206D
:101270007A0F0020A1220020702C0020942400204E
:1012800014010020F88201081C19002050120020CF
:10129000901100208013002058240020340F0020DB
:1012A000541200205A1200205AB9012007B0BDE89C
:1012B000F04FF5F713BC034600E05346002B8CD1EA
:1012C00090E707B0BDE8F08F10B5154A13785907BD
:1012D00025D523F004031370124B1B681B0319D58B
:1012E000114C2378A3F10802012A0BD8FF2000211A
:1012F000F7F732F90D4B1B68C4F8AC31FFF7BAFAB7
:101300000A2306E0012B05D90A2B03D0FFF798FA30
:10131000012323700420BDE81040F5F7BDBB10BDCC
:10132000562F002034240020702C00205824002048
:10133000064B1B7803F0040303F0FF001BB1044BC2
:101340001888C0F3C01000F001007047562F00202D
:10135000181300202DE9F04F2DED028B87B00026E9
:101360000493B24B0392B3F90270B3F900300190C9
:10137000002FB8BF7F42002BB8BF5B429F42B8BF6F
:101380001F46B7F5FA7F8146A8BF4FF4FA77B046FB
:101390000296B3463446A64D2B8813F0030F4FEA4E
:1013A000440A58D0022C56D0A04BA24A33F80A3037
:1013B00032F90A20022113FB0122039B5B429A426D
:1013C00003DB039B9342A8BF13469B4A32F90A20D2
:1013D0009B1A049A32F91420134408EE103AFFF7CE
:1013E000A7FF68B1B8EEC80A944BB2EE048A80EE4B
:1013F000080A185DFFF798FB20EE080ABDEEC08AC8
:1014000018EE102A99F808305343642293FBF2F344
:1014100099F81C206FF0040B0BFB02FB5B4504DB0F
:1014200002EB820B9B45A8BF9B46854918EE103AFC
:1014300051F82420134442F210729342A8BF13467D
:10144000804A9342B8BF134699F8122041F82430DD
:1014500053431B1302932B8803F00302012A01D18B
:10146000022C3FD17848714A30F90A0032F90A80DB
:101470007649019A51F82460557880EAE07EAEEB17
:10148000E07EBEF5206F4FEA84021EDC022C15D0F0
:1014900008EB8801090191FBF5F5042190FBF1F0BF
:1014A0002D1A2E44B6F57A5F68496948A8BF4FF4F3
:1014B0007A568642ACBF5650505008E088EAE87E23
:1014C000AEEBE87EBEF1640FE2DD002088505F499C
:1014D0007D26525892FBF6F6019AD27A7243402644
:1014E00092FBF6F69A0713D5022C11D00298C7F595
:1014F000FA7307FB06F507FB08F203FB0B224FF418
:10150000FA7103FB005392FBF1F293FBF1F508E053
:10151000DB0704D5022C02D0029D5A4601E0354675
:101520004246494B33F91410042391FBF3F3494924
:10153000615C4B436FF04F0193FBF1F399F851104D
:10154000D3184FEA440A08EE103AB1B1022CB8EEB3
:10155000C80A414B08D14A0803D09142A8BF11469E
:1015600000E001213D4802E03D4800EBC400D3ED1E
:10157000000AF8F759FBBDEEC08A334B394A3AF8F6
:1015800003003AF902302AF8020001B202F1080021
:101590001432CB1A50F824E0042193FBF1F152F8F5
:1015A000243040F8241073440B4499F8501042F84A
:1015B00024E04FEA840C00EE103A79B1264B2A4819
:1015C000D3ED000ACDF814C0B8EEC00A00EBC40099
:1015D000F8F72AFBDDF814C0BDEEC00A234A2449FF
:1015E000125D10EE103A5343202293FBF2F318EEF3
:1015F000102A2A44D21A2AF801201E4A18EE101A7C
:101600004CF802101C4A4CF802501C4A5B424CF841
:101610000230019B01340133032C01937FF4BBAEF4
:1016200007B0BDEC028BBDE8F08F00BF3412002084
:1016300018130020502F00202C2400207C82010849
:101640003C1A0020F0D8FFFF74110020C8190020B8
:1016500080C1FFFF441A0020C4190020BC190020DB
:10166000AC190020242E0020F81900205C1A00205C
:10167000101A0020181A0020241A0020301A002006
:101680002DE9F04F2DED088BC94F83B00446009330
:101690003B88019713F0020F0AEE102AF7EE009A2A
:1016A0004CD0149BC348DD89B0F900305B1B03F2BA
:1016B000F31640F2E632964203D8002BB8BF5B42E5
:1016C00001E04FF4FA73B0F90220521B02F2F31555
:1016D00040F2E630854203D8002AB8BF524201E00A
:1016E0004FF4FA7294F84C0058B39342B8BF1346C3
:1016F000C3F5FA7307EE903A9FEDAF7AF8EEE77A0A
:101700006423C7EE877A93FBF0F307EE103A77EE87
:10171000E97AB8EEC77AB0EE699AA7EE879AF7EE43
:10172000006AB5EEC09AF1EE10FA0AD4B4EE669AE9
:10173000F1EE10FAC8BFB0EE669A04E0B0EE699A16
:1017400001E09FED9E9ACE1C25464FF0000ABAF1AB
:10175000020F16F801BF9A4F4FEA4A09F2EE04AAA7
:101760000ED1B7F904209FED977A0BF10A0B02FB1B
:101770000BF307EE903AF8EEE77AC7EE877A68E067
:10178000F8EE4A7A9FED8C6A37F91A30C7EE867AFE
:1017900006EE903A8C4B33F91A3007EE103A1AEEF7
:1017A000103AF8EEE66AB8EEC77A5B42A6EEA77A80
:1017B00007EE903AF8EEE77AB4EEE77AF1EE10FA37
:1017C00008D4F8EECA7AB4EEE77AF1EE10FAD8BF90
:1017D000F0EE477A7D4B33F9093008EE103A009B62
:1017E000B8EEC88A33F91A3077EEC87A08EE103AA4
:1017F000B8EEC88A37EE888A88EE2A8AFFF798FD05
:1018000040B1734B13F80A00B0EE480AFFF78CF9A9
:10181000B0EE408A019B1A88D10704D5D4ED117A25
:1018200068EE277A15E037F909309FED667A0BF1FB
:10183000140B03FB0BF307EE903AF8EEE77A9307ED
:10184000C7EE877A42BF94ED127A28EE078AE8EE57
:10185000097A604BDFF8ACB133F9093095ED08BA7D
:101860009FED5D8A94F85110DFF89C8107EE103AE5
:101870005A4BB8EEC77AD3ED046A1AF80B30E7EE8C
:10188000667AF0EE48BAF0EE678A67EE8B7A0BEE76
:10189000103AB8EECBBA27EE8BBA8BEE08BAC1B1CC
:1018A000BAF1020F0AD14B0803D09942A8BF1946DA
:1018B00000E00121B0EE4B0A494804E04948B0EE8F
:1018C0004B0A00EBCA00D8ED000AF8F7ADF9B0EE0C
:1018D00040BAD8ED000A444995ED0B7A4FEA8A07E1
:1018E00068EEA07A394467EE877A91ED007AA7EE28
:1018F000AA7ADFED3E7AB4EEE77AF1EE10FAF0EE76
:1019000047AA09D4DFED3A7AB4EE677AF1EE10FA1D
:10191000C8BFF0EE67AA01E0F0EE67AA89EEA07AF0
:10192000344AC1ED00AAD119D1ED007AC1ED008A87
:1019300078EEE77A02F10C013944183267EE877AC3
:101940003A4491ED007A92ED000AC1ED007A82ED01
:10195000007A37EE000A94F8501030EE270A21B1D1
:10196000254800EBCA00F8F75FF9F0EE087A80EE40
:10197000270A1BF80A30D5ED0E7A08EE103A60EE11
:10198000277AB8EEC88A27EE880ADFED1C7A80EE47
:101990002B8AB4EEE78AF1EE10FA37D4DFED187A2D
:1019A000B4EE678AF1EE10FAC8BFB0EE678A2FE096
:1019B00018130020702400200000FA4300000000EB
:1019C0003412002000004842502F00202C24002018
:1019D0007C820108741100200000C842A414002079
:1019E000BC190020AC190020841A002000007AC322
:1019F00000007A43442E0020F8190020000096C30E
:101A000000009643A8190020C4190020B0EE678A90
:101A10003BEE2A0A0AF1010A30EE080A03F012FD31
:101A2000144AB0F57A7FA8BF4FF47A709042B8BFDD
:101A30001046BDEECBBA104A1BEE103A22F8090050
:101A4000FDEEEAAA0D4ABDEEC88ABB500C4A1AEE5A
:101A5000903ABB500B4A18EE103ABAF1030FBB5044
:101A600005F104057FF473AE03B0BDEC088BBDE84F
:101A7000F08F00BF18FCFFFF101A0020181A00207A
:101A8000241A0020301A0020044B00221A605A60E9
:101A9000034B00221A605A60704700BF3C1A0020B6
:101AA000901A0020022803D0431E58425841704724
:101AB000064B1B681B7823B1054B1868C0F3C04068
:101AC0007047044B1878C0F3800070475806002018
:101AD00054110020562F002010B50A4C5E280146F4
:101AE000206805D15D21F5F757F820683E2105E013
:101AF0005D2903D1F5F750F820683D21BDE810407D
:101B0000F5F74AB8682E002030B50028104C114A6D
:101B1000B8BF40423C2590FBF2F304FB030068434E
:101B20000D4D90FBF2F22D682D7B25B903EB83035D
:101B300003EB830301E0C3EB031302EB83030B808E
:101B400004FB02024FF47A7392FBF3F24A8030BD39
:101B5000806967FF809698004412002010B5044603
:101B6000C0B2FFF7B9FFC4F30720BDE81040B3E7E8
:101B7000024B5E211868F5F70FB800BF682E0020F1
:101B800038B5064C05465E212068F5F705F8206853
:101B90002946BDE83840F4F7FFBF00BF682E00209B
:101BA000674B73B51878674DFFF77CFF2B7883423E
:101BB000044620D0C8B1644B1B68E3B193F9000020
:101BC00002230093614B1B685B78003318BF01232D
:101BD000019304214FF416530022F6F7D9F85C4B19
:101BE000186040B101232B7005E0594E3068F6F7BC
:101BF000BCF834602C70574B574D1878FFF752FFE4
